:020000040800F2
:1000000000000110E90907089D2B0008F96D02089E
:10001000890A0708890A0708890A070800000000FA
:100020000000000000000000000000002D4A000851
:10003000314A000800000000354A0008F1080108B4
:10004000890A0708890A0708890A0708890A070828
:10005000890A0708890A070821CC000825CC00086E
:10006000890A070829CC00082DCC0008B532000801
:10007000C9320008DD320008F132000805330008FB
:10008000193300082D330008890A0708890A070870
:10009000890A0708890A0708890A070831CC000875
:1000A0006131000889310008B13100084D31000884
:1000B000D9310008ED31000801320008890A07082B
:1000C000890A0708890A0708890A0708890A0708A8
:1000D000890A0708052D0008112D0008890A07085C
:1000E00035CC0008890A0708394A00083D32000863
:1000F000653200088D3200082932000841330008BB
:10010000890A07088137000815320008890A07089C
:100110001D2D0008890A0708890A0708890A0708A7
:1001200055330008693300087D3300089133000817
:10013000A5330008890A0708890A0708890A0708F9
:10014000890A0708890A0708890A07088D4A0008EA
:10015000B9330008CD330008E1330008292D000829
:10016000890A0708890A0708890A0708890A070807
:10017000890A0708890A0708890A0708890A0708F7
:08018000890A0708890A070833
:10019000D0E907239A422FBFD01AC0688018C01A2E
:1001A000704700BFD0E9092300699A4238BF12188E
:1001B000D31A0138C01A7047D0E90902101AB0FAF0
:1001C00080F04009704700BF0246036A4069D16869
:1001D000C05C01338B4228BF00231362704700BF0D
:1001E000436A8269D154436A0169426B01338B428D
:1001F00028BF00234362D36843F08003D360704775
:10020000436B188810F0100002D01A889B880120D8
:10021000704700BF436B99891A88890610B5044658
:100220000AD592B2900607D5E26A002A29D09888AA
:10023000216B80B29047636B99891A88090692B244
:100240000FD510060DD5D4E909128A4214D0A16940
:100250002069895C99800132B2FBF0F100FB112228
:10026000A262998A1A88C90592B204D5D20744BFFE
:100270004FF6F7721A8010BDDA6822F08002DA6059
:10028000EFE79B88E2696169DBB28B54E269E16860
:10029000636B0132B2FBF1F001FB1022E261CBE7AC
:1002A000036942681F2B10B40AD95468A3F1200CCB
:1002B000202101FA0CF1214207D15DF8044B70476F
:1002C0001468202199402142F7D081690024C86830
:1002D0000C7480684C68016821F00101016020689D
:1002E00094F805C00C4C818934F81C4089B221EA8D
:1002F00004011F2B818107D9A3F1200120238B400A
:100300005DF8044BD3607047202101FA03F35DF8D8
:10031000044B9360704700BFBC8507084B1C10B4AA
:1003200008BF4FF0800C4D4C18BF4FF0450C4FF4F8
:10033000003300E003B3626B12EA0C0F03F1FF33EA
:10034000F8D0002923DD626B52071CD403291ED08C
:10035000424A536B13F0010320D1022908D01369DC
:10036000DBB283421ED1012953692AD006291BD052
:1003700000205DF8044B7047002904DD636B5C07C7
:1003800001D40329E4D103205DF8044B7047002B0E
:1003900014BF002003205DF8044B704701205DF876
:1003A000044B70471020EFE713F4604F04BF2C4A52
:1003B0001360990431D45A04F4D41B04D8D50F2007
:1003C000E2E7284818400028DED0002B29DB5C003B
:1003D00025D4980029D4D90025D41A0129D45C0148
:1003E00025D4D8012FD41902E9D45A02DAD49C02B8
:1003F00027D4D8022FD419030FD45A0329D49C032D
:1004000025D4D80321D4190419D45A0415D49C0432
:1004100011D41807ACD51A20B6E71320B4E7092089
:10042000B2E71C20B0E70B20AEE70A20ACE70D20B6
:10043000AAE70C20A8E71920A6E71820A4E71720B0
:10044000A2E71120A0E70E209EE716209CE71520CA
:100450009AE7142098E7122096E700BF002C01408D
:10046000301D002008E0FFFDF8B5154DEB6A93B193
:10047000696B0129044614D0124BDA6A22F0080293
:10048000DA6240F2FF5100229963EA62236823F0A6
:1004900001032360F8BD0B4AD36B43F48073D3632D
:1004A000F8BD084E40F2FF570023B763B36040F237
:1004B0004C43F3600C20FFF731FFB763DCE700BF6C
:1004C000301D0020002C0140B34BD3E9011270B560
:1004D0008C0F83F83840C1F3836483F83940C1F34B
:1004E000016483F83A40100EC1F3074483F83B409F
:1004F0000001C1F30724C9B283F83C4083F83D10E2
:10050000D887D98FC2F3035089B20143C2F30344A1
:10051000D987C2F3C03083F84040C2F34031C2F300
:10052000803483F8410083F8424083F84310C2F3DB
:10053000003183F8441093F8901000200129C2F391
:10054000072C83F8450040F2D880022900F0B180E2
:10055000D9682A204FEA4C0C0CF07E0C83F85140ED
:1005600083F852C093F85240C1F3C01214431A6981
:1005700083F8524001F07F01D40F83F8531083F8C1
:100580005440910DC2F3417483F8554001F00C01C1
:10059000C2F3826483F8564083F8571093F85710DB
:1005A000C2F381542143C2F3405583F8571083F8B6
:1005B0005850002583F85950C2F3004583F85A502B
:1005C000C2F3C03583F85B50C2F3803583F85C50CA
:1005D000C2F3403583F85D505C69C2F3003583F89F
:1005E0005E50C2F3812583F85F50C4F30741C2F324
:1005F0000125C2F3460283F860504FF0010C83F8E6
:1006000061200902220E83F862C083F86420A3F8F7
:100610006610B3F86610C4F3072289B211432406AA
:10062000A3F8661099699C669A6E0C0E42EA044221
:100630009A669C6E0A0A02F47F4222439A669D6E75
:10064000DA69C1F307242C43C9B29C6683F86C10A5
:10065000110E83F86D10110C090619671C6F110239
:1006600001F47F0121431967196F120292B20A4304
:100670001A67196F1A6A41EA1261196793F87410C0
:10068000C2F30354214383F87410110A01F470611A
:10069000A3F87610B3F87610C2F3072489B2214389
:1006A000C2F34602A3F8761083F8782083F879C065
:1006B00070BD120402F47C129A64D9689A6C0C0E14
:1006C00042EA04229A649C6CC1F3074222439A6472
:1006D0009A6C013240F10004A40244EA925492025E
:1006E000C3F880204FF40072C3F88440C1F3072C94
:1006F000C3F88820C1F380342CE74FEA8C2C0CF42B
:1007000040619964996C920002F47F720A439A6482
:100710009C6CD96844EA91749C64C1F3C265C1F3CE
:10072000026483F84C50CA0B83F84D40C1F3425425
:1007300083F84E4002F00602C1F3824483F84F4032
:1007400083F8502093F85020C1F3C034224383F83B
:1007500050209D6C93F8502093F8404002F1020E17
:10076000012202FA04F602FA0EF24FEAE27EA2FB3E
:10077000062406FB0E4405F1010EA2FB0E2E05FB1E
:1007800004447444C3E92024C1F3072CC3F88860EF
:10079000C1F38034DEE600BF301D00202F4B1A6805
:1007A000910102D59A6D52074BD42C4B1A68500216
:1007B00002D5DA6E11063CD4284B1A68D20102D554
:1007C0009A6D90072DD4254B1A68510102D59A6D68
:1007D000120717D4214B1A68120112D59A6DD00650
:1007E0000FD59A6D510334D49A6DD20503D49A6D06
:1007F00022F010029A65194B19484FF000629A6076
:1008000032E670479A6D500307D49A6DD10503D430
:100810009A6D22F008029A65104B4FF080629A6040
:10082000D8E79A6D4FF0807122F002029A659960C4
:10083000C9E7DA6E4FF4800122F08002DA6699602F
:10084000BAE79A6D4FF0007122F004029A65996040
:10085000ABE74FF000629A60704700BF006402404F
:1008600058640240384B5A68110303D5D3F8A020CE
:1008700052075BD4344B5A68D00303D5D3F8B42065
:10088000110649D4304B5A68520303D5D3F8A0203F
:10089000900737D42C4B5A68D10203D5D3F8A02047
:1008A00012071CD4284B5A68920217D5D3F8A020FF
:1008B000D00613D5D3F8A020510341D4D3F8A020FB
:1008C000D20505D4D3F8A02022F01002C3F8A0204E
:1008D0001D4B1E484FF40012DA60C5E57047D3F88F
:1008E000A02050030AD4D3F8A020D10505D4D3F812
:1008F000A02022F00802C3F8A020134B4FF480126E
:10090000DA60CFE7D3F8A0204FF4802122F0020272
:10091000C3F8A020D960BDE7D3F8B4204FF48031EC
:1009200022F08002C3F8B420D960ABE7D3F8A0204E
:100930004FF4002122F00402C3F8A020D96099E707
:100940004FF40012DA60704700640240A064024075
:1009500082B00922274B8DF80720DA68D00319D41A
:10096000DA68D10640D4DA68D20541D4DA6812F0E8
:10097000E00F3BD1DB6813F0020F14BF08230923FB
:100980008DF807309DF80730012B0AD09DF807003D
:1009900002B0704701238DF807309DF80730012B16
:1009A000F4D1144A12E0D368DB0519D4D36813F0EC
:1009B000E00F17D1D36813F0020F14BF08230923E7
:1009C0008DF807309DF80730012BDFD1D168C803BF
:1009D0004FF00103F4D4D368D906E4D50623EFE73A
:1009E0000223EDE70723EBE70623D4E70723D2E74B
:1009F0000223D0E7003C0240704700BF704700BFB1
:100A000001207047044BD3E92503984288BF03F5C2
:100A10000063181A704700BF301D0020064AD2E953
:100A200025318B42FDD0D1180133C3F30A0391F86D
:100A30009C00C2F894307047301D0020064BD3F85C
:100A40009C0800B97047D3F89C08A0F10500B0FAE3
:100A500080F04009704700BF301D0020012380F85E
:100A600049307047064BD3F8A008D3F8A428431E9A
:100A700090428CBF002001209B1A03EBC0207047DE
:100A8000301D002010B5D0F8E83504461B699847A2
:100A9000032384F81231002010BD00BF08B50422E2
:100AA00090F81211D0F8E83580F8131180F812216F
:100AB000DB689847002008BD08B5D0F8E435DB694D
:100AC00003B19847002008BD08B5D0F8E4351B6A8B
:100AD0009847002008BD00BF08B5D0F8E4355B6A30
:100AE0009847002008BD00BF037830B403B3044624
:100AF000C0F1010C04EB0C0314F8015FDBB2002D14
:100B0000F8D101335B00DCB2138003230C704B700F
:100B100004785CB1022300255A1CD2B2CC548D5407
:100B200010F8014F0233DBB2002CF5D130BC704716
:100B300002242346E8E700BF10B5074C2068FF28D1
:100B400008D00649D1F8A82801F6AC0100F080F8D9
:100B5000FF232360002010BD00000020301D002076
:100B6000432301480B8070470400002012230148F2
:100B70000B80704748000020042301480B80704719
:100B80005C00002008B5044B04480A461946FFF7EC
:100B9000ABFF084608BD00BFE42500206424080818
:100BA00008B5044B04480A461946FFF79DFF08465E
:100BB00008BD00BFE42500207824080808B5044BD0
:100BC00004480A461946FFF78FFF084608BD00BFD4
:100BD000E42500208024080808B5044B04480A4690
:100BE0001946FFF781FF084608BD00BFE425002035
:100BF0008C24080808B5044B04480A461946FFF738
:100C000073FF084608BD00BFE425002098240808AB
:100C1000704700BF704700BF704700BF704700BFFC
:100C2000704700BF704700BF044B00200522C3F887
:100C30009C28C3F8B409C3F8B8097047301D0020D8
:100C4000024B0020C3F89C08704700BF301D0020F5
:100C5000212838B50C4605D022282DD0202813D0C5
:100C6000002038BD0029FBD0072AF9D1194BD3F851
:100C7000BC0993F8C01993F8C12993F8C2392060D0
:100C800021716271A371EBE70029E9D0072AE7D14E
:100C9000104DD5F8B83913B109680020984720687D
:100CA00021796279A379C5F8BC0985F8C01985F85E
:100CB000C12985F8C239D3E70029D1D0022ACFD182
:100CC000044BD3F8B439002BCAD0098800209847C8
:100CD000C6E700BF301D002010B4144CD4E9252312
:100CE0009A4286BF03F5006CACEB02029A1A0A44E2
:100CF000B2F5006F14D8B9B101444A1E013810F89A
:100D000001CFE118824203F1010381F89CC0C3F3D3
:100D10000A03F4D1C4F8983000205DF8044B704702
:100D200002205DF8044B70470846F6E7301D0020AE
:100D3000034B93F8E809003818BF0120704700BF43
:100D4000301D002070B5124D124C296840F2FF563C
:100D500040F24D430022A6630D20A160C5F8E429AE
:100D60000121E360FFF7DAFAA66320B96369C3F3F0
:100D70004323042B08D0D5F81C3AC5F8D8390922EA
:100D800085F8E829002070BD85F8E839022070BD9B
:100D9000301D0020002C014070B50F4D95F8E8394A
:100DA000042B04460E460BD0082B07D1D5F8E039AA
:100DB00083420ED0FFF7C6FF022801D0012070BD8C
:100DC000082385F8E839C5F8E469C5F8E049022048
:100DD00070BD022070BD00BF301D0020034B93F892
:100DE000E809032894BF002001207047301D00202F
:100DF000004870471C27002030B4194B00209C7B12
:100E000014B11D688D4206D00130082803F110038B
:100E1000F5D130BC70479AB1124B03EB40218A42A6
:100E200019D0114B93F8B4218AB1104B01225A709A
:100E300000F5817003EB00100123837130BC704713
:100E40000A4B00F5817003EB00108271E1E701228B
:100E500083F8B421E9E7022CE3D1183BE8E700BFAF
:100E6000145A0020144A0020FC590020FC4900209C
:100E700030B41D4C002384F8A03004F1180004E0C5
:100E80000133082B00F110001ED005688D42F7D108
:100E900090F80EC0BCF1030FF2D1BAB1134901EBC7
:100EA0004320824209D094F8B42112B9012284F877
:100EB000B4210F4901224A7000E0183903F581730B
:100EC00001EB031301229A7130BC70470849D4F832
:100ED0009C2003F5817301EB031301320421997106
:100EE000C4F89C20F0E700BFFC590020144A002001
:100EF000FC490020A8B183681BB10E4B07229A70F1
:100F000070470C4A1178D36003294FF004000CBFDE
:100F100080214FF48071C2E9011113611375907043
:100F20007047044A02F580510123537081F8B431AF
:100F3000704700BFFC49002010B5812104466EF0C7
:100F400013FB204601216EF00FFB204682216EF03C
:100F50000BFBFFF775FE002010BD00BFC1690269E1
:100F600010B4002340F20114A0F844410B60D16991
:100F7000846D21F002014FF0010CD161A0F89CC3F7
:100F80002360D169044821F4003180F8203A5DF8EB
:100F9000044BD16118467047301D002020230148C2
:100FA0000B80704760000020122301480B807047BF
:100FB00080000020042301480B807047940000202B
:100FC0000A4608B5054920B90548FFF78DFD0348D5
:100FD00008BD0448FFF788FD004808BD54270020DD
:100FE000A8240808C024080808B5044B04480A4689
:100FF0001946FFF779FD084608BD00BF54270020B9
:10100000D82408082048D0F8E837D0F8EC2730B5C5
:101010009B184FF01A040C8001D11C4830BD1B4AAC
:10102000D0F8EA174FF0000E10467546B3F1204F86
:101030004FEA137C0CF130040EF1020E2ABF0CF1C2
:10104000370C847080F802C0BEF1100FC5704FEAF3
:10105000031300F10200E9D100200446B1F1204F52
:101060004FEA117303F1300C00F102002ABF37334D
:1010700082F812C093740828D4744FEA011102F167
:101080000202EBD1014830BD00F0FF1F98000020A4
:1010900008B5044B04480A461946FFF725FD0846E3
:1010A00008BD00BF54270020EC24080808B5044BF5
:1010B00004480A461946FFF717FD084608BD00BF59
:1010C00054270020F824080810B50F4C0F4BD4F813
:1010D000FC1BB4F8000C088303F1B402C4F8702DB3
:1010E000D3F8B430984702E01B69984720B9D4F888
:1010F000703D002BF8D1FEE7D4F8FC3BB4F8002C8F
:101100005A83002010BD00BF301D002000000020C9
:1011100038B5084BD3F8703D53B1DB6914460D4622
:1011200098474FF4007302682A600020236038BD9E
:101130001B68FFDE301D002008B5074BD3F8703D5B
:1011400033B11B69984780F00100404240B208BDAE
:101150004FF0FF3008BD00BF301D00200020704759
:101160002DE9F041164CD4F8C00B1646B4F8C42B48
:10117000428303B30F4603EB060806E000234D68E5
:101180001A4639463046A84738B9D4F8701D0029A8
:10119000F4D1FEE71B69984720B9D4F8703D002BC5
:1011A000F8D1FEE70136B04507F50077EDD1D4F868
:1011B000C00BB4F8C42B02830020BDE8F08100BF4F
:1011C000301D00202DE9F041184CD4F8C00B164614
:1011D000B4F8C42B42832BB30F4603EB060801E09F
:1011E0000B699847D4F8701D51B10023CD681A4699
:1011F00039463046A847D4F8701D08B10029EFD110
:1012000031B10B69984720B9D4F8701D0029F8D185
:10121000FEE70136B04507F50077E3D1D4F8C00BFF
:10122000B4F8C42B02830020BDE8F081301D0020FB
:10123000A64A536823F4FD4323F07F032DE9F041D0
:1012400043F0760353605368032123F480735360A3
:1012500082B011600FF098FB04460D460FF094FB2E
:10126000031B61EB0502B3F57A7F72F10003F5D33E
:101270000FF08AFB04460D460FF086FB031B61EB63
:101280000502B3F57A7F72F10003F5D38F4C6368E2
:1012900040F2FF5043F4807300214FF4806263609A
:1012A000A0634FF40033A160E26001E0002B6DD039
:1012B000626B160603F1FF33F8D5002B66D040F2BF
:1012C000FF554FF4D5724FF48963A5630721A563D9
:1012D0000820A260E360FFF721F8A56300284ED044
:1012E00000277A4C40F2FF55002240F27743A56375
:1012F0000121A2603720E360FFF710F8A563002802
:1013000039D147F000470646804647F4801701E090
:10131000964230D040F27743A5630121C4F808809B
:101320003720E360FEF7FAFF034640F269420321EB
:1013300029200136A563F3B9A563A760E260FEF733
:10134000EDFF4FF6FF72A563A8B96369002BDFDAE2
:101350004FF6FF7296420ED05D0000F1BF80236809
:101360009B0708D05A4D95F89000042840F0BE80A5
:10137000FFF7AAF890B1012002B0BDE8F081544B0C
:10138000012283F890204FF08047AAE74F4B40F2AC
:10139000FF5201209A6302B0BDE8F0814B4C2A68ED
:1013A00040F2474340F2FF56A6630121A2600720A6
:1013B000E360FEF7B3FFA663636823F4FD4323F005
:1013C0007F0363600028D6D195F89030022BD2D8E5
:1013D000636913F00073CED1CDE9003308274FF4D1
:1013E0008A63A6630121A7601020E360FEF796FFE1
:1013F000A6630028BFD12B68A663A36040F27743A1
:10140000E36001213720FEF789FFA6630028B2D1EF
:10141000304B6362A762E36A43F03303E36240F256
:101420007343A6630121A060E3603320FEF776FFDB
:10143000A66300289FD16B4640F22A4206E0616B0A
:10144000880244BFD4F8801043F8041B616B11423A
:10145000F5D0636B19078ED4636B9A078BD4636BDB
:101460009B0688D4636B9F0285D4009B1BBA5E03E6
:1014700081D52A6840F2774340F2FF55A5630121E8
:10148000A2603720E360FEF749FFA56300287FF4E0
:1014900072AF022240F24643A5630121A2600620FA
:1014A000E360FEF73BFFA56300287FF464AF636849
:1014B0001C0509D4054A084953680B4043F40063EE
:1014C000536053681805F7D5002055E7002C0140FC
:1014D000301D002000E1F5050081FFFF314D0220A5
:1014E00085F8900023689C073FF445AF2E49002300
:1014F00040F2FF528A638B6040F2C243CB604FF4EC
:10150000003301E0013B03D04A6B12F0450FF9D0E4
:10151000254B5A6B520741D45A6B12F0010F40F21F
:10152000FF529A637FF427AF5A696A619A69AA6188
:10153000DA69EA611B6A2B6201282AD81A4C40F248
:10154000FF56002240F24343A6630621A260032017
:10155000E360FEF7E3FEA66300287FF40CAF124CB5
:101560002A6840F2FF5640F2C943A6630221A260F6
:101570000920E360FEF7D2FEA66300287FF4FBAEED
:1015800063696B60A369AB60E369EB60236A2B61FD
:10159000EEE600F0FB000228D0D0E0E740F2FF5278
:1015A0009A63E8E6301D0020002C014008B5FFF7E3
:1015B0003FFE58B10E4A92F8DC390133DBB2072BFB
:1015C00082F8DC3903D9002382F8E83908BDD2F863
:1015D000143A23B11868998803691942F3D001239A
:1015E000D2F81C1A82F8E839C2F8D81908BD00BF31
:1015F000301D0020F8B59F4CD4F8180A002800F0E0
:10160000328194F8E8099C4D40F2FF5640F24D4774
:10161000431E082B63D8DFE813F04D005000D900BB
:101620006200950074002500620009002368AE6323
:101630000121AB600D20EF60FEF770FEAE6328B9AC
:101640006B69C3F34323042B00F00881D4F8D83925
:10165000D4F81C2AFA3393423ED2FFF7A7FF94F83E
:10166000E809D5E72368AE630121AB600D20EF6088
:10167000FEF754FEAE630028E8D16B69C3F3432341
:10168000042BE3D1D4F8E43984F8DC09012B40F2CF
:10169000ED80D4F8E0290820013B0132C4F8E43998
:1016A000C4F8E02984F8E809A0F10800B0FA80F055
:1016B0004009F8BD022384F8E8392368AE630121AC
:1016C000AB600D20EF60FEF729FEAE6320B96B69B9
:1016D000C3F34323042B5AD094F8E809431EDBB22A
:1016E000022B0AD8D4F81C3AD4F8D8299B1AC82B54
:1016F000DAD9FFF75BFF94F8E8090428D4D1012078
:10170000F8BD236B002BCFD1D4F8D059D4F81C3AB4
:10171000C4F8D839072084F8E809002DC4D0D4F8DB
:10172000D439D4F8C429D4F8C8190120A84794F8AA
:10173000E809431ED3E7D4F8D839D4F81C2A643317
:101740009342B1D2E36A002BF5D12368AE63012145
:10175000AB600D20EF60FEF7E1FDAE6300287FF483
:101760007EAF6A69C2F34322042A7FF478AFD4F8CB
:10177000D05984F8E82984F8DC09002DBFD0D4F8CA
:10178000D439D4F8C429D4F8C819A847A4E7FEF777
:101790009BFE0028A0D194F89030002BA3F1020307
:1017A000B3FA83F314BF022201225B0984F8DD2916
:1017B00084F8DE39FEF788FE00287FF44EAFD4F8B7
:1017C0008020C4F8EC29032384F8E839FEF77CFE76
:1017D000002881D194F86420B4F86630A4F8F03978
:1017E000A16EA36EC4F8E409090E04201B0C84F852
:1017F000F22984F8E809A26E84F8F31984F8F43920
:10180000A16E94F86C0094F86D3084F8F619120A01
:101810001B0984F8F52984F8F70994F86D2084F8F9
:10182000FC39216FB4F87600B4F87630C4F8F819B2
:1018300002F00F02C3F30B1384F8FD2943EA1023CF
:10184000B4F8762003F00F0303F5FA6302F00F02F9
:10185000A4F8FE3984F8002A0120F8BD042384F896
:10186000E8390120F8BD84F8E809F8BDF6D1FFF7A2
:1018700069FA31E7301D0020002C01402DE9F041CC
:10188000204E96F8743D002BFBD1B9B3014400F112
:10189000FF384F1ED6F8A418D6F8A03818F8010F54
:1018A0004A1CC2F30A029A4234BF002401249B1A44
:1018B000314403EBC423012B81F8780DC6F8A4282A
:1018C0001AD10FF061F804460D460FF05DF8031BC6
:1018D00061EB0501B3F57A7F71F10003F5D3D6F81A
:1018E000A038D6F8A42893428CBF002101219B1A6E
:1018F00003EBC123012BE4D0B845CBD10020BDE8D8
:10190000F08100BF301D002010B50A4CD4F89C387F
:1019100003B910BDD4F89C38052BFAD1002A08462B
:10192000D4F81C3A1146F4DDFFF7A8FFD4F81C3AAE
:1019300010BD00BF301D002090F84820531C024409
:10194000DBB280F8483082F8341090F849200AB1B0
:10195000132B03D9002280F8482003B9704710B533
:10196000084CD4F89C2802B910BDD4F89C28052A4C
:10197000FAD119463430D4F81C3AFFF77FFFD4F877
:101980001C3A10BD301D002090F848100023A0F82C
:10199000483001B9704710B5084CD4F89C381BB1D9
:1019A000D4F89C38052B00D010BD3430D4F81C3A44
:1019B000FFF764FFD4F81C3A10BD00BF301D0020B3
:1019C0002DE9F0475D4E1F4606EB80039C68002C16
:1019D00000F0AD8004F13E03A36104F59F73E36161
:1019E0004FF48073C4E904332836236866600546E3
:1019F000E16094F83D00A36390460BF01DF9814629
:101A000094F8440294F83CA0261D00284FD194F885
:101A1000450268BBD4F8403283BB390734D418F090
:101A2000020F60D118F0010F44D194F9472294F8C5
:101A30004712D4F84832002A10DB41481B018418B1
:101A4000DBB284F800335209012301F01F0103FACD
:101A500001F140F822103046BDE8F087394A01F024
:101A60000F010A441B01DBB213763046BDE8F08754
:101A70006BF098FAD4F84032002BCED0324A116B7A
:101A80000B4339071363CAD50135EDB2B9F1000F25
:101A9000CBD040F20673FA0689F80850A9F8063050
:101AA00036D4BB0694F8462245D4322133E06BF09D
:101AB00079FAACE750460BF0BFF80135EDB20028DB
:101AC000B3D040F206620572C28094F84622022129
:101AD0000BF0B6FA94F9472294F84712D4F848323A
:101AE000002AAADABAE76B1CDBB2B9F1000F99D071
:101AF00089F8083040F20653A9F8063094F84622D7
:101B0000484602210BF09CFA18F0010F8DD0D1E766
:101B100094F84622022148460BF092FA94F94722A3
:101B200094F84712D4F84832002A86DA96E7264617
:101B30003046BDE8F0871221EDE700BFBC850708FD
:101B400000E100E0FCEC00E0003802402DE9F04745
:101B5000038A8489A4B21C4082B045D0814688465D
:101B60004FF0004501F14C0701F13406B4FA84F35B
:101B700025FA03F2D24391B2A9F8101014401B3B8E
:101B8000B8F1000F5DD0042B2CD8DFE803F05046ED
:101B90003B300300D8F80C30D9F82CA033B19B6847
:101BA00023B11FFA8AF108F104009847D8F82430CD
:101BB00033B19B6823B11FFA8AF108F11C009847E2
:101BC000D8F83C302BB19B681BB11FFA8AF1304624
:101BD0009847D8F854302BB19B681BB11FFA8AF193
:101BE00038469847002CC1D102B0BDE8F087D8F83C
:101BF0000C30D9F834105B6808F104009847002CC9
:101C0000B4D1F1E7D8F82430D9F838105B6808F17E
:101C10001C009847002CA9D1E6E7D8F83C30D9F849
:101C20003C105B6830469847002C9FD1DCE7D8F821
:101C30005430D9F840105B6838469847002C95D14D
:101C4000D2E7042B07D8DFE803F00319140F0A00CA
:101C5000D9F840300193019B002C87D1C4E7D9F813
:101C60002C300193019BF7E7D9F834300193019BA5
:101C7000F2E7D9F838300193019BEDE7D9F83C3011
:101C80000193019BE8E700BF38B5284C94F8742D08
:101C9000012A034603D0022A09D0002038BD244976
:101CA000D1F88024A2B984F8742D002038BD002515
:101CB00040F20112C0E95455C0E95655A0F844213C
:101CC00000F5A2716DF060FD84F8745D002038BDF0
:101CD000402AD4F8A00819D9403AC1F880244022FB
:101CE0008118C4F8A01880B2124940F201140144CE
:101CF0000020C3E95411C3E95620A3F84441184613
:101D000003F5A2716DF040FD002038BD4FF00005D5
:101D1000C1F8805402EB0001C4F8A01808BF0221EA
:101D200080B208BF84F8741DDEE700BF301D0020BC
:101D3000282E0020A82A002001EB810138B500EBF5
:101D4000C1010E4DB1F88C1304462846FEF7C4FFBE
:101D5000E378C4F8A85340210022C4E9EC12012220
:101D600093422046A4F89C2304F5677108BFC4F889
:101D7000AC536DF009FD002038BD00BFAC3200202F
:101D800038B52A4BD3F8C4240F2A04D0511CC3F809
:101D9000C414002038BD264A92F8745D0021C3F8AF
:101DA000C414002DF5D1D2F8A018D2F8A448B1F58A
:101DB000006F30D0A14235D002F6785594BF641A36
:101DC000C1F5006415FA81F5402C19D82144C2F8F8
:101DD000A0184FF00001C3F880140CBF02230123A8
:101DE00082F8743D40F201120023C0E95455C0E965
:101DF0005643A0F8442100F5A2716DF0C5FCC8E778
:101E0000403CC3F8804440310123C2F8A01882F856
:101E1000743D4024E6E7C2F8A0581CB1294602F6FA
:101E20007855D1E7002382F8743DB2E7282E0020D0
:101E3000301D002038B5224DD5F8D03495F8E8C4CF
:101E4000044623B195F8D4345CEA030331D001236E
:101E5000E06984F8463140F20112A4F84421026896
:101E60001849002AA8BFC2F380739B0301EA1241FC
:101E700043F020030B4363F31F42BCF1020F0260E7
:101E800000D038BDE278104BC4F8A8331F200021E1
:101E9000C4E9EC01012A4FF00101A4F89C1308BF2A
:101EA000C4F8AC3304F567712046BDE838406DF0E6
:101EB0006BBC01216DF01EFB95F8E8C4C7E700BFBD
:101EC000282E0020DFBFFFFFF032002070B590F811
:101ED000CF2590F8D13590F8CE5590F8D0C590F830
:101EE000CC1590F8CD6505EB02250CEB032C90F892
:101EF000D32590F8D23503EB0223012284B080F879
:101F0000112101F01F029BB2ADB21FFA8CFC012A15
:101F100004468DF80810ADF80A50ADF80CC0ADF8C5
:101F20000E30C0F840318DF809600AD0022A57D02F
:101F3000002A3CD001F080016DF0DCFA002004B0F2
:101F400070BD90F81231032B2BD15FFA8CFCBCF1E1
:101F5000010F26D8D0F8E43502A99B689847BDF850
:101F60000E30002BEAD1C4E94A33C4E94C330421D2
:101F70004FF4807284F81111A4F81C2104F58E71BD
:101F800020466DF093FB636DC44A1A61E278012A22
:101F9000D4D104F2CC545C614FF0802219681A60ED
:101FA000CCE720466AF050FD002004B070BD092E39
:101FB000F7D801A252F826F0632000087321000828
:101FC000A31F0008AD210008A31F0008DB210008A3
:101FD00087200008A31F0008F12000082121000825
:101FE00001F0600120295FFA8CF334D0012E00F05B
:101FF0006181032E00F09581002E9FD190F812216F
:10200000022A00F01B81032ACBD11CF0800F40F084
:10201000A48103EB830300EBC30393F87633002B17
:1020200000F0A6819E4B0122C3F8F8249D4A0223AA
:10203000C4E94E334FF48070002184F81131A4F8C4
:102040001C01C4E94C31C4E94A2204F58E712046D2
:102050006DF02CFB72E7D0F8E43502A99B68984735
:102060006CE790F81231023B012B9AD88C4BD0F8D8
:1020700018210021C3F8F01412B10222C3F8F02491
:10208000894A0223D4E72E0A022EADF8063000F06A
:10209000CD81032E00F09181012E82D1D0F8EC3554
:1020A00080781B680DF106019847BDF80630002BBB
:1020B0003FF444AFBDF80E20002A3FF43FAF9342F7
:1020C00028BF13464FF480720221A4F81C2100227D
:1020D000C4E94A0084F81111C4E94E33C4E94C3212
:1020E00004F58E712046ADF806306DF0DFFA25E775
:1020F000012B7FF456AF90F81221022A00F049819B
:10210000032A7FF44EAF4FF4807100F588720220ED
:10211000A4F81C11C4E94E3384F81101002190E7A2
:10212000EDB25F4E012D86F8E9543FF63AAF90F8D4
:102130001231022B00F02181032B7FF432AF002DEE
:1021400000F07F8190F81011012910D0D0F8E4350B
:102150005B68984796F8E914D4F8E43584F81011D0
:102160001B6820469847D4F8E8359B6898470023B9
:10217000F9E690F81231023B012B3FF612AF012D28
:102180007FF4DCAED0F8E43500259B68C0F8185128
:1021900002A9984704224FF48073C4E94A55C4E960
:1021A0004C5584F81121A4F81C31E7E6012D00F00C
:1021B000CC80022D7FF4C2AE5FFA8CF3002B7FF44B
:1021C000BDAE02694FEA1C23023B5268032B00F2AA
:1021D0005681DFE803F05B426B5F5CEA03037FF448
:1021E000E0AE90F81221032A3FF4DBAE016905F05E
:1021F0007F0680F8146108681A4665F30A120243E4
:102200000A604FF480720421C4E94A33C4E94C33B4
:1022100084F81111A4F81C2104F58E7120466DF08C
:1022200045FA636D1D4A1A61E278012A0DD0002E2D
:1022300000F01281022384F812317FE65A063FF43F
:102240007DAE19466DF056F978E604F2CC525A612B
:102250004FF0802219681A60E9E7032363F306123E
:1022600001210F4D84F816110421002384F8111167
:102270004FF48071A4F81C11C4E94A33C4E94C330B
:1022800004F58E712046C5F8F4247AE6022363F340
:102290000612E5E7052363F30612E1E7180008607C
:1022A000282E00202033002018330020042363F35D
:1022B0000612D5E790F81221022ABFD0032A7FF434
:1022C00070AE002D7FF43AAE13F07F023FF44FAFB3
:1022D0001CF0800F40F0C48003EB830100EBC101D0
:1022E00081F8742381F8765381F87553282101FB16
:1022F000030300EB820293F87713506D03688A1E84
:10230000012A6FF35553D4F8E4258CBFC3F3007151
:10231000012161F31C739268036002A92046904773
:1023200025E790F81221022A88D0032A7FF439AEDB
:1023300025B9590602D019466DF0DCF8D4F8E43519
:1023400002A99B682046984711E7D0F8E43502A916
:102350009B68C0F81851984709E703F07F0303EB27
:10236000830300EBC30393F81E31002B7FF45AAEB6
:10237000454B0022C3F8F82458E6002D3FF40AAF7D
:1023800001210322D0F8E43580F8101180F81221E1
:10239000E6E63E4984F811214FF480700022C4E93A
:1023A0004A11A4F81C01C4E94E33C4E94C3204F5C7
:1023B0008E7120466DF07AF9C0E5EDB2052D3FF63D
:1023C000F0ADDFE805F02B231B130B03D0F8EC3541
:1023D00080789B690DF10601984766E6D0F8EC35E8
:1023E00080785B690DF1060198475EE6D0F8EC3520
:1023F00080781B690DF10601984756E6D0F8EC3558
:102400008078DB680DF1060198474EE6D0F8EC3590
:1024100080789B680DF10601984746E6D0F8EC35C8
:1024200080785B680DF1060198473EE6D0F8E43508
:1024300080789B6A0DF1060198474670C4F8F00554
:1024400033E60222D0F8E43580F8122180F81051EA
:102450005B68294698479DE6012384F812316DE5B3
:10246000282303FB020181F81C2100EB820281F882
:102470001E5181F81D61906991F81F113EE70123FB
:1024800063F30612ECE600BF282E00201433002070
:1024900010B5044629B990F81121032A0DD0002067
:1024A00010BDD0F8E4359B69002BF8D090F81221CC
:1024B000032AF4D19847002010BDD0F890230B4692
:1024C000D0F87C138A4213D9C078521A0128C4F874
:1024D000902336D08A4228BF0A4692B2C4E9E2234A
:1024E00004F55D71A4F8743320466DF0DFF8D6E78B
:1024F000D0F8E4351B691BB190F81221032A1ED0D5
:1025000000234FF480720421C4E94A33C4E94C33F8
:1025100084F81111A4F81C2104F58E7120466DF089
:10252000C5F8636D104A1A61E278012AB7D104F246
:10253000CC545C614FF0802219681A60AFE798476D
:10254000DEE78A42D4F88003A4F8743328BF0A4631
:10255000084492B2C4E9E22304F55D71C4F8800333
:10256000C4F88403C0E700BF1800086038B504460B
:1025700049B990F81131022B11D094F81631012B82
:1025800040D0002038BDD0F8E4355B69002BF8D08E
:1025900090F81221032AF4D19847002038BDD0F8D2
:1025A0003831D0F82421934236D9C178012908BFA7
:1025B000D0F82811A3EB020318BFD0F82821C0F8E7
:1025C000383108BF52189BB24FF480710025C0E922
:1025D0004C35A0F81C11C0E94A2200F58E716DF04F
:1025E00065F8E378C4F88053012BC4E9E255A4F8F8
:1025F000745308BFC4F8845304F55D7120466DF030
:1026000055F8BAE72A4B2269D3F8F4145160002335
:1026100084F81631002038BDD0F83C31B3FBF2F518
:1026200002FB1535ADB99A4213D8D0F84021934238
:102630000FD24FF48073A0F81C31C0E94A55C0E9AD
:102640004C5500F58E716DF031F8E378C4F84051C7
:10265000C8E7D4F8E435DB681BB194F81221032AEB
:1026600023D0E2780023012A4FF0050108BFC4F807
:102670008433C4E9E23384F81111C4F88033A4F838
:10268000743304F55D7120466DF010F8636D094AEE
:102690001A61E278012A7FF470AF04F2CC525A61D9
:1026A0004FF0802219681A6067E720469847D8E7FC
:1026B000282E002018000860F8B50B7813F060068B
:1026C0000D46044620D0202E25D1CE884EB31B06C1
:1026D00049D5384F687832463946FEF7B9FAEB8863
:1026E0000222002684F811214FF48072C4E94E338F
:1026F000C4E94A77C4E94C36A4F81C2104F58E716C
:1027000020466CF0D3FF0AE04B780A2B17D00B2B36
:102710000ED0062B03D120466AF096F902263046E9
:10272000F8BD022248781144FEF792FA3046F8BD0F
:102730008B78002B3AD1204BC3F8FC64EFE70222E0
:1027400080F811214FF48072A0F81C211B4A01234C
:10275000C0E94E33C0E94A22C0E94C3600F58E711B
:102760006CF0A4FFDBE7164B164A4978116003F6BC
:10277000AC020321C0E9E46680F81111C0F8886357
:10278000C0F88023C078C3F8A86801284FF0000380
:10279000C4F88C33A4F8743304F55D7108BFC4F831
:1027A000842320466CF082FF0026B8E76AF04CF9DB
:1027B000B5E700BFDC250020282E002024330020B0
:1027C000301D002000000020002310B519460446EB
:1027D00040226CF0FBFE80212046002340226CF05A
:1027E000F5FED4F8E835A078012284F812215B6860
:1027F0009847002010BD00BF10B5022304464022B8
:1028000081216CF0E3FE20460223402201216CF07E
:10281000DDFE20460323082282216CF0D7FE0E4BFA
:102820000222A3F84C20FEF7FFF9E2780B4BC4F824
:10283000A83340200021C4E9EC01012A4FF0010136
:10284000A4F89C13204604F5677108BFC4F8AC33A4
:102850006CF09AFF002010BD00000020AC32002078
:1028600070B5812182B00446314E6CF07DFE0121AD
:1028700020466CF079FE002502234022812120466B
:1028800086F8205A6CF0A2FE012102234022204645
:102890006CF09CFE274B86F8205AD3F8002583F86D
:1028A000E8541268284690470095009BE16843F081
:1028B00010030093009B0B610A691F4B009203E019
:1028C0000A690092013B02D0009AD006F8D4002396
:1028D0000193019B43F020030193019A164B0120C1
:1028E00060F38A120192019A0A610A69019203E077
:1028F0000A690192013B02D0019A9206F8D4E2786B
:102900000E4BC4F8A83300211F20C4E9EC01012AB2
:102910004FF00101A4F89C1304F5677105D020461F
:102920006CF032FF002002B070BDC4F8AC33F6E7A3
:10293000301D0020282E0020400D0300F032002022
:102940002DE9F843394F8046894615461C4697F8CD
:10295000E81904290CD0082907D1D7F8E0394345F4
:1029600006D0FEF7EFF90228F1D00120BDE8F88388
:10297000012387F8CC393B6397F89030C7F8D449E6
:102980000622022B2A4CC7F8C889C7F8D059C7F8C5
:10299000C49987F8E82918BF4FEA48280A2640F268
:1029A000FF554FF48B63A5630121C4F808801820FC
:1029B000E360FDF7B3FC03464FF0000C40F27742B2
:1029C00001213720A56393B9012148466AF062FAD4
:1029D000174B184959624FF400729A62DA6A002163
:1029E00042F09102DA620846B962BDE8F883A56355
:1029F000C4F808C0E260FDF791FC721EA5630028D0
:102A0000E2D012F0FF06CCD13E63FEF7CFFDD7F83F
:102A1000D04944B10120D7F8D439D7F8C819324683
:102A2000A0470320E1E70320DFE700BF301D0020BF
:102A3000002C014000E1F5052DE9F04F3F4E99468D
:102A400096F8E83983B0042B80460191924609D06C
:102A5000082B03D0002003B0BDE8F08FFEF772F919
:102A60000228F7D196F890300122022BF26263D04F
:102A70004FEA482B324C019800216AF00BFA4FF4D0
:102A80000072304B6362A262E36A40F2FF5743F088
:102A90009303E362A763A2604FF48A62E2600121BC
:102AA0001020FDF73BFC0A25A76340F25142A763C3
:102AB0000121C4F808B01120E260FDF72FFC0246A6
:102AC0004FF0000E40F2774301213720A763AAB9E7
:102AD0000023B362D6F81C3A0199C6F8C41905223E
:102AE0000120C6F8C889C6F8D0A9C6F8D49986F8D6
:102AF000E829C6F8D83903B0BDE8F08FA763C4F859
:102B000008E0E360FDF70AFC013DA7630028DFD081
:102B100015F0FF05C9D1F562B062FEF747FDD6F8A2
:102B2000D049002C96D02846D6F8D439D6F8C81902
:102B30002A46A04728468EE7C3469BE7301D002063
:102B4000002C014000E1F5051049114BD1F8882017
:102B500042F4700210B4C1F888201A680D4C0020AD
:102B600042F001021A6098601A6822F0847222F41E
:102B700080321A605C601A68074C22F480221A6066
:102B8000D8608C605DF8044B704700BF00ED00E03A
:102B9000003802401030002400000008704700BFD9
:102BA0002DE9F84346697EB9D0F80080C8F30D09D5
:102BB00004460F46B9F1000F26D03F68FDF7C8FE66
:102BC000092804D06FF001063046BDE8F8834A4D6D
:102BD0002B6923F440732B612B6943F400732B6141
:102BE0002B6943F001032B61C8F80070FDF7B0FEBC
:102BF0002B69092823F001032B61E3D123680433F7
:102C000023603046BDE8F8833C4B98452AD303F552
:102C10008043984524D303F58043984554D3384BDB
:102C2000984554D903F58033984553D903F50033BB
:102C3000984552D903F50033984551D903F500332F
:102C400098453ED903F5003398454CD903F58023C8
:102C500098454BD9B8F1016F4BD305200DF0F0FE2C
:102C60004FF00809FDF774FE092804D04FF0FF3635
:102C70003046BDE8F883204D2B6923F440732B6167
:102C80002B6943F400732B612B6923F0F8032B614C
:102C90002B6943EA090343F002032B612B6943F4D8
:102CA00080332B61FDF754FE2B6923F002032B6167
:102CB0002B69092823F0F8032B61D7D1D4F80080C1
:102CC0007BE74FF03809CDE74FF01009CAE74FF026
:102CD0001809C7E74FF02009C4E74FF02809C1E7FA
:102CE0004FF03009BEE74FF04009BBE74FF048090D
:102CF000B8E74FF05809B5E7003C02400040000833
:102D0000FFFF00080148FDF785BA00BFD80000208A
:102D10000148FDF77FBA00BF240300200148FDF7FA
:102D200079BA00BF700500200148FDF773BA00BFF3
:102D3000BC070020704700BFF0B5254B026825494D
:102D400083B00646002401E051F834309A4209D09D
:102D500001340E2CF8D100211F4A052005F092FD08
:102D6000002113E01D4F07EB8407D7F8045585B108
:102D7000717901EB410305EBC30300221820C3E97D
:102D8000032200FB01559E601A75291D084603B0F9
:102D9000F0BD07216C2005F06BFE0146C7F8040565
:102DA00070B129466C2273F0DDFB0A4BD7F804554D
:102DB00003EBC404C5E90045ED616D63ED64D7E73D
:102DC0000190074A052005F05DFD0199DEE700BF8F
:102DD000000001401486070808250808282E002056
:102DE00030250808704700BF30B40C4C0022234641
:102DF00004E001320C2A03F114030CD093F804C050
:102E00008445F6D1DD68294201D10029F1D1142091
:102E100000FB024000E0002030BC7047040A0020A4
:102E200038B5D0E9004307EE902A1B68354A206880
:102E30000139934204688DB216D002F58062934244
:102E400012D002F5705293420ED002F58062934286
:102E50000AD002F58062934206D02B4BD3F8F43AA5
:102E60005B0807EE103A04E0274B03F6F42393EDDA
:102E7000007ADFED266AB8EE477AF8EE677A87EED9
:102E8000270A30EE260A6EF0C3FB1E4A238801385B
:102E9000944280B29BB212D002F5806294420ED06E
:102EA000B4F1804F0BD0A2F58032944207D002F5E6
:102EB0008062944203D002F58062944202D123F0F2
:102EC00070039BB2124A944212D002F5806294427F
:102ED0000ED023F4407302F56C429BB294422380DF
:102EE000E56220850AD1002323860123A38238BD11
:102EF0002380E56220850123A38238BD054B9C42D7
:102F0000F1D0F8E700000140000000200AD7233C80
:102F1000001000400004014070B54068837903F060
:102F2000020213F0040300F0C9804FF0000E1346B4
:102F300004247246754690F805C0BCF1030F30D8E2
:102F4000DFE80CF08E5F30020368188C20F48050AC
:102F50000004000C1884188C9C8820F40050000495
:102F60002A43000C40EA0232988B6C4D20F4E64074
:102F70000004000CAB42A4B240F4C04000F0B080AA
:102F800005F58065AB4200F0AB809C8098831964A6
:102F90001A849A8B22F400621204120C42F400622A
:102FA0009A8370BD2A4305685C4E288C20F480709B
:102FB0000004000C2884288CB5F804C020F40070AC
:102FC0000004000C40EA0222A88B20F073000004E9
:102FD000000CB5421FFA8CFC40F0600073D006F57F
:102FE0008066B5426FD0A5F804C0A883E9632A843F
:102FF000AB8B23F008031B041B0C43F00803AB83CB
:1030000070BD2A430568454E288C20F0100000044E
:10301000000C2884288CB5F804C020F0200000049F
:10302000000C40EA0212288B20F4E6400004000C59
:10303000B5421FFA8CFC40F4C04061D006F58066B2
:10304000B5425DD0A5F804C02883A9632A842B8BE0
:1030500023F400631B041B0C43F400632B8370BD3B
:1030600000682E4E2A43058C25F001052D042D0CF9
:103070000584058CB0F804C025F002052D042D0C44
:103080002A43058B25F073052D042D0CB0421FFA41
:103090008CFC45F0600528D006F58066B04224D04F
:1030A000A0F804C0058341630284038B23F0080366
:1030B0001B041B0C43F00803038370BD4FF4807E98
:1030C0001C46012537E722F4006242EA032222F47B
:1030D00080622CF4405C42EA04224CEA0E1C82E737
:1030E00024F4804444EA8E144FE74FF6F3761640FA
:1030F0002CF4407C46EA03024EEA0C0C2243CFE754
:1031000022F0800242EA031222F040022CF4406CCA
:1031100042EA04124CEA8E0C94E700BF0000014022
:1031200042685379032B0FD8DFE803F00B08050240
:1031300010684030704710683C3070471068383075
:10314000704710683430704700207047024B0348C6
:10315000D3F80415FEF7FABC282E00200000014029
:1031600010B5064C0648D4F80415FEF7EFFCD4F869
:1031700024150448BDE81040FEF7E8BC282E0020C6
:10318000000001400040014010B5064C0648D4F84C
:103190000415FEF7DBFCD4F828150448BDE8104000
:1031A000FEF7D4BC282E002000000140004401405E
:1031B00010B5064C0648D4F80415FEF7C7FCD4F841
:1031C0002C150448BDE81040FEF7C0BC282E002096
:1031D0000000014000480140034B4FF08040D3F80D
:1031E0000815FEF7B3BC00BF282E0020024B034891
:1031F000D3F80C15FEF7AABC282E002000040040CE
:10320000024B0348D3F81015FEF7A0BC282E00206F
:1032100000080040024B0348D3F81415FEF796BC93
:10322000282E0020000C0040024B0348D3F8201544
:10323000FEF78CBC282E00200004014010B5064C7F
:103240000648D4F82015FEF781FCD4F83015044860
:10325000BDE81040FEF77ABC282E00200004014093
:103260000018004010B5064C0648D4F82015FEF7AB
:103270006DFCD4F834150448BDE81040FEF766BC78
:10328000282E002000040140001C004010B5064C10
:103290000648D4F82015FEF759FCD4F83815044830
:1032A000BDE81040FEF752BC282E0020000401406B
:1032B000002000400348D0F8043B13B100F6F8208A
:1032C00018477047000000200348D0F8243B13B192
:1032D00000F6183018477047000000200348D0F867
:1032E000443B13B100F63830184770470000002007
:1032F0000348D0F8643B13B100F6583018477047C4
:10330000000000200348D0F8843B13B100F6783069
:1033100018477047000000200348D0F8A43B13B1C1
:1033200000F6983018477047000000200348D0F896
:10333000C43B13B100F6B8301847704700000020B6
:103340000348D0F8E43B13B100F6D8301847704773
:10335000000000200348D0F8043C13B100F6F83018
:1033600018477047000000200348D0F8243C13B1F0
:1033700000F6184018477047000000200348D0F8B6
:10338000443C13B100F63840184770470000002055
:103390000348D0F8643C13B100F658401847704712
:1033A000000000200348D0F8843C13B100F67840B8
:1033B00018477047000000200348D0F8A43C13B120
:1033C00000F6984018477047000000200348D0F8E6
:1033D000C43C13B100F6B840184770470000002005
:1033E0000348D0F8E43C13B100F6D84018477047C2
:1033F0000000002030B44568154CA542154D2C6BDB
:103400000CBF44F4001444F480042C6390F914C0FD
:10341000C160BCF1000F836111DB0F49120101EBA8
:103420000C03D2B283F800234FEA5C1001230CF0A6
:103430001F0C03FA0CF330BC41F820307047074BE7
:103440000CF00F0C12016344D2B21A7630BC7047F4
:10345000006002400038024000E100E0FCEC00E0C7
:103460002DE9F84FDFF814B300210BF6F8204FEAEE
:10347000411C50F80C30C3F30132C3F3032382F034
:10348000020283F0030352EA03040AD00131102937
:10349000EDD1A74E0023C6F8183A86F8E839BDE802
:1034A000F88F6044A24E037FC6F8180A002BF1D1B2
:1034B000DC44A04BDCF8007B9F4202D048339F42A3
:1034C000E8D19D4A536A43F4006353620DF05CFAFD
:1034D000804689460DF058FAB0EB080361EB09010C
:1034E000B3F57A7F71F10003F4D3934A536A23F45E
:1034F000006353620DF048FA804689460DF044FAA5
:10350000B0EB080361EB0901B3F57A7F71F10003B9
:10351000F4D3DFF824928948D9F8443043F40063A7
:10352000C9F84430D9F8303043F48003C9F830305A
:10353000D9F8303043F00C03C9F830304FF00D0AA1
:103540004FF000080C220E21A6F80AAD86F80C8D6B
:1035500009F076FD7A48A6F816AD0C220E2186F801
:10356000188D09F06DFD7748A6F822AD0C220E21CA
:1035700086F8248D09F064FD7348A6F82EAD0C2260
:103580000E2186F8308D09F05BFD7048A6F83AAD43
:103590000C220E2186F83C8D09F052FD0C226C485D
:1035A000A6F86AAD0E2186F86C8D09F049FD694BCD
:1035B000302283F831234FF400325A60D9F830308A
:1035C00043F48003C9F83030634BC3F83C75594B62
:1035D0009F425CD061496248C1F8A080614BC1F84C
:1035E000A8004FF474176048CF60C1F8A00007200E
:1035F000C1F8B4005D4F42461846194605E0013255
:10360000102A01F1200100F08F808D68BD42F6D1B3
:103610000BEB42115201D1F8FC7A55498F4274D01C
:10362000454F396B41F4800139630BEB02054F497B
:103630000D22A5F8142B9A688A4225D00134102C4B
:1036400003F12003F7D100204A4900230122FFF7AC
:10365000D1FED6F8143A4BB119689A880B691A4210
:1036600004D1002386F8E839BDE8F88FFDF7E0FDC6
:103670000028F6D1D6F81C2AC6F8D829012386F8E6
:10368000E83986F8DC090AE700EB4410DCE7344946
:10369000C3F80080DFF8CCC099604FF07460324905
:1036A00043F8500C19600721583B4246D9666046E2
:1036B000634604E00132102A03F1200334D09968F4
:1036C000B942F7D10BEB42135201D3F8FC1A284B45
:1036D000994223D018490B6B43F480030B630BEB27
:1036E00002050D23134AA5F8143BDCF80830934279
:1036F00011D00134102C0CF1200CF6D100201E4901
:1037000000230122FFF776FEA3E70B4F396B41F44C
:103710000011396389E700EB4410F0E706490B6BB1
:1037200043F400130B63DAE700235B68FFDE00BF9E
:10373000301D00205864024000380240342A002026
:10374000402A00204C2A0020582A0020642A002009
:10375000942A002000E100E0282E002000640240AE
:10376000802C0140F80A00206054A308A0640240A5
:1037700000600240650800089D0700080000002066
:1037800070B52D4C636BD9051ED54FF4807340F294
:10379000FF56A363A663E36B284D23F4414323F054
:1037A0003A03E3636B6B9A071FD4012200236A621A
:1037B000AB62214A40F2FF539363D36B23F441433E
:1037C00023F03A03D36370BD636B980703D51B4B9B
:1037D00002229A62EDE7636B190721D4636B9A06A4
:1037E00022D5164B06229A62E3E7154BD3F83C2507
:1037F000136823F001031360E36A002223F0080337
:10380000E3622A636B6BDB07CFD540F24C43A663C0
:103810000121A2600C20E360FCF780FDA663C4E7F1
:10382000064B04229A62C4E7636BDB06C1D5034BE7
:1038300005229A62BDE700BF002C0140301D002028
:10384000282E002002683649002310B422F001021D
:10385000212488420260036043608360C360036187
:10386000446138D02F4B98422ED02F4B98423CD0F9
:103870002E4B984240D02E4B984232D02D4B98423E
:1038800041D02D4B984246D02C4B984217D02C4B10
:1038900098423CD02B4B984216D02B4B984224D0C8
:1038A0002A4B984228D02A4B98421AD0294B98424A
:1038B00029D0294B98422ED0284B984208D14FF05E
:1038C0003D5243F8AC2C03E04FF4746243F8202CD3
:1038D0005DF8044B7047224B5DF8044B3D229A6023
:1038E0007047204A43F8642CF2E74FF474125DF8F5
:1038F000044B43F8382C70474FF074625DF8044B6A
:1039000043F8502C7047184A43F87C2CE0E73D22DE
:1039100043F8082CDCE7154A43F8942CD8E700BF9D
:10392000106002402860024040600240586002403F
:103930007060024088600240A0600240B8600240AF
:10394000106402402864024040640240586402400F
:103950007064024088640240A0640240B86402407F
:10396000006002403D000020400F002000003D208C
:1039700000222DE9F04713460D684FF0010E032693
:1039800004E00133102B02F1020239D00EFA03FCDD
:103990003CEA0504F5D1076806FA02F427EA0407B1
:1039A00007600F79D0F800A007FA02F9013F49EA51
:1039B0000A09012FA046C0F800906FEA040411D84C
:1039C00087683C4084604C79876894403C438460BD
:1039D000446824EA0C0444608C7947689C40A4B293
:1039E0003C434460C46824EA0804C460CC79C768D6
:1039F000944001333C43102BC46002F10202C5D154
:103A0000BDE8F0872DE9F0412348244F244E254C92
:103A100082B03822002172F0A5FD002557F825104C
:103A20003246002301E054F8332091422ED0013376
:103A30000E2BF8D10020053569F0B4FA3C2DEDD1FC
:103A4000DFF85880184F08F1F0054FF0007698F82D
:103A5000040009F0F1F808F11408044688B103687D
:103A600003F13F4303F57E0307EB932393F8C8006C
:103A700069F098FAA3880196206800936946FFF7D9
:103A800077FFA845E3D102B0BDE8F081064A02EB1A
:103A9000C30393F85C00CEE72C330020040A002017
:103AA0000000014014860708BC850708224A936875
:103AB00003F00C03042B10B421D0082B22D01F4B91
:103AC00003601D4C1E4AA168C1F30311114491F813
:103AD000F81CCB404360A168C1F38221114491F8E6
:103AE000F81C23FA01F18160A1685DF8044BC1F371
:103AF00042310A4492F8F82CD340C3607047114B0E
:103B00000360DEE75368516813F4800F01F03F0152
:103B1000536814BF0B4A094AB2FBF1F1064A5268D6
:103B2000C2F30142C3F38813013201FB03F35200D5
:103B3000B3FBF2F30360C4E7003802400024F40052
:103B40000000002000127A0070B5446B8668A389DB
:103B500023F400531B041B0CA38182790546407992
:103B600012F0040F14BF4FF4805C4FF0000C1103EF
:103B700010F0010F4FEA02220CBF0023042302F4CD
:103B80008062800748BF43F0080342EA0C021343F7
:103B9000228A92B201F4005122F440520A43228256
:103BA000A28922F4B05222F00C021204120C1A4321
:103BB000A281A38A23F440731B041B0C84B0A3824C
:103BC0006846FFF773FF244B9C4205D003F58063E2
:103BD0009C4201D0029A00E0039AA3891F491B046A
:103BE00002EB82024CBF7300B30002EB8202B2FB15
:103BF000F3F3A1FB0302A08952096426000406FB2B
:103C000012334FEA02121FD41B013233A1FB0313FC
:103C1000C3F3431313439BB22381AB796A6B13F055
:103C2000080F938A0AD09BB243F0080393829389CA
:103C30009BB243F40053938104B070BD23F008039A
:103C40001B041B0C9382F2E7DB003233A1FB03134E
:103C5000C3F342131343DEE7001001401F85EB510D
:103C60002DE9F8431D462E4B9DF820609DF82490C9
:103C70009842884617463BD02A4B984240D02A4B60
:103C8000984245D0294B984221D14B46324629468D
:103C90000520FDF795FE04460023C4E90B87C4E91F
:103CA0000733C4E909336671A56084F8069020469D
:103CB000FFF74AFFF107626B12D4B3070BD4938965
:103CC0009BB243F4005393812046BDE8F88300245F
:103CD0002046BDE8F883D36843F08003D360EEE765
:103CE0004FF6DF731380D36843F02003D360E4E71B
:103CF0004B46324629460020FDF762FE0446CBE7DC
:103D00004B46324629460120FDF75AFE0446C3E7DA
:103D10004B46324629460320FDF752FE0446BBE7D8
:103D20000010014000440040004C004000140140DD
:103D3000816009E7417107E72DE9F043DFF814825C
:103D400008EBC00985B00546C70099F80C0D08F0CE
:103D500073FF044699F80D0D08F06EFF064699F8BA
:103D60000E0D69F01FF96B1CDBB2002C00F0AD806A
:103D700040F60C122372E280002E00F0C3803372F2
:103D800040F60C232046F38004223A2109F058F92A
:103D9000042230463A2109F053F908EB0703624A3E
:103DA000D3F8084D944200F09880604B9C4200F09C
:103DB0009E805F4B9C4200F0AB80474497F80F2DEC
:103DC000022A5CD0032A7ED05A4B5B4E012A18BFD0
:103DD0001E46A7886846FFF769FE27F03F07029B4B
:103DE000564AB3FBF6F63F04A2FB03233F0C47EA17
:103DF0009347A780228822F001021204120C22802D
:103E0000B2B2C6F30B069B0C002E59D04FF496713C
:103E100001FB03F34A49A1FB03139B0901339BB246
:103E200042F400422384A2832388464A9BB243F093
:103E300001032380238823F4816323F002031B04FE
:103E40001B0C4FF4804143F480632380218123883D
:103E500023F080031B041B0C238023889BB202EBFE
:103E6000451243F0010323800121002382F84055CD
:103E700082F8411582F8423505B0BDE8F083A68886
:103E80006846FFF713FE26F03F06029A2B4B3604D6
:103E9000A3FB0213360C46EA9346A680218821F044
:103EA00001010904090C21809B0C27490133920967
:103EB0002384A1FB02329209042A38BF0422B2E70C
:103EC00042F00102A2E7214E83E7002E3FF465AFE6
:103ED000337240F60C23F3805AE71D4B1A6A42F402
:103EE00000121A621A6A22F400121A6265E703F5D8
:103EF000F0331A6A42F480021A621A6A22F48002CB
:103F00001A625AE7042220463A2109F099F844E758
:103F100003F5EE331A6A42F400021A621A6A22F4B6
:103F200000021A6249E700BF0054004000580040F8
:103F3000005C0040804F1200009F240083DE1B4382
:103F4000D34D6210282E0020632D3E05C0270900A6
:103F500000380240000000202DE9F047954D90F90F
:103F600000108046807805EBC1060138CC0090B087
:103F7000D6F8081D14282ED8DFE810F053012601CA
:103F8000150057006100A200AA00CB01BD017D0011
:103F9000870045020D02E001C500D5003000380061
:103FA000AA019C015B01888A0C8B81B2824841EA9C
:103FB000044130EA010100F02681D8E90210521ACA
:103FC00042F2107163EB00038A4273F1000302D3E3
:103FD000152388F8023010B0BDE8F08798F8130078
:103FE0000882C8E90223122088F80200888A0C8B14
:103FF00080B240EA0440714C34EA000000F0B68020
:1040000000200E900F9001200F910E900E99002924
:1040100000F01E820F9914310F910F99096849051C
:10402000CBD5142388F80230D5E798F8110000F0BA
:10403000FE000882C8E90223052088F80200888A69
:104040000C8B80B240EA04405D4C34EA000000F082
:10405000A48000200090019001200191009000991F
:10406000002900F001820199143101910199096838
:104070004F05D6D4A1E798F8110040F0010008825E
:10408000C8E902230B2088F80200888A0C8B80B2D2
:1040900040EA04404B4C34EA00006FD0002004900A
:1040A00005900120059104900499002900F0D68123
:1040B000059914310591059909684D05B1D47CE73E
:1040C00098F813000882C8E90223072088F8020044
:1040D000888A0C8B80B240EA0440384C34EA0000F5
:1040E0005FD000200290039001200391029002997A
:1040F000002900F0C58103991431039103990968DF
:104100004E058ED459E7088820F480600004000C26
:10411000088098F8110000F0FE000882C8E9022328
:10412000102088F80200888A0C8B80B240EA044094
:10413000234C34EA000012D000200C900D90012096
:104140000D910C900C99002900F094810D99143177
:104150000D910D99096848053FF563AF2DE798F873
:104160001330FF2B06D198F810301BB1132388F8B9
:10417000023030E7112388F802302CE7D8F8140019
:10418000012800F09381022800F049820E20098B5B
:1041900088F80200C8E902231DE7062388F80230E8
:1041A00019E7D8F81400002800F07081082388F877
:1041B000023010E700000020010003008400070027
:1041C0008200070002000300088820F40060000459
:1041D000000C0880088880B240F48060088008885D
:1041E00080B240F480700880032088F80200888A3A
:1041F0000C8B81B2AB4841EA0441C8E9022330EAA2
:1042000001037FF4E8AE98F81230002B40F0D38120
:1042100098F81330FF2B00F04682042388F8023010
:10422000D9E6098889053FF5C8AE002388F8023031
:10423000D1E62C4494F80C0D08F0FEFC064694F8E8
:104240000D0D08F0F9FC984AB2F8A03501339BB285
:104250008246A2F8A03516B13368B2881A83BAF143
:10426000000F04D0DAF80030BAF804201A831121C4
:10427000304605F019FD1121504605F015FD4FF0AF
:10428000090965272EB13368B28819690A4240F0DE
:104290002881013F00F022810CF076FB04460D4698
:1042A0000CF072FB001B61EB0501052871F10003A6
:1042B000F6D3E7E7088880B240F4007008804FF634
:1042C000FF3088820121C8E9022388F8021082E6C3
:1042D000D8F81400002800F07281D8F8184014F8BB
:1042E000016B0E8201381225C8E90504C8E90223D2
:1042F00088F802506FE6888A0C8B81B2694841EADF
:10430000044130EA01017FF458AE0A2388F80230F4
:1043100061E6088880B240F480700880092088F83F
:104320000200888A0C8B81B25E4841EA0441C8E9E8
:10433000022330EA01037FF44EAEE6E700240125B4
:104340000A940B940B910A950A98002800F04A8170
:104350000B9814300B900B98006846077FF52DAE34
:10436000D8F81400032800F07281022800F2468178
:10437000088820F480600004000C0880088880B25F
:1043800040F400700880098A88F81C40C8E90223BC
:1043900088F802501FE60020012408900990099136
:1043A00008940898002800F01781099814300990A3
:1043B0000998006847077FF500AEEFF311851020DC
:1043C00080F31288088880B240F400700880D8F822
:1043D00018000E8A471CC8F81870EDB2067085F3F5
:1043E00011880D8AD8F818106FF001004E1CC8F81B
:1043F00018600D70C8E90223C8F8140088F81C4042
:1044000088F80240E7E50020069007900120079118
:104410000690069C002C00F0EB80079C1434079457
:10442000079C246864067FF5C8AD0C8AD8F818107C
:104430004D1CC8F818500C70D8F8141088F81C00DF
:104440000139C8E90223C8F8141088F80200C2E54F
:104450000F9918310F910F990968AEE50599183138
:10446000059105990968A8E501991831019101990B
:104470000968A2E50D9918310D910D9909689CE51F
:104480000399183103910399096896E5088880B269
:1044900040F4007008800121C8E9022388F8021066
:1044A00099E500BF01000300282E0020088820F4B1
:1044B00080600004000C0880EFF31184102080F36A
:1044C0001288088B088880B240F40070E4B208803B
:1044D00084F311880C2188F802105BE616B133686A
:1044E000B2885A830CF050FA04460D460CF04CFA90
:1044F000031B61EB0501052B71F10003F6D316B127
:104500003368B2881A830CF03FFA04460D460CF06B
:104510003BFA031B61EB0501052B71F10003F6D398
:10452000B9F101097FF4ADAE16B13368B2885A8390
:104530000CF02AFA04460D460CF026FA031B61EB38
:104540000501052B71F10003F6D3BAF1000F04D079
:10455000DAF80030BAF804205A830CF015FA044651
:104560000D460CF011FA031B61EB0501052B71F1EF
:104570000003F6D316B13368B2881A830CF004FA3C
:1045800004460D460CF000FA031B61EB0502052BF7
:1045900072F10003F6D3BAF1000F04D0DAF800305C
:1045A000BAF804201A8398F90000441C3FF43DAE89
:1045B000FFF7C2FB39E60F2388F802300BE50888C5
:1045C00080B240F4007008800121C8E9022388F815
:1045D0001C1088F80210FEE4099918310991099914
:1045E0000968EAE40B9918310B910B990968E4E426
:1045F00007991831079107990968DEE4D8F818007F
:10460000098A441CC8F818400170D8F81410C8F87A
:1046100008200139C8F81410C8F80C30DBE4088809
:1046200080B240F400600880EFF31184102080F322
:104630001288088B088820F480600004000CE4B223
:10464000088084F311880D2188F80210A2E50888FB
:1046500020F480600004000C0880EFF31184102027
:1046600080F31288D8F818000D8A461CC8F8186024
:104670000570088880B240F40070E4B2088084F3CA
:104680001188D8F81800098A441CC8F8184001702D
:10469000D8F814100C200239C8E90223C8F8141005
:1046A00088F8020097E498F81030002B3FF4B5AD7D
:1046B0002BE600BF38B5184D9DF814E005EB40140B
:1046C0004FEA401C94F8410500B938BD490084F810
:1046D0005325C4F8543584F851150023049984F8FF
:1046E00050E5022205F5A86584F85235C4F858153E
:1046F00084F85C3584F8422565440CF045F902469F
:104700000B462846FFF728FC94F84235002BF4D1DD
:1047100094F85C0538BD00BF282E002038B5184D30
:104720009DF814E005EB40144FEA401C94F8410555
:1047300000B938BD84F85325C4F85435012200234C
:10474000490005F5A86584F8522584F85C35049A7B
:1047500084F850E5022384F85115C4F8582584F8EC
:10476000423565440CF010F902460B462846FFF727
:10477000F3FB94F84235002BF4D194F85C0538BD76
:10478000282E0020F0B587B00023824A00930193C1
:10479000136843F48033136003E0009BB3F5A04F2C
:1047A00009D0136803F400330193009B0133009395
:1047B000019B002BF1D0774B1B6813F4003318BF1B
:1047C00001230193019B012B01D000BFFDE7714B39
:1047D00071491A6C714842F080521A640A6842F4B6
:1047E00040420A609A689A609A6842F400429A606D
:1047F0009A6842F4A0529A6058601A6842F0807237
:104800001A601A689201FCD5654A40F20571116080
:10481000996821F003019960996841F00201A2F5BD
:1048200080629960936803F00C03082BFAD19368B7
:1048300003F00C03042B00F08C80082B00F08E801A
:10484000584D594BC5F8F43A524BD5F8F41A9A68BA
:10485000564C5748C2F303122A44002692F8202DE2
:10486000D140544AC5F8F41AE260534A596FA26025
:10487000596B524A21F080015963596F41F08071A0
:104880005967196B0A431A635A6B5A639A6B9A6396
:104890001A6C4B490A431A64596C4A4A0A435A64CF
:1048A00002A948F2FF7302934FF6FF770396FFF7D2
:1048B0005FF800F580600297FFF75AF800F5806016
:1048C0000297FFF755F800F58060FFF751F800F503
:1048D0008060FFF74DF800F58060FFF749F800F5BC
:1048E0008060FFF745F800F58060FFF741F800F5BC
:1048F0008060FFF73DF80846FFF7D8F8D4F8FC30A1
:10490000029A3149314843F08073C4F8FC30304B8F
:10491000C3F8B01F5E60196841F001011960D5F855
:10492000F43A4FF47A71B3FBF1F3013BB3F1807FBA
:104930002849B2FBF1F2C0F8A42508D24FF0E022DA
:10494000F0215361072384F823109661136107B0A7
:10495000F0BD144D204BC5F8F43A75E75368516823
:10496000104D13F4800F01F03F01536814BF1A4A31
:104970000D4AB2FBF1F1074A5268C2F30142C3F398
:104980008813013201FB03F35200B3FBF2F3C5F8C5
:10499000F43A59E7003802400070004008544007DC
:1049A000003C0240000000200024F40000ED00E084
:1049B000000002400003FA0500000008FF916700B4
:1049C000FFC9FE103357070055CEACC5282E002076
:1049D000001000E040420F0000127A0082B0064B47
:1049E000002201920193019B03EB80000190019B47
:1049F000196002B0704700BF5028004010B51C205D
:104A000008F01AF91121044605F04EF94CB123685B
:104A1000A2885A83C8200BF0E5FF2368A2881A8376
:104A200010BDBDE81040C8200BF0DCBF704700BFD0
:104A3000704700BF704700BF10B5124C94F8B235F4
:104A400023B9114B4FF480225A6110BD4FF0E02280
:104A5000D2F8103D23F00603C2F8103DFEF774F8BB
:104A600094F8B235002BECD0D4F8B8359B68DB074E
:104A7000E7D5D4F8B426136823F0030161F30703E4
:104A80001360DEE7282E0020003C01402DE9F04FA6
:104A9000B34CD4F8B4355A69D2078BB002D50BB0F9
:104AA000BDE8F08F5A699B6912EA0309F7D0C9F390
:104AB000074319F4002F009340F0E180009B590751
:104AC00043D419F0020F5FFA89F603D0D4F8B43555
:104AD00002225A61B9F1000FC0F2EE8119F4006FA1
:104AE000C9F3072540F04A81330708D59D4B9E48FE
:104AF000D3F83C3D9847D4F8B43508225A61F706FC
:104B000000F1C481EE0600F16F81A90600F1E88092
:104B1000009BDA0609D5934B9348D3F84C3D984750
:104B2000D4F8B4354FF480125A61009B9B06B6D579
:104B30008C4B8D48D3F8503D9847D4F8B4354FF49A
:104B400000125A610BB0BDE8F08FD4F8B825936914
:104B5000D26913401FFA83FABAF1000FB1D0DFF81F
:104B60001882CDF80C90A8F1180500271AF0010F53
:104B700078D0FEB2D4F8B82504EB86031069D3F8D8
:104B8000C015536B8968F340DB01DBB203430B4074
:104B900013F00109D9B240F0AB810A0740F1C88196
:104BA000D8F8002008239360994619F0800F59D057
:104BB000D5E94CC0D5F82431D8F800E0ACEB0001C1
:104BC0008B42DEF8182028BF0B4692B20333B2EBBB
:104BD000930F47D9D4F8B82594F8AB95323604EB47
:104BE0008603CDE90178674698469446874237D9CF
:104BF000D5F82431391A994228BF194601F1030B1F
:104C0000D5F828314FEA9B0BB9F1000F10D18AB2C9
:104C100003329210D8F8B0650AD04846013053F8F4
:104C2000047B37608242F9D1D5E94C70D5F8283140
:104C300008440B44B842C5F82831C5F83401DEF801
:104C400018300AD195F81C11012202FA01F1DCF8A2
:104C5000342022EA0102CCF834209BB29B45C5D314
:104C6000DDE901785FEA5A0A07F1010708F1040853
:104C700005F128057FF47AAFDDF80C9021E7D4F830
:104C8000B8359D69DB691D402D0C3FF417AF04F565
:104C9000B568DFF8D0B004F2FC560027C24608E041
:104CA0006D0807F1010706F1040608F128083FF432
:104CB00005AFEB07F4D5F9B204EB8103D4F8B825BE
:104CC000D3F8FC359B6852691340D807DAB200F17B
:104CD0003F81930740F16781336802229A60DFE7E2
:104CE000D4F8B835D4F8C0159A680868C2F3410200
:104CF000022A06BF032262F30A006FF30A0008606B
:104D00005A6842F480725A6006A8FEF7CFFED4F8C3
:104D1000B425D4F8B815D368079D6FF38D23D360FD
:104D200088681249C0F34100014491F8D01003296A
:104D300000F05F810E490F480126294484F8AA65D6
:104D400081424FF04006A4F8AC6500F2AC810E2120
:104D500061F38D234FF40051D3605161D8E600BF59
:104D6000282E002000000020D0330020BC8507083A
:104D7000401E1BFF3F420F00E833002000238DF848
:104D8000133094F8BA368DF81330B64BB648D3F8D2
:104D9000443D9847D4F8B835D4F8B425986894F8C9
:104DA000B2354FF400615161002B3FF49DAEC20754
:104DB0007FF59AAE94F8BD36012B7FF495AE9DF841
:104DC0001330032B7FF490AED4F8B436A7491A6899
:104DD00042F001021A601A6842F003021A600B697D
:104DE00043F006030B617FE6D4F8B865D4F8B41538
:104DF0007368002723F0010373600597059B43F058
:104E000020030593059B67F38A130593059B0B61AC
:104E10000B690593BC46964B03E00A690592013B7A
:104E200002D0059A9006F8D494F8A92552B1914B76
:104E300003EB820EFF2253F8040F8260D86B734598
:104E40008260F8D10B2363F3070763F3070C4FF07D
:104E5000FF33B3614FF00113F3617761C6F810C0FF
:104E6000336885486FF30A13336094F8AB25D4F8A0
:104E7000FC35012A186100F0B5804FF480534B6176
:104E8000784B7948D3F8403D98473EE6D4F8B4359E
:104E90009A6922F010029A611A6AC2F3434002280A
:104EA00002F00F0100F0B080062800F087809A69B8
:104EB00042F010029A6125E694F8B2353BB1D4F87D
:104EC000B426136823F0030161F307031360D4F8D9
:104ED000B825644B6448D3F8481D536823F0010398
:104EE00053608847D4F8B4354FF000425A61F5E575
:104EF000516BD8F800005B4B4FF0010C0CFA07FC2B
:104F000021EA0C0151630122D3F8343D826031461D
:104F10005548984794F8AB35012B00F0B18019F053
:104F2000020F3FF442AED8F8003002229A6099E6B0
:104F3000CB0604D5D8F8003010229A6092E64806D5
:104F400058BF8946EBD5D8F8003040229A6089E6F0
:104F500094F8AB25336801208242986007D11A6922
:104F6000D8F87C33C2F312029B1AC8F88C33DBF8F2
:104F7000303D5046984794F8AB35012B7FF490AE06
:104F8000002F7FF48DAE94F8B936052B7FF488AEF0
:104F9000D4F8FC35384A1A61384A5A611A684FF019
:104FA00080221A607CE610077FF57AAEDBF8383D88
:104FB00050469847336808229A6071E601EB8101F8
:104FC00004EBC101D4F87866D1F83409C2F30A12AF
:104FD00002443068C4F8740B3068C4F8780BC1F828
:104FE000342964E7254A5A611A684FF080221A6012
:104FF00043E7002184F8AA154FF40071A4F8AC151A
:10500000092161F38D23A5E647F6F07010423FF4C5
:105010004EAFC2F30A1201EB810004EBC00002F1B3
:10502000030C5FEAAC0CD0F82869D4F878E64FEAB4
:10503000810818BF002006D00130DEF8007046F865
:10504000047B8445F8D1414404EBC101D1F828091F
:105050001044C1F82809D1F834090244C1F83429B0
:1050600025E700BF00000020D033002000ED00E065
:10507000400D0300E4330020180008609C39002034
:10508000002F7FF44CAF94F8B936042B7FF447AF70
:10509000D4F8FC352B4A1A612B4A5A611A684FF032
:1050A00080221A603BE72948A5F57401A1F510514B
:1050B000814203D80D2161F38D234BE62449254815
:1050C0002944814203D20C2161F38D2342E6224818
:1050D000A5F18C71A1F54341814203D80B2161F305
:1050E0008D2337E61D491E482944814203D20A21F7
:1050F00061F38D232EE61B491B482944814203D2CC
:10510000092161F38D2325E61848A5F1B771A1F5B2
:105110005851814203D2082161F38D231AE61449C4
:1051200014482944814203D2072161F38D2311E6FB
:10513000114912482944814234BF0621052161F3F7
:105140008D2307E6180008609C390020DFC8100096
:105150002013FBFE20D61300FF69180000D3CEFEFB
:1051600040771B00C05BB3FEC091210040AC27001C
:10517000C01D6AFE40E13300803C36FEE09C4100E9
:105180000378022B12D00E4943680269D1F8180245
:1051900010B41840D1F81042D1F80C12931E400AF6
:1051A00004FB030008445DF8044B7047044B42685D
:1051B000D3E9800100EB410000EB5220704700BFB3
:1051C000FC5900202DE9F84F12F0020E01D0002802
:1051D0003CD08A4DD5F80872002F43D14FF0FF3CE8
:1051E000874CE146E046E24600262768B84200F0D8
:1051F000D98094F80EB0BBF1000F4ED0BBF1010F77
:1052000016D1804F06F5817B07EB0B1B9BF807B08F
:105210001BF0010F0CD11BF07E0F09D15FEADB17E9
:1052200040F0B480D4F808B0D34501D2DA46B14694
:105230000136082E04F11004D7D1BCF1FF3F38D15C
:10524000B8F1FF3F30D06F4CC44633E06B4D95F85A
:10525000B431A5F58054E3B10123637002263046D2
:10526000BDE8F88FD5E9834606FB0744A042B5D3D5
:1052700095F8B43113B9012385F8B431614B01229B
:1052800000265A703046BDE8F88F95F8B431002BEF
:10529000E2D1012385F8B431DEE7B4460136082EA9
:1052A00004F11004A1D1C8E7B9F1FF3F18BFCC4603
:1052B00074D0544CD5F8986004EB0C1841F21809DE
:1052C000013648F8090041F21C090CF5817748F8CD
:1052D00009604FEA0718C5F8986044F8086004EBC5
:1052E00007164FF00008C6F8048004EB0716B679DD
:1052F000042ECAD8DFE806F0031952192F0012F065
:10530000010868D104EB0710D61090F80790032B22
:1053100066F3C71980F807905BD94FF6FF70834298
:1053200028BF034604EB07108380BEF1000F12D0A4
:10533000D5F89830D5F89C0001330130C5F8983085
:10534000C5F89C0004EB0C1041F21C05435104EB22
:10535000071304209871500705D504EB0710C37993
:1053600043F00103C371D30608D504EB0714E379B6
:10537000C3F34502013262F34603E371224B012677
:1053800003EB4C230B603046BDE8F88FB046013686
:10539000082E04F110047FF428AF4EE700263046B3
:1053A000BDE8F88F174C06F5817704EB071C4FEA30
:1053B00007189CF806C0BCF1000F01D1B44679E78C
:1053C000B446D5F89860013644F80860C5F898608E
:1053D0008BE74346A6E70D4BD3F8703D002BDDD09D
:1053E00009495D680A4A01EB4C210023A8470028BF
:1053F000D4D004EB07140223A37130E7FC5900203A
:10540000145A0020FC490020144A0020301D0020BE
:10541000F90D000870B5104E3378022B0F4B0BBFFF
:10542000020AC0F3D412C4B200F07F04D3F8000221
:1054300082B010440D460023032201A9FFF7C2FEEB
:10544000012807D13378022B019B0CBF23F814509D
:1054500043F8245002B070BDFC490020FC590020E4
:105460002DE9F04FDFF82C8198F80060032E85B00D
:105470000C46154643D001288CBF00220122022E83
:105480000B68019269D14FEA1329DFB24FF4807A99
:105490000138012820D84FF0010B9D4217D93C4E0E
:1054A000D6F878211AB1D6F89411994258D0D6F886
:1054B000000200234844092203A9FFF783FE0128C4
:1054C0002CD0022817D020B123689D42E8D825604F
:1054D000032005B0BDE8F08FF7B12D4B93F8B42150
:1054E00012B9012283F8B4210123022088F8013087
:1054F00005B0BDE8F08F022005B0BDE8F08F0128AF
:105500008CBF0023012301930B684FF0800AC3F383
:10551000D41903F07F07BBE7D346BEE798F8002015
:105520000399DDF804C0022A14D0032AE3D151F80C
:10553000273023F07043B3FA83F35B0963455F447C
:10554000236821D05B4457452360ECD309F101095E
:105550000027BAE731F81730EDE74FF4807AD6E745
:10556000D6F81012013A02EB41224902B2FBF1F2E5
:105570001344B3FBFBF20BFB12320AB15B449B1AE0
:105580009D4223608CD8A2E7AB42A2D39FE700BF25
:10559000FC590020FC4900202DE9F04FDFF86CB1E8
:1055A0009BF800C0BCF1020F894683B009688246AF
:1055B000174640F08C800BF58053CEB2D3F80052E2
:1055C000A6EB010805EB112590444FF48073984435
:1055D000B94208F1FF38B8FBF3F84CD2A844BCF14B
:1055E000030F07EB06040CBF80224FF48072641A8D
:1055F0009442A8EB050328BF144666B994422CBF19
:105600000A220B2201A92846FFF7DCFD012809D058
:1056100003B0BDE8F08F0B2201A92846FFF7D2FDA9
:105620000128F5D19BF800C0D9F80010BCF1020F99
:1056300001F1010323D0B44210D9019906F180424F
:10564000013A01EB8202043901EB840142F8043F84
:10565000914203F10103F9D1D9F80010A61B31449E
:10566000BAF1010FC9F8001021D08F4205F10105F0
:105670004FF00006B3D8012003B0BDE8F08FB4426C
:10568000ECD9019806F10042013A00EB42020238DF
:1056900000EB440022F8023F904203F10103F9D1EC
:1056A000A61B3144BAF1010FC9F80010DDD1B9428F
:1056B000DBD1BCF1020F1DD004F18044019B013C01
:1056C0004FF0FF3243F82420D9F80010CDE70BF556
:1056D000805301F07F06D3F80032BCF1030FC1F311
:1056E000D415A6EB01081D44904414BF4FF48073F9
:1056F00080236CE704F10044019B013C4FF6FF72EC
:10570000504623F8142003B0BDE8F08FFC49002078
:1057100030B50446C06983B010B9012003B030BD74
:105720000D460023032201A9FFF74CFD0128F5D106
:10573000B4F92030002B0ADA144B93F8B4210AB9DB
:1057400083F8B401124B01225A700220E6E7019A55
:10575000012D4FEA431102EB431303D0022D11D167
:10576000E5255554A268DA612278032A04D1002283
:105770001A775A779A77DA77626A5A83120C9A8282
:1057800003B030BDE268DA61EEE700BFFC590020EB
:10579000FC4900202DE9F04190F83C30002982B00E
:1057A000044614BF02210021042B7BD8DFE803F05C
:1057B000030C3D486900FFF7ABFF012870D1626B15
:1057C000002A75D184F83C00404EDFF808814FF67E
:1057D000F77706F5805516E0BA424FD867F00AF918
:1057E00001284FF000011DD1206BFFF713FE0128A7
:1057F00018D1019AD5F814122263531E8B4228BF88
:105800000B46C5F814323278236B032A01A91846D7
:105810009AB2E1D1434531D867F0ECF801284FF056
:105820000001E1D002B0BDE8F081426B04F130012B
:105830000020FFF7B1FE012832D1032384F83C3069
:105840002348E16AD0F89431D0F81022C0F89411BE
:105850005B1A02FB03F3D0F8782102EB4322C0F875
:105860007821D0F87C2102EB4323C0F87C31002161
:1058700000F5B870FFF74CFF012811D1042384F81C
:105880003C3094F82830042B04BF002384F82830DF
:10589000A36B8BB120469847012002B0BDE8F08190
:1058A0000228BFD194F82830042B09D00220B9E790
:1058B000022384F83C30B9E7012002B0BDE8F08152
:1058C000002384F828300220ACE700BFFC49002008
:1058D000FC590020F7FFFF0F38B590F8343004462C
:1058E000052B43D8DFE803F01E033C0F185E006B66
:1058F0004FF0FF31FFF78EFD012837D1E06AB8BBCA
:10590000032384F8343000212046FFF701FF0128EB
:105910002CD1042384F8343094F82830082B2BD071
:10592000012038BD204DD5F8082200F130010232A7
:105930000120FFF795FD012823D00238C0B20128CD
:1059400014D8052384F8343094F82830082B04BF89
:10595000002384F82830012385F8B531022038BDB2
:10596000C06A216BFFF756FD0128C9D0002038BD61
:10597000022384F83430F4E7002384F8283001202F
:1059800038BDE368D5F81012D4E90B2003EB4123AE
:10599000C5F81402C4E9033002B96062012384F837
:1059A0003430A5E7004DCFE7FC59002010B590F842
:1059B00038300446032B4DD8DFE803F0022F38437C
:1059C0002B4AC068117802F580530329D3F81012CE
:1059D000D3F894210CBF4FF0800C4FF4807C01FB76
:1059E0000CF100EB4120C4E90302D3F87801A0EBED
:1059F0004120C3F87801D3F87C01A0EB4121E06A93
:105A0000C3F87C1102EB0C01C3F89411C4E90C211A
:105A100048BB6262012384F8383016480021FFF742
:105A200077FE012811D1022384F83830626B04F12B
:105A300030010120FFF7B0FD012806D1032384F8CF
:105A4000383000212046FFF763FE431EDBB2012BF6
:105A500001D910BD022094F82830062B04BF002382
:105A600084F8283010BDA2EB0C022263D2E700BFFD
:105A7000FC4900206C5B00202DE9F0434368C3F330
:105A800008020A44B2F5007F83B004460D4605D2F1
:105A90002B446360012003B0BDE8F08390F91A2025
:105AA000501C0AD0444902F5817201EB0212D179EF
:105AB0006FF30001D171FF22A27694F91B20511CD3
:105AC00016D03D4802F5817100EB011200EB011187
:105AD000D279C879C2F34502012A86BF02F1FF32AA
:105AE00002F03F020022FF2662F34600C871E6760C
:105AF00094F800C0BCF1020FCAD0DFF8C480D8F817
:105B00001022B5EB422F4FEA422915DCD8F8187263
:105B10001F407A42AA420FDCEA194A4510D2206996
:105B20000028B7D0244A1278032A40D080B24FF61A
:105B3000F7729042ACD9ADE7002003B0BDE8F08326
:105B4000227E206912F0080626D0D8F89421411C44
:105B50008A4213D300D100214B44A5EB0905DB1B7E
:105B6000BCF1020F60613D44216163600846D7D1FA
:105B7000D8F82022B3EB422F8AD38BE798F8B421D0
:105B800022B9012388F8B431636820690A4A0126E2
:105B9000567094F800C0DFE701A966F02BFF0128DA
:105BA000CAD10199636894F800C02069D4E7034A18
:105BB00090427FF66DAF6DE7FC490020F7FFFF0FC5
:105BC000FC5900202DE9F04790F8384082B0054696
:105BD000032C00F2AD80DFE804F00219730BFFF72D
:105BE0007BFE012810D002280AD1032385F8383023
:105BF0002B6C002085F82800002B71D098470224D8
:105C0000204602B0BDE8F08785F838002B78022BDB
:105C100062D0484A6B68D2F8182203EA0208C8F337
:105C20004F282846FFF7ACFA424F0646A8EB00087B
:105C3000A7F5805901A9022200233046FFF7C2FAD6
:105C400008EB060401281FFA84FA4FF400724FF0A3
:105C500000010446D4D1019870F084FCEB694FF444
:105C60000071284613B16B68002B3DD0D7F8103275
:105C70005A1E924506F101060DD2FFF7FDFE0028DF
:105C8000D8D197F8B43113B9012387F8B43101237F
:105C900089F80130CEE7C3EBC353590201F5007117
:105CA0002846FFF7E9FE40B997F8B43113B901234C
:105CB00087F8B431204B01225A70022385F838301E
:105CC0002B6C002285F8282063B1284698470124D0
:105CD000204602B0BDE8F0876B68C3F34F28A0E709
:105CE00002248DE701248BE7019B4FF020324FF017
:105CF0002E0E4FF0100C1A605A6083F800E0C3F8C3
:105D000007206C6A1A625A6283F80BC0C3F8272016
:105D100083F820E083F821E0EA6B5C835A8724FA59
:105D20000CF422FA0CF29C8283F82BC09A869DE731
:105D3000002465E7FC590020FC4900202DE9F041D2
:105D4000B1F904300F2B82B00E460446174635D009
:105D50002046FFF715FA94F91B80B8F1FF3F3ED0BB
:105D6000554B41F2180203EB08118A58904211D1A9
:105D7000183303EB4825B38801331BB205EB4315F9
:105D8000B38020463D60FFF7FBF93060012002B090
:105D9000BDE8F08103F5805292F8B41100296AD071
:105DA00001225A702278022A69D02369002B50D12F
:105DB000002301203B6002B0BDE8F0814FF4007188
:105DC000FFF75AFE002852D04FF6FF73B3802046EB
:105DD000FFF7D6F994F91B80B8F1FF3FC0D12278C4
:105DE000022A54D02369002BDDD0334909780329D6
:105DF0000EBF32499BB24FF6F7718B4294BF00231E
:105E00000123002BCFD138B92D4A92F8B431002BA1
:105E10004ED0294B01225A700023112201A9FFF70D
:105E2000D1F9012842D1019D264BEB1A48BF03F25C
:105E3000FF13B3F5805F4FEA632230D3204A92F814
:105E4000B43113B9012382F8B4311B4B01225A70CB
:105E500027E0194A1278032A0EBF184A9BB24FF660
:105E6000F772934294BF00230123002BA0D100209E
:105E700002B0BDE8F081012182F8B41190E7104A28
:105E80006368D2F82022B3EB422F91D2EFE70C4A9D
:105E90006368D2F82012B3EB412FB4D3F1E74FFA85
:105EA00082F884F81B80002D7FF465AF22787AE7B2
:105EB000012382F8B431ACE7FC490020F7FFFF0F63
:105EC000FC590020144A00202DE9F04790F83030AA
:105ED00086B00446042B54D8DFE813F005000E000A
:105EE0005600F8004F00C44867F03EF94FF6FF72C5
:105EF0000123228484F83030DFF8FC8204F11C0591
:105F000001AE04F13109324629464046FFF716FF3B
:105F1000012800F00281022833D1B84901F58055EB
:105F200095F9D221531C0AD002F5817201EB0212BD
:105F3000D3796FF30003D371FF2385F8D23195F93C
:105F4000D3315F1C16D003F5817301EB031201EB13
:105F50000313D279D979C2F34502012A86BF02F12F
:105F6000FF3202F03F02002262F34601FF22D971A4
:105F700085F8D321042384F830300020E36A2070B0
:105F8000984706B0BDE8F0879D4D95F8E031002BAD
:105F9000F7D1994F04F11C0901AE4FF009083246C0
:105FA00049463846FFF7CAFE012840F02181019892
:105FB000002800F0FD800378E52B01D0002BEED106
:105FC000904A821A48BF02F2FF12B2F5805F4FEA90
:105FD000622380F05C8189491B018B4A13449A7BC0
:105FE000042A0CD0D5F898200132C5F898205A60C0
:105FF00004229A73D5F89C300133C5F89C3095F98A
:10600000D2315E1C0AD003F5817301EB0313FF222A
:1060100085F8D221DA796FF30002DA7195F9D3317C
:106020005A1C18D003F5817301EB031201EB031323
:10603000D279C2F34502012A4FF0FF0188BF02F175
:10604000FF3285F8D311D9798CBF02F03F020022CC
:1060500062F34601D9712022002170F083FA019B7E
:10606000D4F83120D4F8351059601A60B4F83920CA
:1060700094F83B1099721A81019B627EDA7203A830
:1060800003F01EF8002800F0E5809DF80E509DF802
:106090000F10BDF80C00019B9DF8102041EA45113E
:1060A000A0F2BC7041EA40218DB219829DF8111016
:1060B000D20242EA41129DF8121042EA510290B215
:1060C000DA8103221D83D88284F83020237E98064B
:1060D00008D5E0690023112202A9FFF773F801280F
:1060E0007FF44FAF204667F03FF82369002B00F0A4
:1060F0008D80237E03F0F70213F00403227640F034
:106100009380122A00F0B1800022E36A84F82820EC
:106110002046984706B0BDE8F087019F002F00F0A9
:10612000C2803B78002B00F0BE8097F80BA01AF0DD
:10613000080F7FF4E8AE0B224946384670F0ACF900
:1061400000287FF4E0AE637E8AEA0303D90640F1BB
:10615000EB802A4901F5805595F9D2315A1C0AD0B5
:1061600003F5817301EB0313FF2285F8D221DA795D
:1061700060F30002DA7195F9D321571C3FF4FAAEAF
:1061800002F5817201EB021301EB0211DB79CA798E
:10619000C3F34503012B86BF03F1FF3303F03F0335
:1061A000002363F34602FF23CA7185F8D331E1E689
:1061B00095F8B831022B3FF4DDAE95F8E031002BB5
:1061C0007FF4D8AEC5E97D3385F8F03185F8EC3140
:1061D000D5F8CC31C5F8E431D5F8143285F8E08132
:1061E000C5F8E8313846FFF7EDFC01283FF4D7AE9B
:1061F00002283FF4BFAEC4E6B45B0020FC49002097
:10620000FC590020144A0020145A0020237E19074C
:106210007FF57AAF664B93F89821002A7FF4B1AEF0
:10622000072283F898216FE7A568E66A002384F8BF
:10623000283029462046FFF71FFC00286ED194F82D
:106240002830002B7FF49DAE0223C4E90B6584F84F
:10625000283096E6019B6FF07E01472219745A742C
:106260009873D87344F281752BE7626AE16AA1637F
:10627000042084F82800C4E90B22C4E9023384F81E
:106280003C3063636362204666F06EFF79E695F802
:10629000B43113B9012385F8B431464901234B7059
:1062A0006FF00F0399E6434901F5805595F9D23116
:1062B0005F1C0AD003F5817301EB0313DA796FF3E6
:1062C0000002DA71FF2385F8D23195F9D3315E1CD3
:1062D00016D003F5817301EB031201EB0313D2799E
:1062E000D979C2F34502012A86BF02F1FF3202F0DA
:1062F0003F02002262F34601FF22D97185F8D321C3
:10630000237ED8067FF536AE2B4866F02DFF4FF67C
:10631000FF720223228484F8303036E6002E3FF4E8
:1063200030AE2046B0472CE6BA8A7B8B204D43EA3C
:1063300002436362D5F81022FB69A3605202B3FBEB
:10634000F2F102FB113109B113445B1AE36084F8E6
:1063500019A095F9D23117495E1C0AD003F5817353
:1063600001EB0313DA796FF30002DA71FF2385F88A
:10637000D23195F9D321501C16D002F5817201EB70
:10638000021301EB0211DB79CA79C3F34503012B38
:1063900086BF03F1FF3303F03F03002363F346029C
:1063A000FF23CA7185F8D331032384F830308DE69A
:1063B000FC590020FC490020B45B002010B5037894
:1063C00090F818C0023B012B044602D91CF0060FBE
:1063D0006AD11CF0200F44D194F91A30591C0AD00C
:1063E000384A03F5817302EB0313FF21DA796FF367
:1063F0000002DA71A17694F91B305A1C16D031498B
:1064000003F5817301EB031201EB0313D279D97900
:10641000C2F34502012A86BF02F1FF3202F03F02B9
:10642000002262F34601FF22D971E2761CF0080FC8
:106430000ED0254B93F89821072A06D093F8B42163
:10644000002A3BD01F4A01215170002283F8982175
:10645000E26A0023237084F8283022B3BDE810409C
:10646000104700231949E0691A018A58904206D062
:106470000133082BB0D01A018A589042F8D1114943
:1064800003F5817301EB0312D279C2F34502012AAD
:1064900012D9013A02F03F0201EB0313D97962F3FA
:1064A0004601D97198E710BD0121FFF731F90128A4
:1064B000F9D194F818C08CE70022EDE7012283F8A7
:1064C000B421BFE7FC490020FC590020145A0020E9
:1064D0004FF0FF302DE9F041344A354D044600239A
:1064E00004E00133082B02F1100216D011780429C0
:1064F000F7D103F5817105EB0111C979CF07F0D40C
:10650000661C52F80A1C01D08142EAD21C460133B3
:10651000082B084602F11002E8D1631C02D10120C9
:10652000BDE8F081224DDFF8988004F5817705EB16
:1065300007139988F9B91F4ED8F8703D06EB44212E
:1065400023B3D3F80C801C4A41F2180305EB041462
:10655000E0580023C047C8B1022824D106F6E876E7
:1065600005EB0715D6F89C300122013BC6F89C309C
:10657000AA710020D4E7D8F8703D3BB19A6841F287
:10658000180005EB041318589047D4E70B4BD3F8C9
:106590009C2005EB07150320013A0121C3F89C203C
:1065A000A87183F8A0100020BDE8F081225A0020D5
:1065B000FC490020144A0020710E0008FC590020FC
:1065C000301D00202DE9F04F90F82830013B83B0BA
:1065D0000446082B0BD8DFE803F0383C1E230529BE
:1065E0000A2E33000121FFF7D5F8012802D003B0AD
:1065F000BDE8F08F2378002284F82820002BF6D005
:10660000D4E901138B4238BF0B46226CA3600321EF
:1066100084F82810E262204603B0BDE8F04FCDE6D2
:10662000002103B0BDE8F04FFFF7B4B803B0BDE8F8
:10663000F04FFFF7BBB903B0BDE8F04FFFF74CB91F
:1066400003B0BDE8F04FFFF7BDBA03B0BDE8F04FAF
:106650003AE4534F4368D7F81852016BD7F8102229
:106660001D406818B0EB422F4FEA42269C46C0F00E
:10667000938094F800E0DFF82C91A7F5805A4FF64C
:10668000F778BEF1020F14D02069002857D1D4F852
:1066900004C0A368E26A634538BF63460021A36073
:1066A00084F82810002AA2D0204603B0BDE8F04F9D
:1066B0001047D4F804C0D7F82022BCEB422FE8D210
:1066C0002069227E12072CD5D7F8942100F1010C05
:1066D000624522D297F8B42122B9012387F8B43158
:1066E0006368216B01228AF8012094F800E0891B7D
:1066F000294433445B1B8E42C4E904C063602163B8
:106700009C464FF00005BCD9BEF1020F3ED0206977
:106710000028BED0DFF890B01FE0E8D14FF0000CA9
:10672000E5E701A966F066F901287FF460AF20690A
:10673000DDF804C094F800E06368216BD7E79AF8AD
:106740000020032AD3461AD082B2424594BF0022C9
:106750000122002AB5D0D4F804C09BF80030032BE6
:106760000EBF104B80B24FF6F773984294BF0020D3
:10677000012000288DD18C44C4F804C089E7484525
:1067800094BF00220122002A9BD0E4E7D7F8202200
:10679000B3EB422FEFD37CE794F800E0B4E700BFFF
:1067A000FC590020F7FFFF0FFC49002010B5184CE2
:1067B0001848442200216FF0D5FE237804F5805458
:1067C0004FF6FF70D4F81C22A4F8D201022B4FF030
:1067D000030118BF03234FF0100C84F8D01104F507
:1067E000DC700021C4F8C82184F8B831C4F8DC2179
:1067F00084F8D1C1FFF740F938B994F8E03123B9F2
:10680000C4E97933022284F8E021012010BD00BFE1
:10681000FC490020B45B002070B51A4D1A4BC5F836
:106820009C3B1A4B85F8A81B002683F8206A05F6C6
:106830009C33C0E954330D230446C0F8583140F26C
:106840000113C0F85C6100F5A271A0F8443168F052
:106850009BFFE378C4F8B4631F22C4F8B02301227D
:1068600005F599659342C4F8A853A4F89C2308BF82
:10687000C4F8AC5304F567712046BDE8704068F079
:1068800083BF00BF282E002055534253301D0020E7
:10689000F0B50B7813F0600683B00C46054633D094
:1068A000202E2DD14A78FE2A6BD0FF2A63D14A8848
:1068B000002A40F08B80CA88002A40F087801906A1
:1068C00000F184806148624B80F8202AC5F8B42327
:1068D000EA78012183F8E814A5F89C1303F599637D
:1068E0001F21012AC5F8B013C5F8A83305F5677153
:1068F00008BFC5F8AC33284668F046FF002600E024
:106900000026304603B0F0BD4B780A2B6AD00B2B23
:1069100063D0012BF5D18B88D9B21B0676D40196B2
:10692000019BC06843F010030193019B036103695D
:106930000193484B03E002690192013B02D0019AA6
:10694000D206F8D42846424F68F00EFE0223217981
:106950004022284668F03AFE97F8E834022B6DD0C2
:1069600094F90420002ACCDA012BCAD00121284650
:10697000FFF752FFC5E766F067F80226304603B01E
:10698000F0BD4E8816BBCC88012C1FD118061DD532
:106990002F4FD7F800359B699847C0B287F8AC0BEA
:1069A000A0B1022307F6AC3785F811314FF480739C
:1069B000C5E94E44C5E94A77C5E94C46A5F81C31FE
:1069C00005F58E71284668F071FE9AE7284666F054
:1069D0003BF80226304603B0F0BD1D4B4A8883F8D1
:1069E000AD2B8EE7022280F811214FF48072A0F8BF
:1069F0001C21194A0123C0E94E33C0E94A22C0E9EB
:106A00004C3600F58E7168F051FE7AE70096009BD7
:106A1000C06843F020030093009B61F38A13009346
:106A2000009B0361036900930A4B03E00269009233
:106A3000013B87D0009A9706F8D483E78121284646
:106A400068F058FD002387F8E8345AE7301D00202D
:106A5000282E0020400D0300D539002010B50D4B25
:106A600093F8203A022B07D0033B012B02D80021D8
:106A7000FFF7D2FE002010BD074B93F8D514044653
:106A800065F0EEFB0028F5DA01212046FFF7C4FE91
:106A9000F0E700BF301D0020282E0020F8B5404E42
:106AA00096F8205A074655B1012D06D13D4B93F873
:106AB000D51465F0D5FB002832DB0020F8BD394C39
:106AC000B0F8B433D4F8CC24C4F8A02B1F2BD4F8DE
:106AD000D024C4F8A42B08D1334BD4F8C8249A424C
:106AE00003D194F8D51401291FD994F8AE3B04EBD7
:106AF000C3020133DBB2042B4FF0050108BF0023B2
:106B000082F8B01B4FF4005184F8AE3B38460223A4
:106B1000C2F8B41B84F8E834FBF78CF90020F8BD08
:106B200029463846FFF778FEC7E794F8D634013B8C
:106B30000F2BDAD865F094FB002827DB96F8203A73
:106B4000013B022BB9D9B4F8D03B1BB3042286F821
:106B5000202A164AC7F85C51C7E95422D4F8D02439
:106B600084F8A85B934228BF1346D4F8A42BC7F837
:106B7000583140F20111A7F84411D31A07F5A27158
:106B80003846C4F8A43B68F0FFFD96E73846FBF7AB
:106B900051F992E719463846FFF73EFE8DE700BFF0
:106BA000301D0020282E002055534243FC39002080
:106BB00000207047704700BF704700BFD0ED007ADB
:106BC000D0ED036A30EE677AE6EE877AB0EE670AB8
:106BD000C0ED007A704700BFD0ED017AF5EE407A43
:106BE000F1EE10FA09D1DFED0E7A60EEA70AB7EEEA
:106BF000007AC7EE207AC0ED017A31EE277AD0ED27
:106C0000007A80ED021AC1EE076A30EE677AC0EDB5
:106C1000036AE6EE877AB0EE670AC0ED007A704745
:106C2000DB0FC94090ED017AD0ED036AD0ED027A16
:106C300030EE470AA6EE807A90ED000A80ED017AE8
:106C400037EE676AE6EE867A37EEC07AC0ED027AF2
:106C5000A6EE870A80ED000A704700BFD0ED056AF6
:106C6000D0ED017A90ED007A90ED066AD0ED025AEF
:106C700090ED035A80ED050A66EEA77AC0ED066A2C
:106C8000E7EE007A90ED077AE5EE867A90ED086AF5
:106C9000D0ED045A80ED087AE5EE477AE5EEC67A43
:106CA000B0EE670AC0ED077A704700BFD0ED057AF5
:106CB00090ED006A90ED037AD0ED025AE6EE007A8C
:106CC000F0EE406AB0EE670A90ED016AD0ED047A0A
:106CD00027EE407A67EEC07AA6EE267AE5EEA67A2F
:106CE00090ED066AC0ED067A36EE077A80ED057AF9
:106CF000704700BF03685A1C02601970704700BFDC
:106D000003685A1C02601970704700BF024B186874
:106D100003681B68184700BF205C0020007970479B
:106D20000079C0F34010704700794009704700BFF8
:106D300090F83C20034602F0FF0012B1002283F8D5
:106D40003C2070474FF48053838170474FF40063B9
:106D5000838170474FF40063838170474FF4006371
:106D6000838170474FF40063838170474FF4006361
:106D7000838170474FF4006383817047074B10B4E1
:106D800003F11001002453F8042B824208BF43F89A
:106D9000044C8B42F7D15DF8044B7047245C002013
:106DA00070B5374C638CA08AB4F92C50B4F92660C6
:106DB000B4F91AC0C01A238C00FB03F3B4F92A00FB
:106DC00005EBE335C00290FBF5F000EBE330A0F5F6
:106DD0007A6EB4F9243020630EFB0EF52D1305FBFB
:106DE00006F605FB03F3B4F91C500EFB0CFC4FEA4E
:106DF000EC2C0EFB05FE1B14B4F918500CEBE62C22
:106E000003EB6E330CEB850C0233B4F93450A66BF4
:106E1000E48B9B1003F500430CFA05FC04FB03F321
:106E20000CF1020C4CF25034A6EBAC0C2C4104FBE0
:106E30000CF4002C4FEAD333ABBF6400B4FBF3F384
:106E4000B4FBF3F35B0089B11C120E4D04FB04F498
:106E500040F6DE3606FB04F403FB05F5241404EBD0
:106E6000254404F6CF6403EB24130B602AB100EB36
:106E700080004000083000111060012070BD00BF8C
:106E8000205C002043E3FFFF012070470120704792
:106E90002DE9F84F6E4DD5F83CC0B5F84000B5F976
:106EA0004A90B5F846E0C0EB2C1303FB03F4B5F9A8
:106EB0004430241303FB04F44000B5F94230C0EB26
:106EC000EC0003FB00F0A41304EBE024B5F9483018
:106ED000AC650F46A4F5FA31164683FB013281FBFF
:106EE000018C12034FEAE97B42EA13524FEA033A5C
:106EF00009FB0CF308FB0B3BA9FB0839D9441B0A1F
:106F000043EA096313EB0A0342EB292202F500422C
:106F1000A3FB0E390EFB029E4FEAEE734FEA6E02A0
:106F200053EA6E0E4FF0000000F08580B5F95090E6
:106F300009FB0CFEB5F94EC08CFB011C4FEAE97A47
:106F40004FEA4C4C08FB0AEE4CEAD13CA9FB0898EE
:106F5000490411EB0901F04448EB0C0C4018E96DB1
:106F6000C1F58019B5F94C1009F0004E4FEAC97807
:106F7000B8EB00080CEBC1014EEA590E6EEB010EA6
:106F800018EB080C4EEB0E011CEB080C4EEB01014C
:106F90004FEA81194FEA8C1049EA9C691CEB000CFE
:106FA00041EB0901890041EA9C714FEA8C0C1CEB12
:106FB000080C4EEB01014FEA8C00890010EB080031
:106FC00041EA9C714EEB010169F0A4FCB5F9562031
:106FD000B5F954E0B5F952504FEA6138430B43EA32
:106FE000C14302FB08FC4FEAE27903FB09C9A2FB9B
:106FF000032CCC4402FB08F803FB0C88A2FB032CF7
:10700000C444520E42EACC12121841EB6C6C4FEAA7
:10701000EE730EFB01F103FB0011AEFB00300144E7
:10702000DB0C43EA4133D0184CEBE141000A40EA63
:10703000016000EB05100FB1000A386026B104EBC7
:1070400084048034241234600120BDE8F88F00BF2E
:10705000205C002031B10A4BD3ED1E7AFDEEE77AB9
:10706000C1ED007A52B1064B9FED067AD3ED1F7A3F
:1070700067EE877AFDEEE77AC2ED007A012070476D
:10708000205C00200000C8422DE9F04F634D85B020
:10709000B5F88E30D5F88000B5F88C8001911B02D0
:1070A000B5F88810B5F88A60B5F89040C01A67EB5B
:1070B00007074FEA014EA8FB001CB5F8863008FB15
:1070C00007CCC90941EA4C6111EB0E0193464FEA26
:1070D000C332A6FB003E06FB07EE4FEA132343EA4A
:1070E0000E634FEAEC1C4CF1000C9B18A4FB00262D
:1070F00004FB07644FEAD25242EA44224FEA2E2EA2
:107100004FEAE4544EF1000E12F5FA6944F100061C
:10711000B9F5FA6F029476F10004039631DA029C15
:10712000A2FB02A602FB04F806EB48044FEA84081F
:107130004FEA8A0616EB0A0648EA9A7844EB0808F2
:107140004FEA560A4AEAC87AB608354CB1EB0A014A
:1071500046EA88766CEB680C9B1B039E6EEBA80ED0
:10716000A1454FF0FF3476EB040427DB00FB07F763
:10717000A0FB000202EB4707C00F40EA4700B9EB53
:107180000009019C8CB1D5F89400A0FB033200FBF0
:107190000E2E5B0D43EACE235B1A4FEA6E5E6EEB5A
:1071A0000C0CDB0B43EA4C432360BBF1000F01D016
:1071B000CBF80090012005B0BDE8F08F40F6AC564A
:1071C000029C921944F1000402FB04F4A2FB028227
:1071D00002EB4404E6004FEAC802B8EB020246EABA
:1071E000587664EB060651184CEB060C18EB0806B3
:1071F00044EB040A16EB080644EB0A0A4FEA8A0A33
:107200004AEA967AB600B6EB08026AEB0404520822
:1072100042EAC4729B1A6EEB640EA7E7205C002062
:1072200024FAFFFF0120704710B4114B114C1B686A
:10723000D4F898001B1AFA2B0FD811B1D4F8A0304B
:107240000B6032B1D4F8A430136001205DF8044B18
:10725000704701205DF8044B7047074A136800200F
:1072600023F0040384F89C0013605DF8044B70471E
:107270004C270020205C002000000010064B00225C
:107280000021C3F8A820C3F8AC20C3F8B020C3F88D
:10729000B4100120704700BF205C0020104B114A41
:1072A0001B68D2F8B4105B1AFA2B16D8D2ED2A6AF2
:1072B00092ED2B7AD2ED2C7AFDEEE66ABDEEC77A1E
:1072C00016EE903AFDEEE77AC38617EE103A038782
:1072D00017EE903A4387012070470020704700BFA7
:1072E0004C270020205C0020024BD3F8B8305B68AC
:1072F000184700BF205C0020024BD3F8B83008309C
:107300009B681847205C00200120704701207047CF
:107310000120704738B51446002944D0344B9FED06
:10732000356AD3ED2F7AB3F9D42093ED310AB8EE54
:10733000E77AD3ED367AC7EE066A0D4604EE902A58
:10734000B3F9D020F8EEE77A05EE902AB3F9D2200F
:1073500087EE864AF8EEE44A05EE102AF8EEE55A82
:10736000B3F9CE20D3ED327AB3F9CC30E6EEA45A9D
:1073700006EE102AB8EEE77AB8EEC55AB8EEC66A3D
:10738000A6EEA57AA6EE856A07EE903AB8EEC00A98
:10739000F8EEE77AA6EE870AE6EE867AA4EE270AEA
:1073A0006AF036F928600CB3114BDFED125A93EDF9
:1073B000367AB3F9C220B3F9C0309FED0F0AB8EEA8
:1073C000C76A07EE902A86EE257A06EE903AF8EE26
:1073D000E77AF8EEE66A67EE277AB6EE006AE6EE3E
:1073E000867A27EE800A6AF013F92060012038BD02
:1073F000205C00200000F04A0000C8422DE9F04166
:107400000446D0E90030134483421DD88E188E42C2
:1074100017D00D4604F10C08002701E0AE4210D051
:1074200023695A1C2261234415F8010B1873042A9E
:10743000F4D141462046FBF7B3FBAE42C4E90470E9
:10744000EED16069BDE8F0814FF0FF30FAE700BF90
:1074500070B50446234894F9103003EB83031546B6
:1074600050F82300A3689A0782B00CD5019068F009
:107470008DFA0198294668F089FAA3689B0717D509
:10748000012002B070BD636913B11A689B885383F1
:10749000154B164A1B6856684FEAC30C144BA3FBE6
:1074A0000C3C4FEA9C1C53689B1B9C45FBD2DDE7C0
:1074B0000D4B0E491A680E4B4FF4FA7000FB02F2A6
:1074C000A3FB0232486892094B681B1A9A42FBD20E
:1074D0006369002BD4D01A689B881383012002B003
:1074E00070BD00BF600D0020CC330020001000E014
:1074F000D34D621010B504682379012B84B010D0ED
:10750000022B0BD1A368DB074FF0F0024CBFFF2129
:107510007F21204604B0BDE8104099E7002004B068
:1075200010BDA268617C94F9100002F00102019282
:107530000DF10F020092F024FF228DF80F40FDF7AD
:10754000EDF804B010BD00BF10B504682379CA433C
:1075500041EA0211012B84B0CAB20ED0022B09D12C
:10756000A368DB074CBFD2215221204604B0BDE8FE
:1075700010406DE7002004B010BD8DF80F20A26808
:10758000617C94F9100002F001020DF10F04CDE9C5
:107590000042D222FDF7C2F804B010BD10B5046855
:1075A0002379012B84B010D0022B0BD1A368DB0709
:1075B0004FF0B4024CBFFF217F21204604B0BDE84C
:1075C000104045E7002004B010BDA268617C94F92A
:1075D000100002F0010201920DF10F020092B4249A
:1075E000FF228DF80F40FDF799F804B010BD00BFE1
:1075F00010B504682379012B84B00FD0022B0AD177
:10760000A368DB070A4620464CBFA521252104B00C
:10761000BDE810401CE7002004B010BDA26894F93A
:1076200010008DF80F1002F00102617C0DF10F04C3
:10763000CDE90042A522FDF771F804B010BD00BFEE
:1076400010B504682379012B84B010D0022B0BD124
:10765000A368DB074FF096024CBFFF217F21204635
:1076600004B0BDE81040F3E6002004B010BDA268ED
:10767000617C94F9100002F0010201920DF10F02F9
:1076800000929624FF228DF80F40FDF747F804B0D2
:1076900010BD00BF10B504682379012B84B00FD052
:1076A000022B0AD1A368DB070A4620464CBF87217C
:1076B000072104B0BDE81040CAE6002004B010BDA8
:1076C000A26894F910008DF80F1002F00102617C9D
:1076D0000DF10F04CDE900428722FDF71FF804B039
:1076E00010BD00BF10B504682379C901012B84B017
:1076F000CAB20AD0022B05D17821204604B0BDE8D9
:107700001040A5E6002004B010BD8DF80F20A2683F
:10771000617C94F9100002F001020DF10F04CDE933
:1077200000427822FCF7FAFF04B010BD10B50468DF
:107730002379012B84B010D0022B0BD1A368DB0777
:107740004FF055024CBFA5212521204604B0BDE8CD
:1077500010407DE6002004B010BDA268617C94F961
:10776000100002F0010201920DF10F020092552467
:10777000A5228DF80F40FCF7D1FF04B010BD00BF6B
:1077800010B504682379012B84B010D0022B0BD1E3
:10779000A368DB074FF02E024CBFF4217421204672
:1077A00004B0BDE8104053E6002004B010BDA2684C
:1077B000617C94F9100002F0010201920DF10F02B8
:1077C00000922E24F4228DF80F40FCF7A7FF04B09E
:1077D00010BD00BF10B5154B04689A8E2379920135
:1077E0003432012B84B0D2B20ED0022B09D1A3685F
:1077F000DB074CBFF4217421204604B0BDE81040E3
:1078000026E6002004B010BD8DF80F20A268617C30
:1078100094F9100002F001020DF10F04CDE90042CD
:10782000F422FCF77BFF04B010BD00BF205C0020F9
:1078300010B504682379012B84B00ED0022B09D136
:10784000A368DB074FF031024CBFF42174212046BE
:10785000FFF7FEFD012004B010BDA268617C94F921
:10786000100002F0010201920DF10F02009231248A
:10787000F4228DF80F40FCF751FF012004B010BD39
:1078800010B504682379012B84B00BD0022B06D1EC
:1078900001225821204604B0BDE81040D8E5002060
:1078A00004B010BDA26894F91000617C8DF80F300F
:1078B00002F0010201920DF10F0200925822FCF732
:1078C0002DFF04B010BD00BF10B504682379012B53
:1078D00084B00BD0022B06D101224821204604B0EF
:1078E000BDE81040B4E5002004B010BDA26894F9D2
:1078F0001000617C8DF80F3002F0010201920DF151
:107900000F0200924822FCF709FF04B010BD00BF2F
:1079100010B504682379012B84B00BD0022B06D15B
:107920001A460821204604B0BDE8104090E500202A
:1079300004B010BDA268617C94F9100002F001024D
:1079400001920DF10F020092022408228DF80F40DF
:10795000FCF7E4FE04B010BD10B504682379012BD8
:1079600084B00BD0022B06D101220821204604B09E
:10797000BDE810406CE5002004B010BDA26894F989
:107980001000617C8DF80F3002F0010201920DF1C0
:107990000F0200920822FCF7C1FE04B010BD00BF28
:1079A0002DE9F0410C4E356873691D4011D0DFF8A8
:1079B0002C800127B5FA85F4C4F11F0408EB840379
:1079C00007FA04F4D3F8DC0003689847A543746110
:1079D000F0D1BDE8F08100BF003C0140205C0020F8
:1079E0002DE9F041684CD4F81C0190B028B1674AE9
:1079F0000321FBF715FAD4F81C01654D0021FBF7B4
:107A00008BFAD4F81C61D6F80480D8F81030002125
:107A10001F0B4FEA132E4B0105EB4110EA5887EA82
:107A2000123C8EEA12220CF0030C02F00F025CEA08
:107A3000020401F1010106D01029ECD10020F06010
:107A400010B0BDE8F081017FD8F80020F06019B1D6
:107A5000204610B0BDE8F081B2F844104D4F6FEAF7
:107A600041416FEA514189B2A2F84410118889B2AC
:107A700041F08001118098F80610B2F820C011F092
:107A8000040F98F8051017F801E014BF0421012134
:107A900001FA0EF189B21FFA8CFC2CEA010CA2F853
:107AA00020C0B2F820C01FFA8CFC41EA0C011184FE
:107AB000118889B241F0010111804168364A914232
:107AC00036490A6B1D440CBF42F4001242F4800296
:107AD0004FF0070C0A6333463149A5F81CC0032256
:107AE000FBF788FCF3689868FBF7ACFEF3689868CE
:107AF000036823F001030360FBF7A4FE0023716811
:107B00000693CDE90C33CDE90E330A934B79032B61
:107B100006D8DFE803F035312D020A6802F140048F
:107B20000B7CF16807EB83071E4B88687A6801922B
:107B3000CDE902434FF400330B9340F22B31402246
:107B40004FF480430591049209934FF480624FF4FF
:107B5000805301A90792089365F0F8F9F3689A68D1
:107B60001368012043F01003136010B0BDE8F081EA
:107B70000A6802F13C04D3E70A6802F13804CFE74F
:107B80000A6802F13404CBE7205C0020009F240047
:107B9000F80A0020B0860708006002400038024062
:107BA000A1020008405D002010B5114CD4F81C0162
:107BB00028B1104A6421FBF733F9D4F81C010021E5
:107BC000FBF7AAF9D4F81C315B681A68B2F84430A4
:107BD0006FEA43436FEA53439BB2A2F844301388E1
:107BE00001219BB20B43138084F8CC1D10BD00BF54
:107BF000205C0020009F240010B54FEA511E024473
:107C000000EB8E0C624529D901F01F014FF0FF34C3
:107C100004FA01F350F82E100B4093FAA3F3B3FAD1
:107C200083F3DBB2202B16D10CF104018A4202D877
:107C300017E08A4212D98C460431DCF8003093FAFE
:107C4000A3F3B3FA83F3DBB2202BF2D0ACEB00004A
:107C500003EBC00010BD03EB4E1010BD4FF0FF3022
:107C600010BD204610BD00BF30B503694268474DC6
:107C700083B00BB9002A63D0D0ED067AC46A013311
:107C800077EE807A0361631C012BC0ED067AC36234
:107C900046D0D0ED075A90ED097A296807EE903A60
:107CA00030EE656AF8EEE76A8A1AC6EE267A8168CF
:107CB0008A4277EEA57A30EE670AC0ED087AA6EE22
:107CC000007AC0ED077A80ED0A7A80ED097A01D852
:107CD00003B030BD012B4BDD07EE904AF8EEE77A9A
:107CE00087EE270AB5EEC00AF1EE10FA43DBB5EED7
:107CF000400AF1EE10FA41D4F1EEC07AF4EE677A60
:107D0000F1EE10FA37D690ED057AB4EEE77AF1EE9F
:107D100010FA18D5037B23B30323037003B030BDDF
:107D20002B688168DFED1A7A80ED080A9A1A8A4278
:107D300080ED070AC0ED097ACAD9B0EE670ADBE721
:107D40002A68426098E7D0ED047AD0ED066AF8EE32
:107D5000677A022386EEA77A037080ED067A03B075
:107D600030BD29684160002203618261C362AFE7D0
:107D70009FED070AC0E7DFED067AC4E7019069F0DE
:107D800055FD0198F0EE407AB8E700BF4C2700207F
:107D90000000000070B52DED028B044682B000F1AA
:107DA000480503460026B1EC017AD3ED067ADA6A7B
:107DB00077EE877A0132012AC3ED067ADA626DD056
:107DC00093ED075A93ED096A07EE902A77EE455A2C
:107DD000F8EEE77AC5EEA76A76EE857AF0EE466AA7
:107DE00037EE677AC3ED087AE5EE876AC3ED077A66
:107DF000C3ED0A6AC3ED096A1833AB42D3D10369F4
:107E0000394E42680133036133689B1A826893429A
:107E100040D99FED368AE36A012B4DDD013B07EE29
:107E2000903A94ED0A7AF8EEE77A87EE270AB5EEF3
:107E3000C00AF1EE10FA4DDBB5EE400AF1EE10FA91
:107E40004BD4F1EEC07AF4EE677AF1EE10FA41D637
:107E500090ED057AB4EEE77AF1EE10FA24D41834F6
:107E6000AC42D8D1D0ED047AD0ED066A90ED0C7A10
:107E7000D0ED125AF8EE677A022386EEA76A0370F5
:107E8000C7EE276A85EEA77A80ED066AC0ED0C6A18
:107E900080ED127A02B0BDEC028B70BD83ED087AE2
:107EA00083ED077A5E62A7E7037B43B10323037088
:107EB00002B0BDEC028B70BDB0EE480AC1E70022F3
:107EC0003168416003618261C3620263436482641A
:107ED000C365DFE7F0EE487ABAE7019069F0A6FCE7
:107EE0000198F0EE407AAEE74C2700200000000039
:107EF000DFED0A7AC0ED020A20EE270AB7EE007A1B
:107F0000C7EE007A0023036030EEA77AC0ED017A55
:107F1000C0EE877AC0ED037A704700BFDB0FC9401F
:107F2000F0EEC07AB0EEE07AB4EEE77AF1EE10FA55
:107F3000D4BFB0EE676AB0EE476AB5EE406AF1EEC4
:107F400010FA48D0B4EEE77AF1EE10FA54BFF0EE32
:107F5000675AF0EE475AC5EE866ADFED202ADFED5C
:107F6000203ADFED204A9FED205A9FED203A9FED09
:107F7000204A9FED206AE6EEA23AA6EE834AE6EE9C
:107F8000A34AF7EE005AA6EEA45AE6EE845AA6EEED
:107F9000856AB1EE466AC6EE256AB4EEE77AF1EE7E
:107FA00010FA48BFDFED147AF5EEC00A48BF77EE4D
:107FB000E66AF1EE10FA48BFDFED107AB5EEC00ABE
:107FC00048BF77EEE66AF1EE10FA48BFF1EE666A56
:107FD000B0EE660A7047DFED0A6ADEE739094E3D0A
:107FE000E3B59EBE88FA16BE45FE7FBF99FB243FCF
:107FF00069A2163EA7DFA8B4DB0FC93FDB0F4940DB
:10800000A7DFA83491ED007AD0ED047AD0ED055ABF
:1080100090ED064AD0ED074A90ED085A90ED096AB6
:10802000D0ED0A6AE7EE077AF7EE003AC0ED047A7F
:1080300091ED007AD1ED017AE7EE275A90ED0B7AB7
:10804000C0ED055AD1ED025A91ED003AD0ED0C7A0F
:10805000A3EE254A80ED064AD1ED005A74EEA54AFA
:10806000C0ED074AD1ED014AD1ED005AA4EEA55A60
:1080700080ED085A91ED015AA5EE056A80ED096A76
:10808000D1ED015A91ED026AE5EE866AC0ED0A6A09
:10809000D1ED016A37EE267A80ED0B7AD1ED026AD6
:1080A00091ED007AE6EE877AC0ED0C7A91ED026AE6
:1080B000D1ED016AD0ED0D7A90ED0E7A90ED0F4A78
:1080C000D0ED104A90ED115AD0ED135AE6EE267A13
:1080D00075EEA35AC0ED0D7AD1ED026AD0ED127A99
:1080E00090ED006AA6EEA67AD0ED016A80ED0E7AD8
:1080F00091ED027A34EE074A90ED027A80ED0F4A54
:1081000091ED004A74EE844AC0ED104AD1ED014A67
:1081100035EE245A80ED115A91ED025AC0ED135AF2
:1081200077EE857AC0ED127AD1ED017AD1ED005A61
:1081300091ED025A67EEA77AE5EEA57AE5EE057AAB
:10814000A5EEA76A80ED006A91ED016AE6EE276A66
:10815000C0ED016AD1ED026AA6EEA77A80ED027A3F
:1081600090ED037A77EE277AC0ED037A704700BF6F
:108170002DE9F04F89B0CDE9011200F110098346D5
:1081800000F13008CE4607464E4605468446002498
:10819000CDF80C906246284684B1D2ED007A0146B3
:1081A0003B468946F3EC016A99ED007AE6EEC77A20
:1081B000634501F11001C2ED007AF2D1043272453B
:1081C00000F10400E8D1032C04F1010A30D062462A
:1081D0003046ABEB05099CB1D2ED047A009409EB73
:1081E000000329460C46F3EC016A94ED007AE6EEB2
:1081F000C77A834201F11001C2ED047AF2D1009CEA
:10820000D2ED046A16ED047AC6EE877A1032424542
:1082100000F11000C2ED007ADDD10CF1140C08F170
:108220000408043514360EF1100E10375446B1E729
:10823000DDE9022900250023013505930693079304
:10824000042D52F8043B049305A80BF1140418D034
:10825000F2EC017A04A9C0ED007A4B46B1EC017A48
:10826000F3EC016AE6EEC77AA342C0ED007AF5D1DD
:108270000135042D09F1100900F1040004F1140482
:10828000E6D1019A08AE76ED017A022510320BF1A3
:108290004004022D2046A2F1040142ED017A20D0D3
:1082A0002346F3EC016AB2EC017AE6EEC77A984213
:1082B000C1ED007AF5D154ED016A87EEA67A6B1C08
:1082C00081ED007A14D076ED017A013D0A46022D47
:1082D000A4F11404A0F11000A2F1040142ED017A0E
:1082E000DED154ED016A87EEA67A02ED017AEAE763
:1082F00009B0BDE8F08F00BF10B584B00C4602464F
:1083000069461030FFF734FFDDED007A9DED017A0C
:10831000DDED026AB6EE006A67EE867A27EE067A2F
:1083200066EE866AF4EE677AF1EE10FAC4ED007A32
:1083300084ED017AC4ED026A0DD6B4EE477AF1EE0F
:1083400010FA13D6F4EE666AF1EE10FA78BF012047
:1083500016D604B010BD9FED106AF0EEE77AF4EE89
:10836000467AF1EE10FAE8DD0020F2E7DFED0A7A56
:10837000B0EEC77AB4EE677AF1EE10FAE2DDF3E719
:10838000DFED057AF0EEE66AF4EE676AF1EE10FAD8
:10839000D4BF01200020DCE7FFFF7F7FDFED257ADF
:1083A000B4EEE70AF1EE10FA08DD9FED237A30EE25
:1083B000470AB4EEE70AF1EE10FAF8DCDFED1F7AB7
:1083C000B4EEE70AF1EE10FA08D59FED1B7A30EE15
:1083D000070AB4EEE70AF1EE10FAF8D4DFED187AE6
:1083E000B4EEE70AF1EE10FA18DD30EE670A37EE68
:1083F000C00A60EE007A9FED137A9FED136ADFEDFD
:10840000136AA7EE876A9FED127AE7EE866A60EE3E
:10841000275AA7EEA67AA5EE870A70479FED0D7A38
:10842000B4EEC70AF1EE10FA44BF30EE270A37EE79
:10843000400ADEE7DB0F4940DB0FC940DB0F49C0D4
:10844000DB0FC93F9A7C2E36FAAF4FB93587083C0F
:10845000A4AA2ABEDB0FC9BF10B53E4CB4FBF2F490
:10846000A1420DD300234FF07E520260436083602F
:10847000C36003610023836143610362C36110BD74
:1084800007EE902AB8EE677ADFED337A27EE277A87
:10849000B7EE006AC6EE076A07EE901A9FED2F7AD4
:1084A000F8EE677AB0EE405A67EE877AC7EEA64AD2
:1084B000FDEEE47A17EE902A2032402A47D8B0EE3B
:1084C000640AFFF76BFFB0EE404A9FED250A34EED9
:1084D000800AFDEEC07A17EE902A2032402A31D869
:1084E000FFF75CFFF8EE006A60EE266A012B24D0ED
:1084F000F7EE007A37EEC00AF6EE005A60EE255A23
:1085000035EE055AB7EE007A84EE056A76EE077A04
:1085100037EE467A80EE275A85EEA76AC6EEA75A4E
:10852000C7EE276A80ED006A80ED015A80ED026A8D
:10853000C0ED035AC0ED046A9CE7B0EE660AF7EEA0
:10854000005ADDE7DFED076A9FED070ACEE79FEDF2
:10855000064ABAE720A10700BD378635DB0FC940C0
:10856000DB0FC93F0000008000000000DFED077A4C
:1085700030EE270AFDEEC07A17EE903A2033402BFA
:1085800000D80BE79FED020A704700BFDB0FC93F21
:108590000000000091ED005A9FED520A35EE000AEE
:1085A00008B5FDEEC07A17EE903A2033402B7DD807
:1085B000FFF7F4FEFDEEC57AB0EE403A17EE903AC2
:1085C0002033402B7BD8B0EE450AFFF7E7FEB0EE34
:1085D000405AF1EE402A91ED014A9FED420A34EEF5
:1085E000000AFDEEC07A17EE903A2033402B74D883
:1085F000FFF7D4FEF0EE404AB1EE402AFDEEC47A19
:1086000017EE903A2033402B64D8B0EE440AFFF7BF
:10861000C5FEB0EE404AD1ED021A9FED320A31EEAE
:10862000800AFDEEC07A17EE903A2033402B4ED8E8
:10863000FFF7B4FEF0EE403AFDEEE17A17EE903A25
:108640002033402B40D8B0EE610AFFF7A7FE63EE5F
:10865000836A20EE037A63EE857A20EE055AF0EE07
:10866000475AB0EE666AE7EE845AA5EE446AE7EE32
:10867000047AA6EEC45A63EEA43A62EEA42A22EE6D
:10868000000A64EE834AC0ED003A80ED010A80EDF5
:10869000024AC0ED035A80ED046AC0ED052A80ED60
:1086A000065AC0ED077AC0ED084A08BDFDEEC57A4E
:1086B0009FED0D3A17EE903A2033402B83D9DFED32
:1086C0000B2A9FED095A86E79FED070ABFE7DFED0A
:1086D000063AB1E79FED044A9DE79FED042ADFEDDE
:1086E000024A8BE7DB0FC93F00000000000000805A
:1086F0002DE9F04F83B005469DF830400D9E019264
:10870000002C14BF4FF030094FF020091C1E884682
:108710004ADB16F8010B014600286CD0002C65D00E
:108720004FF0000A324601E0002C34D012F8013B31
:108730002746013C002BF7D1BAF1000F3CD1023F94
:10874000002C65D0BA4645450AF1FF3A494628460D
:1087500001D2019B9847BAF1FF3FF4D10D9A1078EE
:1087600023463C1B01469B4688B14FF0000A01336B
:108770009F1B454506EB070B284601D2019B9847F6
:1087800016F8011B0029F4D1BAF1000F18D1584690
:1087900003B0BDE8F08FBAF1000F31D00146834637
:1087A0000028F4D02346E2E716F8010B634258B3E1
:1087B0001C464FF0010AB5E7014683460028D6D192
:1087C000002C04F1FF36E2DD3446454506F1FF3664
:1087D0004946284601D2019B9847731CF5D10BF1FD
:1087E000010BA344584603B0BDE8F08F2346A246D0
:1087F0004FF0FF34BBE7671EA346002CA2D1C6E7AB
:1088000023464FF0FF34ADE7E64383463446DCE7CA
:1088100023463C46A6E700BF0FB430B583B006AB95
:108820000B4C53F8042BD4F8F01FD4F8EC0F019341
:1088300064F066FD0546206803685B699847002878
:10884000F9D0284603B0BDE8304004B0704700BFFF
:10885000205C00200EB410B583B005AB044653F87D
:10886000042B0749009301A8019464F049FD019B82
:1088700000221A7003B0BDE8104003B0704700BF7B
:10888000016D00080CB4F0B53C4CD4F8F43FADF5E4
:10889000277D002B4CD094F8FC3F994240D8384BB0
:1088A000384A1B68A2FB031292094FF47A7101FB4C
:1088B000123306A83449FFF7CDFF06AB0344334912
:1088C000AC9A01930646ADAB01A8009364F018FD85
:1088D000019BD4F8F45F0A210246581C01901970DC
:1088E000019B591C01910021197035B32B681B6A3B
:1088F0001BB128469847D4F8F45F9DF8181049B189
:108900000DF119042B6828461B68984714F8011BC1
:108910000029F7D10DF5277DBDE8F04002B0704782
:108920001B4A0123126803FA00F01042B7D1F1E7A5
:10893000D4F8F83F002BAED1ECE7D4F8F87F002F45
:10894000E8D0901926AB841CFD20CDE9045506A97A
:108950002246ADF8100018466BF066FC0222034672
:10896000044402A93846CDE9023435F0C9FA0DF5C0
:10897000277DBDE8F04002B0704700BF205C0020BA
:108980004C270020D34D621058250808F56C0008CC
:10899000206C002030B54FF4004087B033F0ECFC81
:1089A00058B14FF40041044633F010FD022806D1BF
:1089B000226848F201039A4224D007B030BD002358
:1089C0004FF46121022294F904008DE80E001A464A
:1089D0004FF4004133F004FD1C4BC3F8F40F0028A2
:1089E000EBD01B4A1B4B1C4C1C481D490091CDE988
:1089F0000332CDE901041B4B1B4A02210020FFF783
:108A000041FFDAE7194C00254FF4004084F8A051EB
:108A100062F03CFC0028D0D054F8F43C83420BD0E8
:108A200054F8183C83420CD0D4F8C43098420AD091
:108A3000064BC3F8F85FC0E7F43C044BC3F8F84FAB
:108A4000CFE7183CF9E7C434F7E700BF205C00200B
:108A50007C2508088825080894250808A02508080A
:108A6000642408087824080864250808186D002084
:108A700038B5184CD4F8A451033005EB9003B3F586
:108A8000007F18D804EB810120F00302D1F8A80977
:108A9000C4F8A4311044C3F5007304F5D474C1F8CC
:108AA000A8090D4A04EB85049B0004210020FFF770
:108AB000E9FE204638BD00210846084AFFF7E2FEDD
:108AC000074AD2F89C30002443F00073C2F89C306F
:108AD000204638BD186D0020A8250808CC250808B8
:108AE0000000001038B50568EB690446F3B19878CA
:108AF00000B938BDB3F90A2007EE902AF8EEE77AFC
:108B00000120C4ED057AB3F90C2007EE902AF8EEA7
:108B1000E77AF1EE677AC4ED047AB3F90E3007EE26
:108B2000903AF8EEE77AC4ED067A38BD09211420B0
:108B3000FFF79EFF0346E861D9E700BF38B5056837
:108B4000EB690446E3B1987800B938BDB3F9042065
:108B500007EE902AF8EEE77A0120C4ED047AB3F923
:108B6000062007EE902AF8EEE77AC4ED057AB3F90D
:108B7000083007EE903AF8EEE77AC4ED067A38BD91
:108B800009211420FFF774FF0346E861DBE700BF0B
:108B900038B50568EB690446E3B1987800B938BD8B
:108BA0009A88D2BA07EE902AF8EEE77A0120C4ED4F
:108BB000047ADA88D2BA07EE902AF8EEE77AC4EDA2
:108BC000057A1B89DBBA07EE903AF8EEE77AC4ED36
:108BD000067A38BD09211420FFF74AFF0346E861F1
:108BE000DBE700BF38B50468E3690D467BB19878D0
:108BF00000B938BD5B89094ADBBA82FB0312DB1777
:108C0000C3EB221303F26D132B80012038BD092121
:108C10001420FFF72DFF0346E061E8E779787878C4
:108C200070B50568E8690C461646A0B3D0F8013067
:108C3000CCB1D0F805209FED1B7ADFED1B5ADFED9C
:108C40001B6A07EE902AF8EE677AB7EE006A77EEB5
:108C5000C77A77EEA77A87EEA57A77EE467A67EE3F
:108C6000E67AC4ED007AAEB107EE903A9FED107A45
:108C7000DFED106A9FED106AF8EEE77A67EE877A0B
:108C800087EEA67ADFED0D6A77EE467A77EEA67A62
:108C9000C6ED007A70BD09211420FFF7E9FEE861F6
:108CA000C4E700BF9AC9CC449AC94C460E76D74552
:108CB0000000484300E0FF440000484233938843EB
:108CC0002DE9F041944603EB43031CF8068B86B074
:108CD000144602EB430315464FFA88F69CF80070E1
:108CE000A0EB070E821BBEF1000FB8BFCEF1000E45
:108CF000002AB8BF52429645B8BF65460CF1060C33
:108D0000B8BF7EB26345E9D1B0456F88A3F10602D2
:108D100006D0BE46A24216D014F8068FB045F8D150
:108D2000B4F80280CB1BA1EB080C002BB8BF5B4250
:108D3000BCF1000FB8BFCCF1000C6345BE46E9DDC5
:108D400047462546E5E76B7904932B7903932B7807
:108D5000064A0091CDE9013E032103460120FFF7B9
:108D600091FD284606B0BDE8F08100BFDC2508086B
:108D700003681A46591C016012F8021B02605878F9
:108D800041EA0020704700BF02681146531C03608F
:108D900011F802CB0160D31C5178036093781B0457
:108DA00043EA0123111D0160D07843EA0C0343EA32
:108DB0000060704712B370B50446864604E0981B05
:108DC00017D114EB0C0C15D01EF8013BA3F1410098
:108DD000192811F8010BA0F1410598BF2033192D76
:108DE000A2EB0E0C00F12006E9D91B1A04D10028D1
:108DF000E7D170BD604670BD184670BD1046704723
:108E000010B40288C378174CA2F5FA6202F003018D
:108E100040F2B55C9208013B0CFB0233827801EB17
:108E20004101013A02EB810204EB420102798C8E8E
:108E30004179234403EB430302EBC30384790A4AD9
:108E40000089C3EB031301EB8303C3EB0313224439
:108E500002EB830200214FF47A73C2FB03015DF839
:108E6000044B7047B086070880436D382DE9F04108
:108E700017461E4605464FF47A720023384631469F
:108E800067F048FD4349444A014482FB0143C81747
:108E90000B44C0EB631382FB03021A44D8173F4C08
:108EA000C0EB621284FB02044FEAE27C3C48CCEB4C
:108EB000A40C80FB0C404FEAEC74C4EBE010C3EB55
:108EC0000314A1EB8401A971C2EB0211A3EB81038E
:108ED0006B710CEB4C03A2EBC30240F2B55303FBE6
:108EE00010CCBCF5896F2A714FEA800044DA40F259
:108EF000DA239C4547DCBCF5B77FB4BF00220122D2
:108F0000284B02EB420103EBC1034FEA4208B3F8DE
:108F10004A3091B2244C08EB020E04EBCE04163416
:108F20004FF00B0E01E034F8023D63451FDDBEF14A
:108F3000010EF8D11B4B424403EBC2024FF0010E6D
:108F4000938E85F802E000F5FA600CF1010C0844FC
:108F5000ACEB030C288085F803C04FF47A72002331
:108F60003846314667F0D6FC2A81BDE8F0810EF123
:108F7000010E5FFA8EFEE4E7032140F296530A46A3
:108F80004FF00608C6E7022140F229430A464FF097
:108F90000408BFE780BC92C789888888ABAAAA2A40
:108FA00073B06D16B0860708E486070830B52E4DFD
:108FB00084468E460FCD8DB06C460FC40FCD0FC4C6
:108FC00095E80F001CF0030F84E80F000DD1274B2C
:108FD000274A03FB0CF3B2EBB30F43D3254AB2EBA2
:108FE000331F2CBF1D241C2400E01C240CF1FF3374
:108FF000002B40F26D12194602FB0CF2B8BF0CF1C7
:10900000020102EBA1021C491C4D019481FB0301EA
:10901000DB17A3EB61100244C3EBE1131A442532C2
:1090200085FB02301044D317C3EBA000C0EBC00097
:10903000ADF10403101A0DF1040C03EB8E0E01E0E8
:109040005CF8044F031985FB0320C218D817C0EB46
:10905000A200C0EBC000E645A3EB0000F0D1201A4F
:109060000DB030BD1D24C1E744870708295C8FC2BD
:10907000285C8F020AD7A3001F85EB5193244992E5
:1090800008B50D4BD3F8302AD3F8343A52EA030C22
:1090900009D1002340F20112428083808371038052
:1090A0000381184608BD054909688A1843F1000381
:1090B000FFF7DCFE012008BD186D00204C270020C2
:1090C00030B5144DD5F8302AD5F8343A52EA0301B8
:1090D00083B0044609D1002040F201132080638050
:1090E000A080A071208103B030BD0B4909688A18A7
:1090F00043F10003FFF7BAFEB5F8383AADF8063091
:1091000020460DF10602214663F0BEFB012003B0AC
:1091100030BD00BF186D00204C27002088422DE98B
:10912000F0414FF001043DD301FB04F4B0FBF4FC2B
:109130008C45F9D23CB3002616E0BCF1090F274656
:1091400098462C4623DD002A14BF4FF0370E4FF00F
:10915000570EF444B94288F800C003F1010306F148
:10916000010610D8B0FBF5FCB4FBF1F504FB1C00C4
:10917000002EE2D1BCF1000FDFDCA1420AD90CF1D4
:10918000300C03F801CB00221A70BDE8F0814FF0DB
:10919000300EDEE7B0FBF5FC2C4605FB1C00B5FBF2
:1091A000F1F5E7E78446C6E790422DE9F0410B462A
:1091B000044615460AD2B0FBF5F6134A05FB1644E1
:1091C0001846135D00F8013BBDE8F081B0FBF2F6F4
:1091D0009642B6FBF2F706D20B4A05FB1767D15D44
:1091E00003F8011BEAE7BA42B7FBF2F807D9064ACF
:1091F00005FB187812F8081003F8011BEDE740464C
:10920000FFF7D2FF0346F2E718260808B5EEC00ABA
:10921000DFED347AF1EE10FACCBF30EE270A30EEF3
:10922000670ADFED317A20EE270A70B5FDEEC07ACD
:1092300086B017EE904A054684EAE470002303A93D
:10924000A0EBE470CDE90033029363F013FF002C30
:10925000ACBF20232D2303A88DF8003066F092FCCC
:1092600001286E4628D0022832D003281CD003A93A
:1092700030466EF0C7F8304666F084FC0338C4B25E
:109280002246314628466AF0CFFF00232B55284658
:1092900066F078FC2E232B540130311928446EF0EF
:1092A000CDF8284606B070BD302303A930468DF8AE
:1092B00001306EF0A7F8DEE7302303A930468DF8C1
:1092C00001308DF802308DF803306EF09BF8D2E754
:1092D000302303A930468DF801308DF802306EF04E
:1092E00091F8C8E76F12033A00007A440278202A06
:1092F000034600F10100F9D0092AF7D02D2A29D020
:109300002B2A03BF5A78B7EE000A0346B7EE000ACD
:10931000A2F13001C8B20928DFED4C7A10D8F2EE84
:10932000046A07EE101AB8EEC77A13F8012FA7EEF9
:10933000A67AA2F13001C8B20928F0EE477AF0D936
:109340002E2A49D0197801F0DF01452907D020EEF7
:10935000270A70475A78BFEE000A0346D8E710B4D0
:1093600059782D2962D02B2954D0A1F13002092A35
:1093700003F1010355D80024002202EB820201EB25
:10938000420213F8011FA1F130000928A2F13002B6
:10939000F3D9B2F59A7F134628BF4FF49A73072A80
:1093A00050D9DFED2B6A1A46B7EE007A083A072A41
:1093B00027EE267AFAD803F007032BB1F2EE046AFF
:1093C000013B27EE267AFBD16CB3C7EE877A5DF8B6
:1093D000044B20EE270A70475978A1F13002D0B231
:1093E000092803F10103AED8F2EE046AF0EE665AE2
:1093F00007EE102AB8EEC77A13F8011F87EE266A27
:10940000A1F13002D0B2092866EEA56A77EE867A1D
:10941000EED998E79978A1F13002092A03F1020305
:10942000A9D9B7EE007A67EE877AD0E79978A1F1EB
:109430003002092A03F1020388BFB7EE007AC4D8CC
:10944000012499E7B7EE007AB7E700BF00000000FB
:1094500020BCBE4C00B50378202B014600F1010072
:10946000F9D0092BF7D02D2B03BF4B784FF0FF3EDF
:1094700001464FF0010E0022A3F1300C5FFA8CF38D
:10948000092B03D90EFB02F05DF804FB02EB82020C
:1094900011F8013F0CEB4202EEE700BFF0B5384D8A
:1094A0002B78082141F221008B4002E0013993B270
:1094B00009D013F4004F4FEA4302F7D080EA430388
:1094C00001399BB2F5D1B5F80120002A55D0DFF85B
:1094D000C0C02C4EB4452DD2ACF1060C0CEB0204EE
:1094E000B44227D2052A41F2210022D9A44514D042
:1094F0000CF1FF3C04F1FF3E1CF8011F082283EA37
:10950000012313F4004F80EA43010ABF5B008BB2D2
:109510009BB2013AF5D1E645EED1228862B1A11D98
:10952000B14206D2A118B142A44602D2052A0C4685
:10953000DCD800210846F0BDA71C264641F22100D8
:1095400016F8011B082283EA012313F4004F80EA76
:1095500043010ABF5B008BB29BB2013AF5D1B7421F
:10956000EED16188084AC91AB1FA81F1231D49096F
:109570005B1BA2F83C3A0846F0BD044FBC1EDCE77A
:1095800000000E0800001008186D002003000E08EF
:1095900007000E082DE9F04F9B4B9C4A8FB09A1A9A
:1095A000CDE9013203230393984B0793029B099360
:1095B000019B08930023CDE90A33CDE90C33944A8B
:1095C0001369002BC0F2A181914B9249F322DA601A
:1095D00000220C92019A01238A428DF83430C0F0A7
:1095E0008C810B937E238DF8283008224FF4FC43A6
:1095F00041F2210103E05B00013A9BB206D018045E
:10960000F9D581EA4303013A9BB2F8D1824AADF819
:109610001230824B934280F08E8103F1140801993D
:109620007A4B41F2210538F8120C38F8142CC0F3AB
:109630000B06B41DADF81440C2F30B04120B8DF8E9
:10964000182000270204ADF816408DF819705DD47B
:1096500006338B4200F251810DF114090DF11A0A03
:109660004C4601E0A24513D00B9B14F8011B03F1FB
:1096700038026A440133042B02F8101C0B93F1D119
:109680000AA907A8F9F78CFAA245CDE90B70EBD12E
:109690000C9B002BC0F23181BDF8124019F8013B40
:1096A00084EA0324082327044CBF85EA44046400A9
:1096B000013BA4B2F7D1CA45F0D158F8101C32468C
:1096C00007A8FDF79BFE0028C0F2178158F8102C60
:1096D00091198A4210D0013A013912F8013F84EA07
:1096E0000324082320044CBF85EA44046400013BA2
:1096F000A4B2F7D19142F0D1474BADF81240984552
:1097000074D2DDE9073108F114088CE7B946CDF8C9
:10971000008009F1010906335FFA89F98B428DF85F
:10972000199000F2EA800DF1140A0DF11A0BD046DF
:10973000002401E0C34513D00B9B18F8011B03F173
:1097400038026A440133042B02F8101C0B93F1D148
:109750000AA907A8F9F724FAC345CDE90B40EBD1D4
:109760000C9B002BC0F2C980BDF812401AF8013BD7
:1097700084EA0324082322044CBF85EA44046400DD
:10978000013BA4B2F7D1D345F0D1009B53F8102C84
:1097900002EB070A5146324607A8FDF72FFE0028C4
:1097A000C0F2AB800AEB06018A4511D00AF1FF3204
:1097B000013912F8013F84EA0324082320044CBF36
:1097C00085EA44046400013BA4B2F7D18A42F0D197
:1097D000B9F1030FADF81240374402D0DDE907318B
:1097E00097E7DDF800800C4B98458AD3DDE9073117
:1097F000023300229942ADF814207ED30DF11504F6
:109800000DF1160516460FE00000100800000E08C6
:10981000003C024001000E08A0A10808A09C080816
:10982000A54213D014F8012B0B9B03F138016944B6
:109830000133042B01F8102C0B93F1D10AA907A8CE
:10984000F9F7AEF9A542CDE90B60EBD10C9B002BEB
:1098500053DBBDF81230082241F221011C0454BF31
:109860005B0081EA4303013A9BB2F7D1082241F23F
:10987000210118044CBF81EA43035B00013A9BB20B
:10988000F7D1ADF81230079B089902338B4234D8D8
:1098900014460DF1120505AE01E0B54213D00B9B45
:1098A00015F8011B03F138026A440133042B02F856
:1098B000101C0B93F1D10AA907A8F9F771F9B54269
:1098C000CDE90B40EBD10C98002816DB0B9B13B3B2
:1098D000079A08991A448A420FD80AA9C818C3F1EE
:1098E000040200216CF03EFE0AA907A8F9F758F916
:1098F000002398420C900B930DDA039B013B0393DA
:109900007FF452AE052007F09BF80F4B536003F134
:109910008833536058E69DF834307BB90028ECD189
:109920000A4B1B787E2BEDD1FFF7B8FD0028E9D05C
:109930000FB0BDE8F08F0199044B59E7044A136951
:1099400043F000431361E9E72301674500000E0877
:10995000003C024070B545880B460446C5F30B0534
:109960002A46002118466CF0FDFD2169084A914203
:10997000034602D3074A914205D319B1BDE87040AE
:109980001846084770BD2A46BDE870406AF04CBCD6
:10999000A0A1080847A6080810B50379012B84B0D8
:1099A0008E460ED0022B09D18368DB0758BF01F029
:1099B0007F0104B0BDE81040FDF74ABD002004B0AF
:1099C00010BD144682688DF80F4002F0010201922A
:1099D0000DF10F020092417C90F910007246FAF7E7
:1099E0009DFE04B010BD00BFF8B5782204460021EA
:1099F0000068FFF7D1FF052706F0C6FF05460E46B3
:109A000006F0C2FF431B61EB0602B3F57A7F72F1E9
:109A10000003F5D3013FEFD1206820220121FFF799
:109A2000BBFF052706F0B0FF05460E4606F0ACFF6B
:109A3000431B61EB0602B3F57A7F72F10003F5D3A5
:109A4000013FEFD120683A460221FFF7A5FF6426C7
:109A500006F09AFF04460D4606F096FF031B61EBE5
:109A60000502B3F57A7F72F10003F5D3013EEFD121
:109A70000120F8BDF8B5072204460A210068FFF767
:109A80008BFF052706F080FF05460E4606F07CFF9B
:109A9000431B61EB0602B3F57A7F72F10003F5D345
:109AA000013FEFD1206824224121FFF775FF0527F0
:109AB00006F06AFF05460E4606F066FF431B61EBA3
:109AC0000602B3F57A7F72F10003F5D3013FEFD1BF
:109AD0002068C0224221FFF75FFF052606F054FFF1
:109AE00004460D4606F050FF031B61EB0502B3F57B
:109AF0007A7F72F10003F5D3013EEFD10120F8BD6A
:109B000010B50446002221210068FFF745FF2068B8
:109B1000FC222021FFF740FF206840222421FFF78C
:109B20003BFF20680C222321FFF736FF206800222C
:109B30002221FFF731FF012010BD00BFF8B501223F
:109B4000074610210068FFF727FF00B9F8BD14266B
:109B500006F01AFF04460D4606F016FF031B61EBE4
:109B60000502B3F57A7F72F10003F5D3013EEFD120
:109B70003868A022BDE8F84011210DE730B505682E
:109B80002B79012B85B0044611D0022B0CD1012278
:109B90000B212846FDF75CFC30B120681D2209210D
:109BA00005B0BDE83040F7E6002005B030BDAA683A
:109BB00095F91000697C8DF80F3002F001020192D6
:109BC0000DF10F0200920B22FAF7A8FDE4E700BFA7
:109BD00010B50446C06900B110BD09211420FEF77C
:109BE00047FFE06110BD00BF184B03EB80004068E9
:109BF00048B310B5164C00EB400004EB800393F91A
:109C000041CABCF1FF3F1FD093F8490AD0B104EB21
:109C10000C0293F8480A92F894EA8C23142103FB6F
:109C20000CFC00220CEB000304EB43030139B3F8F6
:109C3000983A704412FA83F2F4D10648A0FB02303D
:109C4000C0F30F1010BD7047002010BD205C002035
:109C5000186D0020CDCCCCCC30B5032083B00D46A0
:109C60001446FFF7C1FF01909DB107EE900A9FEDEA
:109C70000B7AF8EE677AF0EE006A67EE877AB8EE54
:109C8000047AA7EEA67ADFED067A67EE277AC5EDAD
:109C9000007A0CB1034B236003B030BD6740533AE8
:109CA00000007A443313904328B30368124A30B556
:109CB00003F13F4303F57E039B0A054683B00C4640
:109CC000D05C63F06FF9A988009104F00303C4F33A
:109CD00081028DF8043028688DF80520C4F3001344
:109CE0006946C4F341148DF806308DF80740F9F742
:109CF0003FFE03B030BD70478486070870B5114B36
:109D0000114CA34203D319E00C33A34216D293F8AB
:109D100005C08C45F8D193F804C0844501D00028D3
:109D2000F2D193F807E09645EED11D6895F804E06E
:109D3000E645E9D12E689E42E6D100E0002528469E
:109D400070BD00BF48A60808F8A708080379022BD1
:109D500000D0704710B590F91020204882B008312B
:109D6000694403244FF0000C02EB82024FF0010E15
:109D70008DF800C08DF801E08DF802308DF80340B9
:109D800050F8222011F8084C15498A4222D0A1F53A
:109D900078418A4220D001F580618A4218D1118829
:109DA00021F04001090403EB8303090C118000EB4F
:109DB00083001388C16823F0380331F824101B0492
:109DC0001B0C0B43138013889BB243F0400313809A
:109DD00002B010BD6346E2E77346E0E7600D002085
:109DE00000300140F8B5074600210068FFF7AEFFDC
:109DF0003868B6221421FFF7CFFD642606F0C4FDB3
:109E000004460D4606F0C0FD031B61EB0502B3F5E9
:109E10007A7F72F10003F5D3013EEFD18122102148
:109E20003868FFF7B9FD06F0AFFD04460D4606F0B1
:109E3000ABFD031B61EB0502B3F57A7F72F1000302
:109E4000F5D3802215213868FFF7A6FD06F09CFDAA
:109E500004460D4606F098FD031B61EB0502B3F5C1
:109E60007A7F72F10003F5D338680321BDE8F8402A
:109E70006CE700BFF8B5044600210068FFF766FFF5
:109E80002068B6227E21FFF787FD642706F07CFD5F
:109E900005460E4606F078FD431B61EB0602B3F55E
:109EA0007A7F72F10003F5D3013FEFD13A46206883
:109EB0007C21FFF771FD642706F066FD05460E461E
:109EC00006F062FD431B61EB0602B3F57A7F72F187
:109ED0000003F5D3013FEFD1206804227D21FFF775
:109EE0005BFD642706F050FD05460E4606F04CFD6E
:109EF000431B61EB0602B3F57A7F72F10003F5D3E1
:109F0000013FEFD18C2240212068FFF745FD06F08C
:109F10003BFD05460E4606F037FD431B61EB06028E
:109F2000B3F57A7F72F10003F5D302224121206854
:109F3000FFF732FD06F028FD05460E4606F024FD2B
:109F4000431B61EB0602B3F57A7F72F10003F5D390
:109F500020680221FFF7FAFE4FF40063A381F8BDE9
:109F60002DE9F041046884B00546B6227E212046E2
:109F7000FFF712FD4FF0640806F006FD06460F4697
:109F800006F002FD831B61EB0701B3F57A7F71F1E7
:109F90000003F5D3B8F10108EED102212046FFF706
:109FA000D5FE636913B11A689B88538306F0ECFCF5
:109FB00006460F4606F0E8FC831B61EB0702B3F58B
:109FC0007A7F72F10003F5D3636913B11A689B8835
:109FD00013834FF00A0806F0D7FC06460F4606F03A
:109FE000D3FC831B61EB0701B3F57A7F71F10003AA
:109FF000F5D3B8F10108EED142467C212046FFF7A7
:10A00000CBFC06F0C1FC06460F4606F0BDFC831BE8
:10A0100061EB0702B3F57A7F72F10003F5D30022FA
:10A0200059212046FFF7B8FC06F0AEFC06460F4665
:10A0300006F0AAFC831B61EB0702B3F57A7F72F18D
:10A040000003F5D394F91030A2688D4903EB830324
:10A050005E2092078DF80F0051F8230040F1E48054
:10A0600001230DF10F020021019065F03FFC4FF438
:10A07000A473844A0198002165F038FCA3689B070B
:10A0800040F1E5804FF00A0806F07EFC06460F46D8
:10A0900006F07AFC831B61EB0701B3F57A7F71F15F
:10A0A0000003F5D3B8F10108EED101225921204671
:10A0B000FFF772FC06F068FC06460F4606F064FCEB
:10A0C000831B61EB0702B3F57A7F72F10003F5D3CE
:10A0D0008C2240212046FFF75FFC06F055FC064627
:10A0E0000F4606F051FC831B61EB0702B3F57A7F44
:10A0F00072F10003F5D3032241212046FFF74CFC07
:10A1000006F042FC06460F4606F03EFC831B61EB60
:10A110000702B3F57A7F72F10003F5D3AA6B5A4EAA
:10A1200095F83500B6FBF2F2092391B2574AFEF7D3
:10A13000C7FD4388B6FBF3F62E640279422142F054
:10A14000C0022046FFF728FC06F01EFC05460E461E
:10A1500006F01AFC431B61EB0602B3F57A7F72F13D
:10A160000003F5D3082243212046FFF715FC06F033
:10A170000BFC05460E4606F007FC431B61EB06028E
:10A18000B3F57A7F72F10003F5D3042258212046FB
:10A19000FFF702FC06F0F8FB05460E4606F0F4FB5E
:10A1A000431B61EB0602B3F57A7F72F10003F5D32E
:10A1B0000A2253212046FFF7EFFB06F0E5FB054698
:10A1C0000E4606F0E1FB431B61EB0602B3F57A7F16
:10A1D00072F10003F5D300227C212046FFF7DCFB5F
:10A1E00006F0D2FB05460E4606F0CEFB431B61EBA4
:10A1F0000602B3F57A7F72F10003F5D306227D21C2
:10A200002046FFF7C9FB06F0BFFB04460D4606F0EB
:10A21000BBFB031B61EB0502B3F57A7F72F1000310
:10A22000F5D304B0BDE8F081636913B11A689B8867
:10A230005383174B17491A68174B4E68D200A3FB7C
:10A24000023292094B689B1B9A42FBD208E7104BE3
:10A2500010491A68104B48684FF4FA7606FB02F270
:10A26000A3FB023292094B681B1A9A42FBD2636924
:10A27000002B3FF407AF1A689B88138302E700BFE7
:10A28000600D00207487070840420F00BC88070853
:10A29000CC330020001000E0D34D62102DE9F041D6
:10A2A000604A0468816B604FB7FBF1F106461023EA
:10A2B00089B290F83500FEF703FD00214388B7FB13
:10A2C000F3F7054637642046FFF740FD80226B21F7
:10A2D0002046FFF761FB4FF0640806F055FB064689
:10A2E0000F4606F051FB831B61EB0701B3F57A7F44
:10A2F00071F10003F5D3B8F10108EED10322682112
:10A300002046FFF749FB4FF0640806F03DFB064688
:10A310000F4606F039FB831B61EB0701B3F57A7F2B
:10A3200071F10003F5D3B8F10108EED101226B21E0
:10A330002046FFF731FB4FF00F0806F025FB0646DD
:10A340000F4606F021FB831B61EB0701B3F57A7F13
:10A3500071F10003F5D3B8F10108EED118221B21E9
:10A360002046FFF719FB4FF00F0806F00DFB0646DD
:10A370000F4606F009FB831B61EB0701B3F57A7FFB
:10A3800071F10003F5D3B8F10108EED118221C21B8
:10A390002046FFF701FB4FF00F0806F0F5FA0646DE
:10A3A0000F4606F0F1FA831B61EB0701B3F57A7FE4
:10A3B00071F10003F5D3B8F10108EED12A791A2121
:10A3C0002046FFF7E9FA4FF00F0806F0DDFA0646DF
:10A3D0000F4606F0D9FA831B61EB0701B3F57A7FCC
:10A3E00071F10003F5D3B8F10108EED16A791921B2
:10A3F0002046FFF7D1FA642706F0C6FA05460E4656
:10A4000006F0C2FA431B61EB0602B3F57A7F72F1E4
:10A410000003F5D3013FEFD120460321BDE8F04111
:10A4200094E400BFF488070840420F002DE9F04192
:10A430006C4A0468816B6C4FB7FBF1F10646102340
:10A4400089B290F83500FEF73BFC00214388B7FB4A
:10A45000F3F7054637642046FFF778FC80226B212E
:10A460002046FFF799FA4FF0640806F08DFA064689
:10A470000F4606F089FA831B61EB0701B3F57A7F7B
:10A4800071F10003F5D3B8F10108EED1072268217C
:10A490002046FFF781FA4FF0640806F075FA064689
:10A4A0000F4606F071FA831B61EB0701B3F57A7F63
:10A4B00071F10003F5D3B8F10108EED142466B21EA
:10A4C0002046FFF769FA4FF0640806F05DFA064689
:10A4D0000F4606F059FA831B61EB0701B3F57A7F4B
:10A4E00071F10003F5D3B8F10108EED101226B211F
:10A4F0002046FFF751FA4FF00F0806F045FA0646DE
:10A500000F4606F041FA831B61EB0701B3F57A7F32
:10A5100071F10003F5D3B8F10108EED118221B2127
:10A520002046FFF739FA4FF00F0806F02DFA0646DD
:10A530000F4606F029FA831B61EB0701B3F57A7F1A
:10A5400071F10003F5D3B8F10108EED118221C21F6
:10A550002046FFF721FA4FF00F0806F015FA0646DD
:10A560000F4606F011FA831B61EB0701B3F57A7F02
:10A5700071F10003F5D3B8F10108EED12A791A215F
:10A580002046FFF709FA4FF00F0806F0FDF90646DE
:10A590000F4606F0F9F9831B61EB0701B3F57A7FEB
:10A5A00071F10003F5D3B8F10108EED16A791921F0
:10A5B0002046FFF7F1F9642706F0E6F905460E4656
:10A5C00006F0E2F9431B61EB0602B3F57A7F72F104
:10A5D0000003F5D3013FEFD120460321BDE8F04150
:10A5E000FFF7B4BBF488070840420F001EE700BF26
:10A5F000F0B5044683B000680021FFF7A7FB0C22EA
:10A6000025212068FFF7C8F90A2226212068FFF7D4
:10A61000C3F9002263212068FFF7BEF92068812278
:10A620002721FFF7B9F9142706F0AEF905460E46C3
:10A6300006F0AAF9431B61EB0602B3F57A7F72F1CB
:10A640000003F5D3013FEFD10C2225212068FFF74D
:10A65000A3F90A2226212068FFF79EF90F22632121
:10A660002068FFF799F9206881222721FFF794F9E4
:10A670000A2706F089F905460E4606F085F9431BC0
:10A6800061EB0602B3F57A7F72F10003F5D3013F67
:10A69000EFD1032301AA1021204661F02BF90A27EC
:10A6A00006F072F905460E4606F06EF9431B61EBA3
:10A6B0000602B3F57A7F72F10003F5D3013FEFD1C3
:10A6C0009DF804009DF805109DF806202B4B803066
:10A6D00080318032A3F8E00DA3F8E21DA3F8E42D49
:10A6E00025210C222068FFF757F926210A2220682D
:10A6F000FFF752F93A4663212068FFF74DF92068C9
:10A7000081222721FFF748F90A2706F03DF905467F
:10A710000E4606F039F9431B61EB0602B3F57A7F6A
:10A7200072F10003F5D3013FEFD10DF103020123D4
:10A730000221204661F0DEF801230DF10302092118
:10A74000204661F0D7F820680C222521FFF724F974
:10A7500020680A222621FFF71FF9206812226321B0
:10A76000FFF71AF9812220682721FFF715F92068E1
:10A770000321FFF7EBFA012003B0F0BD186D0020B4
:10A78000F0B5054690F91000244C00EB800085B030
:10A7900054F82000AC68A40710D5CDE9022301903D
:10A7A00065F0F4F8DDE902230198002165F09EF8D8
:10A7B000AB689B0718D5012005B0F0BD6C6914B1DA
:10A7C0002668A4887483164C164E246877684FEA6E
:10A7D000C40E154CA4FB0E4E4FEA9E1E7468A4EBEB
:10A7E000070CE645FAD2D8E70D4B0E491A680E4B16
:10A7F0004FF4FA7000FB02F2A3FB023248689209A0
:10A800004B681B1A9A42FBD26B69002BD3D01A6893
:10A810009B881383012005B0F0BD00BF600D0020B0
:10A82000CC330020001000E0D34D621030B5057924
:10A83000012D83B08E460DD0022D08D18468E40727
:10A8400058BF41F0800103B0BDE8304098E70020D8
:10A8500003B030BD14468268009402F00102417CCE
:10A8600090F9100001927246F9F758FF03B030BD1D
:10A87000F0B50546164695F91020244802EB8202F1
:10A8800083B050F82200AA6892070FD5CDE90003E3
:10A8900065F07CF8019B00980022314665F026F8AF
:10A8A000AB689B0718D5012003B0F0BD6A6912B1EF
:10A8B000146892886283164A1468164A4FEAC40ED6
:10A8C000154C5768A4FB0E4E4FEA9E1E5468A4EB2D
:10A8D000070CE645FAD2D9E70D4B0E491A680E4B24
:10A8E0004FF4FA7000FB02F2A3FB023248689209AF
:10A8F0004B681B1A9A42FBD26B69002BD3D01A68A3
:10A900009B881383012003B0F0BD00BF600D0020C1
:10A91000CC330020001000E0D34D621030B5057933
:10A92000012D83B08E460DD0022D08D18468E40736
:10A9300058BF41F0800103B0BDE8304098E70020E7
:10A9400003B030BD14468268009402F00102417CDD
:10A9500090F9100001927246F9F7ACFE03B030BDD9
:10A960002DE9F043814A0568816B814CB4FBF1F11C
:10A9700085B00646102389B290F83500FEF7A0F99D
:10A9800000214388B4FBF3F4074634642846FFF7FC
:10A99000DDF980226B212846FEF7FEFF4FF0960975
:10A9A00005F0F2FF0446884605F0EEFF031B61EB5D
:10A9B0000801B3F57A7F71F10003F5D3B9F101090C
:10A9C000EED1032268212846FEF7E6FF4FF09609F4
:10A9D00005F0DAFF0446884605F0D6FF031B61EB5D
:10A9E0000801B3F57A7F71F10003F5D3B9F10109DC
:10A9F000EED103226B212846FEF7CEFF05F0C4FFFF
:10AA00000446884605F0C0FF031B61EB08010F2BCD
:10AA100071F10003F6D310226A212846FEF7BCFF2D
:10AA200005F0B2FF0446884605F0AEFF031B61EB5C
:10AA300008010F2B71F10003F6D300226C21284688
:10AA4000FEF7AAFF05F0A0FF0446884605F09CFF2C
:10AA5000031B61EB08010F2B71F10003F6D37A7928
:10AA600019212846FEF798FF05F08EFF0446884618
:10AA700005F08AFF031B61EB08010F2B71F1000346
:10AA8000F6D318221B212846FEF786FF05F07CFF2F
:10AA90000446884605F078FF031B61EB08010F2B85
:10AAA00071F10003F6D318221C212846FEF774FF2B
:10AAB00005F06AFF0446884605F066FF031B61EB5C
:10AAC00008010F2B71F10003F6D33A791A212846B9
:10AAD000FEF762FF05F058FF07460C4605F054FFED
:10AAE0008C4208BF8742F9D003212846FFF72EF990
:10AAF0003068062302AA4321FFF710FF28B3BDF8F0
:10AB00000810BDF80A30BDF80C20C9BA07EE901A3B
:10AB1000DBBAD2BAF8EEE76A07EE102A07EE903AEF
:10AB2000B8EEC77AF8EEE77AC6ED076AC6ED087A9E
:10AB300086ED097AFDEEE77ACDED017A9DF90430D4
:10AB4000013305D005B0BDE8F083D6ED087AF1E712
:10AB5000D6ED077AFDEEE77ACDED017A9DF9043066
:10AB60000133EFD1062005F06BFF00BFF488070822
:10AB700040420F0010B504460068037982B0022BF2
:10AB80000CBF4321032106236A46FFF7C7FE68B1C5
:10AB9000BDF80010BDF80220BDF8043049BA52BA21
:10ABA0005BBAE1866287238702B010BDE086A063AE
:10ABB00002B010BD2DE9F047154D95F8E93D074667
:10ABC0008A4663B90021386895F8EA3D85F8E91DA1
:10ABD00052464921FFF7A2FE0120BDE8F08705F0AB
:10ABE000D3FED5F8F04D001BC0F5FA54002CE9DD7A
:10ABF00005F0CAFE4FEAE4790646884605F0C4FE31
:10AC0000831B61EB0801A34271EB0903F6D3D9E77B
:10AC1000186D0020F0B5614C0546D4F8F80DC5F864
:10AC2000360094F8E83DB4F8FC2D6A87012B83B018
:10AC30000AD0022B2ED003B3002384F8E83D84F819
:10AC4000FE3D184603B0F0BD94F8E93D002B41D11C
:10AC500069462846FFF7AEFF002851D09DF8003026
:10AC600099074DD007220321284662F03FFD0222BA
:10AC700094F8FE3D84F8E82DE3E7284601220221FE
:10AC800062F034FD94F8FE3D0122184684F8E82D68
:10AC900003B0F0BD94F8E93D05F1360704F6F85627
:10ACA00023BB69462846FFF785FF9DF8062003462B
:10ACB0000028C1D01207BFD4B4F8E01DBDF80020B1
:10ACC00012FB01F236498A4222DBB2F5000F5EDB4D
:10ACD000344A1EE005F058FED4F8F03DC01AC0F525
:10ACE000FA500028B4DD94F8FE3DAAE705F04CFECA
:10ACF000D4F8F03DC01AC0F5FA500028D1DDF2E7D3
:10AD000094F8FE3D0022184684F8E82D03B0F0BD0B
:10AD1000254AB4F8E21DEA86BDF8022012FB01F2D2
:10AD20001F498A4205DBB2F5000F2ADB47F6FF72A6
:10AD300000E01D4AB4F8E41D2A87BDF8042012FB88
:10AD400001F217498A4204DBB2F5000F12DB154A03
:10AD500000E0154AD5F83600C4F8F80D6A87BA88BD
:10AD6000B28000210122184684F8E81D84F8FE2DE7
:10AD700003B0F0BD002AB8BFFF321212524212B225
:10AD8000E8E7002AB8BFFF3242F30F22D2E7002AD9
:10AD9000B8BFFF321212524212B2BAE7186D002049
:10ADA00001FF7FFF0180FFFF0080FFFFF0B5066815
:10ADB000F56983B00446002D65D000232B70042371
:10ADC0000DEB03023046FF21FFF7A8FD10B900206C
:10ADD00003B0F0BD206804236A46FF21FFF79EFD03
:10ADE0000028F4D09DF804108A09023A012AEED90D
:10ADF0009DF8053003EB012343F6FF74C3F30D0305
:10AE0000A342E4D0002BE2D09DF806109DF8072065
:10AE100002EB012240F2FF71B1EB521F4FEA6216C2
:10AE2000D5D0002ED3D09DF800C09DF8012002EBB4
:10AE30000C22C2F30D02A242C9D0002AC7D09DF84D
:10AE400002709DF8034004EB0724B1EB541F4FEA56
:10AE50006417BCD0002FBAD0991A0029B8BF494254
:10AE6000FF29B4DCF11B0029B8BF4942FF29AEDC41
:10AE700013445B10F2195210C5F805300123C5F8D0
:10AE800001202B70A4E709211420FDF7F1FDF061EA
:10AE90000546266891E700BF70B50668F46982B080
:10AEA0000CB30025042325700DEB03023046FF216F
:10AEB000FFF734FDA8B19DF804108B091CD19DF853
:10AEC00005209DF806509DF8073002EB012292B252
:10AED00003EB0523C4F805205B1101222270C4F89E
:10AEE000013002B070BD054609211420FDF7C0FDF8
:10AEF000F06104462E68D4E7034A04210320FDF7DD
:10AF0000C1FC284602B070BD4026080810B50446B2
:10AF100000680179012984B028D0022923D18368EF
:10AF200013F0010F08BF8221062302AAFFF7A0FC3D
:10AF3000B8B1BDF9083006EE903ABDF90A3007EE17
:10AF4000103ABDF90C3007EE903AF8EEE66AB8EE2A
:10AF5000C77AF8EEE77AC4ED076A84ED087AC4EDA3
:10AF6000097A04B010BD002004B010BD8368417C94
:10AF700090F9100003F00103019302AB0093022249
:10AF80000623F9F797FB0028D3D1EAE730B504464A
:10AF900000680379012B85B014D0022B0FD1826891
:10AFA00002AD12F0010F18BF03212A4608BF83210A
:10AFB000FFF75EFC18B19DF90930002B10DB002073
:10AFC00005B030BD8368417C90F9100003F00103A7
:10AFD00002AD0193009502230322F9F76BFBE9E729
:10AFE000206807232A461221FFF798FC0028E6D0A4
:10AFF0009DF90A209DF809309DF90C1043EA0223BF
:10B0000013EB430248BF03329DF80B30921043EA22
:10B01000012307EE902A13EB4302F8EEE77A48BFCC
:10B0200003329DF90E109DF80D30C4ED047A921094
:10B0300007EE902A43EA012313EB4303F8EEE77A85
:10B0400048BF03339B10C4ED057A07EE903AF8EE43
:10B05000E77AC4ED067AB3E770B50668F46982B0A2
:10B060000546002C3FD03379012B04F1040205D0B2
:10B07000022B2CD00020A07002B070BDB368717C90
:10B0800096F91000009203F0010301930C231A4675
:10B09000F9F710FBA0700028EED0B4F9043007EEE9
:10B0A000903AF8EEE77AC5ED077AB4F9063007EE84
:10B0B000903AF8EEE77AC5ED087AB4F9083007EE71
:10B0C000903AF8EEE77AC5ED097A02B070BDB36840
:10B0D00013F0010F4FF00C03304614BF19468C21BA
:10B0E000FFF7C6FBD6E709211420FDF7C1FCF0618C
:10B0F00004462E68B7E700BF70B50668F46982B0F1
:10B100000546002C3FD03379012B04F1030205D012
:10B11000022B2CD00020A07002B070BDB368717CEF
:10B1200096F91000009203F0010301930C220D2305
:10B13000F9F7C0FAA0700028EED0B4F90A3007EE93
:10B14000903AF8EEE77AC5ED077AB4F90C3007EEDD
:10B15000903AF8EEE77AC5ED087AB4F90E3007EECA
:10B16000903AF8EEE77AC5ED097A02B070BDB3689F
:10B1700013F0010F30464FF00D0314BF0C218C214A
:10B18000FFF776FBD6E709211420FDF771FCF0618B
:10B1900004462E68B7E700BF10B500680379012B9D
:10B1A00084B00C4618D0022B13D1836813F0010F22
:10B1B00014BF2221A221032303AAFFF759FB30B1B8
:10B1C000BDF90D3003EB83031B12E633238004B07B
:10B1D00010BD002004B010BD8368417C90F91000C0
:10B1E00003F00103019303AB009322220323F9F739
:10B1F00061FA0028E4D1EAE710B504460068037953
:10B20000012B84B02DD0022B28D1836813F0010FBD
:10B2100002AA4FF0060314BF1F219F21FFF728FB4E
:10B22000D0B1BDF80810BDF80A20BDF80C30C9BA7D
:10B2300007EE901AD2BAF8EEE76A07EE902ADBBA68
:10B24000B8EEE77A07EE903AF8EEE77AC4ED046AD2
:10B2500084ED057AC4ED067A04B010BD002004B078
:10B2600010BD8368417C90F9100003F00103019345
:10B2700002AB00931F220623F9F71CFAD0E700BFA8
:10B2800010B5044600680379012B84B02DD0022B41
:10B2900028D1836813F0010F02AA4FF0060314BFF0
:10B2A0002521A521FFF7E4FAD0B1BDF80810BDF8BB
:10B2B0000A20BDF80C30C9BA07EE901AD2BAF8EEDF
:10B2C000E76A07EE902ADBBAB8EEE77A07EE903A23
:10B2D000F8EEE77AC4ED076A84ED087AC4ED097ADE
:10B2E00004B010BD002004B010BD8368417C90F90B
:10B2F000100003F00103019302AB00932522062303
:10B30000F9F7D8F9D0E700BF70B50668F46982B0E4
:10B310000546002C3FD03379012B04F1040205D0FF
:10B32000022B2CD00020A07002B070BDB368717CDD
:10B3300096F91000009203F0010301933B220E23C3
:10B34000F9F7B8F9A0700028EED0A389DBBA07EEB0
:10B35000903AF8EEE77AC5ED077AE389DBBA07EEB3
:10B36000903AF8EEE77AC5ED087A238ADBBA07EE61
:10B37000903AF8EEE77AC5ED097A02B070BDB3688D
:10B3800013F0010F30464FF00E0314BF3B21BB21D9
:10B39000FFF76EFAD6E709211420FDF769FB044692
:10B3A000F061B8E700B500680379012B85B012D0D1
:10B3B000022B0CD103AAF621FFF75AFA20B1BDF8EF
:10B3C0000C300C4A5BBA938205B05DF804FB002098
:10B3D00005B05DF804FB8368417C90F9100003AA76
:10B3E00003F00103CDE900230223F622F9F762F905
:10B3F000E4E700BF205C002000B500680379012B62
:10B4000085B01FD0022B19D1032303AAF621FFF721
:10B410002FFA80B19DF80D309DF80CC010499DF8B1
:10B420000E201B0243EA0C431343B1F93420C2F14E
:10B430000802D3408B6305B05DF804FB002005B023
:10B440005DF804FB8368417C90F9100003AA03F0C7
:10B450000103CDE900230323F622F9F72BF9D8E7FE
:10B46000205C002010B500680379012B84B032D035
:10B47000022B25D1062302AAF721FFF7F9F9F8B12B
:10B480009DF809209DF808409DF80A109DF80C30A1
:10B490009DF80BC0120142EA043242EA11121B016C
:10B4A0009DF80D10134C43EA0C3343EA1113124973
:10B4B000E265E363C1F8002EC1F8043E04B010BD9C
:10B4C0000D4A0C4BD2F8001ED2F8042ED96500208C
:10B4D000DA6304B010BD8368417C90F9100002AAC1
:10B4E00003F00103CDE900230623F722F9F7E2F880
:10B4F000C5E700BF205C0020186D002000B5006883
:10B500000379012B85B01DD0022B0AD1836813F07B
:10B51000010F03AA4FF0030314BF00218021FFF79E
:10B52000A7F99DF80D309DF80C009DF80E100C4AFF
:10B530001B0243EA00430B430120C2F8803005B0F0
:10B540005DF804FB8368417C90F9100003AA03F0C6
:10B550000103CDE9002303230022F9F7ABF8E0E76C
:10B56000205C002000B500680379012B85B01DD058
:10B57000022B0AD1836813F0010F03AA4FF00303D3
:10B5800014BF00218021FFF773F99DF80D309DF85D
:10B590000C009DF80E100C4A1B0243EA00430B43BB
:10B5A0000120C2F8943005B05DF804FB8368417C4B
:10B5B00090F9100003AA03F00103CDE9002303234F
:10B5C0000022F9F777F8E0E7205C002010B500686A
:10B5D0000379012B84B029D0022B24D1836813F086
:10B5E000010F4FF0030303AA14BF19468321FFF78D
:10B5F0003FF9B0B19DF80C309DF90C109DF80D206D
:10B600009DF80EC01B04002943EA0223B8BF4FF087
:10B610007F410D4AA8BF002143EA0C030B43C2F847
:10B62000D83004B010BD002004B010BD8268417C49
:10B6300090F9100002F00102032303ACCDE90042AF
:10B640001A46F9F737F8D4E7205C002000B5006807
:10B650000379012B85B02BD0022B25D1836813F001
:10B66000010F03AA4FF0030314BF00218021FFF74D
:10B67000FFF8B0B19DF80C309DF90C109DF80D202D
:10B680009DF80EC01B04002943EA0223B8BF4FF007
:10B690007F410E4AA8BF002143EA0C030B43C2F8C6
:10B6A000BC3005B05DF804FB002005B05DF804FB7C
:10B6B0008368417C90F9100003AA03F00103CDE9EF
:10B6C000002303230022F8F7F5FFD2E7205C0020D7
:10B6D00010B5044600230068E386A3630279012ABB
:10B6E00084B022D0022A1DD1836813F0010F02AA70
:10B6F0004FF0060314BF03218321FFF7B9F878B197
:10B70000BDF90A30BDF80810BDF80C205B4201EB12
:10B71000410103EB430302EB4202E1862387628788
:10B7200004B010BD184604B010BD8368417C90F988
:10B73000100003F00103019302AB009303220623E0
:10B74000F8F7B8FFDBE700BF00B500680379012B0D
:10B7500085B00DD0022B07D1012303AAFF21FFF7EB
:10B7600087F805B05DF804FB002005B05DF804FB28
:10B770008268417C90F9100002F00102019203AA54
:10B780000092FF22F8F796FF05B05DF804FB00BFBA
:10B7900070B50446244894F9103003EB8303154632
:10B7A00050F82300A3689A0782B00ED5019064F088
:10B7B000EDF8012301980022294664F097F8A36868
:10B7C0009B0717D5012002B070BD636913B11A68D9
:10B7D0009B885383154B164A1B6856684FEAC30C67
:10B7E000144BA3FB0C3C4FEA9C1C53689B1B9C45D1
:10B7F000FBD2DBE70D4B0E491A680E4B4FF4FA7083
:10B8000000FB02F2A3FB0232486892094B681B1A44
:10B810009A42FBD26369002BD4D01A689B881383A9
:10B82000012002B070BD00BF600D0020CC330020AD
:10B83000001000E0D34D621010B50379012B82B0E7
:10B840008E460DD0022B08D18368DB0758BF41F02C
:10B85000800102B0BDE810409AE7002002B010BDA0
:10B8600014468268009402F00102417C90F91000B5
:10B8700001927246F8F71EFF02B010BD70B5056860
:10B880002B79012B84B004460E4615D0022B10D123
:10B89000AB68E122DB074CBF114661212846FBF76C
:10B8A000D7FD30B120683246FF2104B0BDE87040BA
:10B8B000C2E7002004B070BDAA68697C95F9100049
:10B8C00002F001020DF10F0501920095E1228DF8C1
:10B8D0000F20F8F723FFE4E770B505682B79012BFB
:10B8E00084B004460E4616D0022B11D1AB68DB079C
:10B8F0004FF0C3024CBFE12161212846FBF7A8FDB0
:10B9000030B120683246FF2104B0BDE8704093E7B3
:10B91000002004B070BDAA6895F91000697C02F09F
:10B92000010201920DF10F020092C3228DF80F2047
:10B93000E122F8F7F3FEE3E770B505682B79012BF8
:10B9400084B004460E461AD0022B15D1AB68DB0733
:10B950004FF0F0024CBFE12161212846FBF778FD52
:10B9600050B12246FF2152F8040BFFF765FF18B1D2
:10B970002379337004B070BD002004B070BDAA6894
:10B9800095F91000697C02F0010201920DF10F029D
:10B990000092F0228DF80F20E122F8F7BFFEDFE7DA
:10B9A000F0B5044683B000680021FEF7CFF92068A7
:10B9B00015227E21FDF7F0FF642704F0E5FF054620
:10B9C0000E4604F0E1FF431B61EB0602B3F57A7FFC
:10B9D00072F10003F5D3013FEFD1206811227E21DF
:10B9E000FDF7DAFF052704F0CFFF05460E4604F009
:10B9F000CBFF431B61EB0602B3F57A7F72F10003C4
:10BA0000F5D3013FEFD120680DF107020321FFF7C5
:10BA100013FF9DF8073003F03C03142B40F09A808D
:10BA20000C2240212068FDF7B7FF04F0ADFF05466A
:10BA30000E4604F0A9FF431B61EB0602B3F57A7FC3
:10BA400072F10003F5D3454DA16B454AB5FBF1F109
:10BA5000092389B294F83500FDF732F94388B5FB24
:10BA6000F3F52564027920684221FDF795FF04F083
:10BA70008BFF05460E4604F087FF431B61EB060271
:10BA8000B3F57A7F72F10003F5D3082241212068D3
:10BA9000FDF782FF04F078FF05460E4604F074FFC0
:10BAA000431B61EB0602B3F57A7F72F10003F5D315
:10BAB000002243212068FDF76FFF04F065FF054673
:10BAC0000E4604F061FF431B61EB0602B3F57A7F7B
:10BAD00072F10003F5D3102251212068FDF75CFFBD
:10BAE00004F052FF05460E4604F04EFF431B61EB87
:10BAF0000602B3F57A7F72F10003F5D30A225321CF
:10BB00002068FDF749FF04F03FFF05460E4604F0AC
:10BB10003BFF431B61EB0602B3F57A7F72F1000332
:10BB2000F5D3802256212068FDF736FF04F02CFF64
:10BB300005460E4604F028FF431B61EB0602B3F5F1
:10BB40007A7F72F10003F5D320680321FEF7FEF837
:10BB500003B0F0BD062004F073FF00BF40420F00A9
:10BB6000548907082DE9F0417C4A0468816B7C4FB9
:10BB7000B7FBF1F182B006460F2389B290F8350089
:10BB8000FDF79EF800214388B7FBF3F705463764BD
:10BB90002046FEF7DBF80F224E212046FDF7FCFE83
:10BBA0004FF00F0804F0F0FE06460F4604F0ECFEDE
:10BBB000831B61EB0701B3F57A7F71F10003F5D3C5
:10BBC000B8F10108EED16A794F2102F00F02204648
:10BBD000FDF7E2FE4FF00F0804F0D6FE06460F46D2
:10BBE00004F0D2FE831B61EB0701B3F57A7F71F19C
:10BBF0000003F5D3B8F10108EED16A79502102F0C3
:10BC00000F022046FDF7C8FE4FF00F0804F0BCFEFF
:10BC100006460F4604F0B8FE831B61EB0701B3F53F
:10BC20007A7F71F10003F5D3B8F10108EED16A799A
:10BC300042EA02125221D2B22046FDF7ADFE0F2792
:10BC400004F0A2FE05460E4604F09EFE431B61EB87
:10BC50000602B3F57A7F72F10003F5D3013FEFD10D
:10BC6000032214212046FDF797FE0F2704F08CFED7
:10BC700005460E4604F088FE431B61EB0602B3F551
:10BC80007A7F72F10003F5D3013FEFD13A46632189
:10BC90002046FDF781FE642704F076FE05460E4639
:10BCA00004F072FE431B61EB0602B3F57A7F72F17A
:10BCB0000003F5D3013FEFD1082265212046FDF7AF
:10BCC0006BFE0DF1070264212046FFF7B5FD9DF8DC
:10BCD000072022F0100242F06002642120468DF815
:10BCE0000720FDF759FE0F2704F04EFE05460E46CD
:10BCF00004F04AFE431B61EB0602B3F57A7F72F152
:10BD00000003F5D3013FEFD10DF106024D2120468E
:10BD1000FFF792FD9DF8062002F03F0242F040023C
:10BD20004D2120468DF80620FDF736FE0F2704F042
:10BD30002BFE05460E4604F027FE431B61EB060270
:10BD4000B3F57A7F72F10003F5D3013FEFD1032100
:10BD50002046FDF7FBFF02B0BDE8F0818C890708A3
:10BD600040420F00F0B583B015460DF107021C46A6
:10BD700006460F46FFF760FD9DF8072005EA02031F
:10BD8000A34201D103B0F0BD22EA050222433946A5
:10BD9000304603B0BDE8F040FDF7FEBDF0B5044607
:10BDA00083B00D461746061D20680379012B18D075
:10BDB000022B13D18368DB0732464FF0FF015CBFD3
:10BDC0003246FF21FFF7E4FC30B115B12379DB07E0
:10BDD000EAD40FB123793B7003B0F0BD002003B06B
:10BDE000F0BD8268417C90F9100002F00102CDE9BB
:10BDF0000062FF22F8F75EFCE6E700BF30B50446BC
:10BE000083B0051D20680379012B14D0022B0FD1BC
:10BE10008368DB072A464FF0FF015CBF2A46FF21FB
:10BE2000FFF7B6FC10B12379DB07EBD403B030BDCC
:10BE3000002003B030BD8268417C90F9100002F010
:10BE40000102CDE90052FF22F8F734FCEAE700BF17
:10BE500030B50246044652F8040B0379012B83B037
:10BE60000ED0022B09D1FF21FFF792FC18B12079E7
:10BE7000C04300F0010003B030BD002003B030BD6E
:10BE80008568417C90F91000009205F0010501954C
:10BE9000FF22F8F70FFCE9E730B5B42283B004467F
:10BEA000FF210068FDF778FD10B9002003B030BD18
:10BEB00020680379012B04F1040514D0022BF4D17E
:10BEC0008368DB072A464FF0FF015CBF2A46FF214B
:10BED000FFF75EFC0028E8D02379DB07E6D5206871
:10BEE0000379012BEAD18268417C90F9100002F0BD
:10BEF0000102CDE90052FF22F8F7DCFBEAE700BFC0
:10BF000030B50A4683B00446A5210068FDF744FD1C
:10BF100010B9002003B030BD20680379012B04F173
:10BF2000040514D0022BF4D18368DB072A464FF0B6
:10BF3000FF015CBF2A46FF21FFF72AFC0028E8D05A
:10BF40002379DB07E6D520680379012BEAD18268E3
:10BF5000417C90F9100002F00102CDE90052FF226D
:10BF6000F8F7A8FBEAE700BF70B582B0CDE900237F
:10BF70000446FFF791FF10B9002002B070BD2068A1
:10BF80005522A521FDF708FD0028F5D0251D2068C4
:10BF90002A46FF21FFF750FC0028EDD02379DB076C
:10BFA000F5D40DF1FF350DF1070615F8011F2046F8
:10BFB000FFF7A6FF0028DFD0B542F6D1DDE700BFCE
:10BFC000002A37D0F0B5013A83B004464E1E51FA2C
:10BFD00082F7051D16F8012F2068A521FDF7DCFC6E
:10BFE00090B9002003B0F0BD8268417C90F9100048
:10BFF00002F00102CDE90052FF22F8F75BFB0028B6
:10C00000EFD02379DB0710D520680379012BEBD023
:10C01000022BE6D18368DB072A464FF0FF015CBFA5
:10C020002A46FF21FFF7B4FBE9E7B742D2D101204E
:10C0300003B0F0BD0120704770B5962282B004466F
:10C040000E460068FF21FDF7A7FC10B9002002B0E2
:10C0500070BD251D20680379012B1FD0022BF5D15F
:10C060008368DB072A464FF0FF015CBF2A46FF21A9
:10C07000FFF78EFB0028E9D02379DB07EAD4E12221
:10C0800020681146FDF788FC0028DFD02068324682
:10C09000FF2102B0BDE87040FFF7CEBB8268417C53
:10C0A00090F9100002F00102CDE90052FF22F8F7EA
:10C0B00001FBDFE7002A46D0F0B5013A4F1C83B000
:10C0C00004460E4657FA82F7051D20689622FF2186
:10C0D000FDF762FC90B9002003B0F0BD8268417C9E
:10C0E00090F9100002F00102CDE90052FF22F8F7AA
:10C0F000E1FA0028EFD02379DB0710D52068037917
:10C10000012BEBD0022BE6D18368DB072A464FF0E8
:10C11000FF015CBF2A46FF21FFF73AFBE9E7E12276
:10C1200020681146FDF738FC0028D4D0206832463C
:10C13000FF21FFF781FB0028CDD00136BE42C4D1DC
:10C14000012003B0F0BD0120704700BF70B5054667
:10C150000B460446164655F8040B82B087211A4652
:10C16000FDF71AFC20680379012B18D0022B13D19C
:10C170008368DB072A464FF0FF015CBF2A46FF2198
:10C18000FFF706FB30B12379DA07EBD416B1C3F31E
:10C190004013337002B070BD002002B070BD8268E1
:10C1A000417C90F9100002F00102CDE90052FF221B
:10C1B000F8F780FAE6E700BF70B5782182B0044650
:10C1C000164600680022FDF7E7FB10B9002002B018
:10C1D00070BD251D20680379012B14D0022BF5D1E9
:10C1E0008368DB072A464FF0FF015CBF2A46FF2128
:10C1F000FFF7CEFA0028E9D02379DA07EAD45B0901
:10C20000337002B070BD8268417C90F9100002F07A
:10C210000102CDE90052FF22F8F74CFAEAE700BF2D
:10C2200030B5CC2283B00446A5210068FDF7B4FBED
:10C2300010B9002003B030BD20680379012B04F150
:10C24000040514D0022BF4D18368DB072A464FF093
:10C25000FF015CBF2A46FF21FFF79AFA0028E8D0C9
:10C260002379DB07E6D520680379012BEAD18268C0
:10C27000417C90F9100002F00102CDE90052FF224A
:10C28000F8F718FAEAE700BF30B5B42283B00446E5
:10C29000FF210068FDF780FB10B9002003B030BD1E
:10C2A000251D20680379012B22D0022BF5D183684C
:10C2B000DB072A464FF0FF015CBF2A46FF21FFF74C
:10C2C00067FA0028E9D02379DA07EAD4CC2120469E
:10C2D000FFF716FE0028E0D002E02379DB07DDD56A
:10C2E00020682A46FF21FFF7A7FA0028F5D1D4E7F6
:10C2F0008268417C90F9100002F00102CDE9005201
:10C30000FF22F8F7D7F9DCE72DE9F04F89B00446B2
:10C31000CDE90623002004F1040B04900291039060
:10C320005D462046049FFFF7B7FD069BFE0003EB2A
:10C33000C70B20B90AE0237913F0010A0CD020685A
:10C340002A46FF21FFF778FA0028F4D1079B049AC8
:10C350001A7009B0BDE8F08F9B07F7D5F021204691
:10C36000FFF7CEFD0028F1D0069B083E334401279D
:10C370000593D0463E46029B002B4AD0082E48D853
:10C3800006F1FF3943FA09F909F0010920684FEA7B
:10C39000C9127821FDF700FB0028D7D02068037967
:10C3A000012B47D0022B43D18368DB072A464FF08D
:10C3B000FF015CBF2A46FF21FFF7EAF90028C5D03C
:10C3C000237913F00102E9D103F0600160294FEAFB
:10C3D000D31C51D0029919B1082E01D8E145B5D12D
:10C3E000BCF1000F3AD01BF808303B430BF8083083
:10C3F0007F00013617F0FF07F6B2BCD108F1010843
:10C400005FFA88F8B8F1080F36D0029B0127002B9D
:10C41000B4D1049BD3B1039BB34217D9059B13F846
:10C4200008301F4214BF4FF001094FF00009ADE77B
:10C4300000208BE78268417C90F9100002F0010235
:10C44000CDE90052FF22F8F735F9B7E7039BA3EBDC
:10C450000609B9FA89F94FEA591997E71BF8081044
:10C4600021EA07010BF80810990941EA531313F068
:10C47000010F08BFB246BBE7402E06D8079B049ABF
:10C480001B7893423FF64DAF60E79BF807C00BF176
:10C49000FF370BF1060B17F8011F082382EA01068C
:10C4A00016F0010F4FEA520218BF82F08C0203F11E
:10C4B000FF3318BFD2B213F0FF034FEA5101EDD1A1
:10C4C000BB45E8D19445D9D1049B0133DBB2049339
:10C4D000BAF1000F3FF43AAFCDF80CA0CEE700BFA1
:10C4E00030B505682B79012B85B0044600F09280A9
:10C4F000022B08D1AB68DB0702AA4CBF08218821B8
:10C500002846FFF745F99DF8083013F0100302D1D3
:10C51000184605B030BD2068062302AA0021FEF7A8
:10C52000FDF90028F5D09DF809209DF808109DF828
:10C530000A309FED3F6A120202EB014213441402DB
:10C5400048BF03F17F4307EE903AF8EEE77A9DF893
:10C550000C109DF80B409DF80D20364BC7EE866AF7
:10C56000090201EB04410A44090248BF02F17F427B
:10C5700007EE902AB3F9742007EE102AB3F9702061
:10C58000F8EEE77A05EE102A87EE864AB3F96C20BA
:10C59000B8EEC77AB8EEC55AD3ED1A7AA6EE875A26
:10C5A000F8EEE75A04EE902AE6EE855AB3F97220C7
:10C5B000D3ED197A03EE902AF8EEE77AB3F96E20FC
:10C5C000E6EEA57A06EE102AB3F96220F8EEE44A08
:10C5D000F8EEE33A07EE102AB8EEC66AB3F9602027
:10C5E000A6EEA36AE4EE247A05EE902AB8EEC77AA6
:10C5F00066EE846AF8EEE55A27EE047AB6EE005A43
:10C60000A5EE857AE6EE867A83ED1F7AC3ED1E7A73
:10C6100005B030BDAA68697C95F9100002F00102EE
:10C62000019202AA00920822F8F744F86BE700BFD3
:10C6300000007848205C002030B505682B7987B071
:10C640000022012B04468DF80F2035D0022B12D189
:10C65000AB68DB070DF10F024CBF2721A72128464D
:10C66000FFF796F828B19DF80F3013F0080305D1B5
:10C67000184607B030BD104607B030BD206806230D
:10C6800004AA2821FEF74AF920B3BDF91030BDF9FC
:10C690001220002BB8BF03339B10E386BDF9143082
:10C6A000002AB8BF0332002BB8BF033392109B108F
:10C6B0002287638707B030BDAA68697C95F91000AE
:10C6C00002F0010201920DF10F0200922722F7F70A
:10C6D000F1FFC7E7E086A06307B030BD30B505467F
:10C6E00000240068EC86AC630379012B87B02AD064
:10C6F000022B0ED18368DB070DF10F024CBF2146E0
:10C700008021FFF745F828B19DF80F4014F0080488
:10C7100002D1204607B030BD2868062304AA0121B3
:10C72000FEF7FCF80028F5D0BDF81430BDF8101065
:10C73000BDF812205BBA49BA52BA5B42E9862A8731
:10C740006B8707B030BD22468468417C90F91000A9
:10C7500004F0010401940DF10F040094F7F7AAFF0F
:10C76000D1E700BF30B5044600202568E086A0630D
:10C770002B79012B87B027D0022B10D1AB68DB07B8
:10C780000DF10F024CBF062186212846FFF700F865
:10C7900028B19DF80F3013F0040302D1184607B0FA
:10C7A00030BD2068062304AA0021FEF7B7F8002850
:10C7B000F5D0BDF81010BDF81220BDF81430E18698
:10C7C0002287638707B030BDAA68697C95F910009D
:10C7D00002F0010201920DF10F0200920622F7F71A
:10C7E00069FFD5E710B50368DA6B82B0044612B171
:10C7F000904740B123685B6B1BB1214601A8984765
:10C8000018B9FF23E38202B010BDBDF80630013B2A
:10C810009BB2F7E7F0B585B0044618460D461646BC
:10C82000039363F0AFF928442768A073E6732046AA
:10C8300000240094039B7C6932462946A04705B03A
:10C84000F0BD00BF38B504468B6801600D469847BF
:10C8500000230B4A226123752B6B13B120469847A6
:10C860002075084B93F8083E1BB1237D23F001038C
:10C8700023750023E3822046BDE83840B2E700BFBD
:10C880000001FF00186D002010B5154BD3F80C4EB9
:10C8900084B024B12379012B10D0022B02D00020C8
:10C8A00004B010BDA16811F00101024618BF80213B
:10C8B000204604B0BDE81040FAF7CABDA268617C0A
:10C8C0008DF80F0002F0010294F910000DF10F0431
:10C8D000CDE900428022F7F721FF04B010BD00BF70
:10C8E000186D00202DE9F041264ED6F80C5E84B07C
:10C8F0009DB1B02280212846FDF74EF840228021CC
:10C900002846FDF749F8002280212846FDF744F823
:10C91000102280212846FDF73FF84FF480644FF045
:10C9200000080DF10F0795B12B79012B15D0022BC3
:10C930000DD1AB6813F001034FF000024FF040013E
:10C94000284602BF1A4640212846FAF781FD013CDD
:10C95000A4B29CB1D6F80C5EE5E7AA6895F9100080
:10C96000697C8DF80F8002F00102013CCDE9007274
:10C97000A4B24022F7F7D2FE002CEBD104B0BDE800
:10C98000F08100BF186D00200B4B10B5D3F80C4E92
:10C990008CB15038C2B280212046FCF7FDFF002246
:10C9A00080212046FCF7F8FF20461022BDE8104009
:10C9B0008021FCF7F1BF10BD186D0020F0B5204CB0
:10C9C000204F203800EB8000661DD7F80C5E85B044
:10C9D00004440644E5B12B792278012B1DD0022BAB
:10C9E0000AD1AB6813F0010F4FF04001284604BF95
:10C9F00040212846FAF72CFD0134B442EAD155B162
:10CA000000224021284605B0BDE8F040FCF7C4BF35
:10CA10000134B442F0D105B0F0BD8DF80F20AA6802
:10CA200095F91000697C02F0010201920DF10F02EC
:10CA300000924022F7F772FED7F80C5EDCE700BFE9
:10CA4000E8890708186D00202DE9F041734ED6F8EB
:10CA50000C5E84B0002D00F09680D4228021284600
:10CA6000FCF79AFF802211462846FCF795FFA82282
:10CA700080212846FCF790FF3F2280212846FCF7C2
:10CA80008BFFD32280212846FCF786FF00228021DD
:10CA90002846FCF781FF402280212846FCF77CFFD6
:10CAA0008D2280212846FCF777FF1422802128461A
:10CAB000FCF772FFA12280212846FCF76DFFC822F7
:10CAC00080212846FCF768FFDA2280212846FCF7FF
:10CAD00063FF122280212846FCF75EFF812280211D
:10CAE0002846FCF759FFCF2280212846FCF754FF47
:10CAF000D92280212846FCF74FFFF12280212846C9
:10CB0000FCF74AFFDB2280212846FCF745FF402244
:10CB100080212846FCF740FFA42280212846FCF70C
:10CB20003BFFA62280212846FCF736FFAF2280215A
:10CB30002846FCF731FFA62280212846FCF72CFF6F
:10CB4000AE2280212846FCF727FF2022802128469C
:10CB5000FCF722FF002280212846FCF71DFFB022AF
:10CB600080212846FCF718FF402280212846FCF748
:10CB700013FF002280212846FCF70EFF102280219F
:10CB80002846FCF709FF4FF480644FF000080DF1D0
:10CB90000F0755B32B79012B2FD0022B0DD1AB688A
:10CBA00013F001034FF000024FF04001284602BF8E
:10CBB0001A4640212846FAF74BFC013CA4B2002C4F
:10CBC000E7D175B1812280212846FCF7E5FEC82215
:10CBD00080212846FCF7E0FEAF2280212846FCF7A2
:10CBE000DBFE012004B0BDE8F081013CA4B2002CC2
:10CBF000E3D1012004B0BDE8F081AA6895F91000E6
:10CC0000697C8DF80F8002F00102CDE900724022AC
:10CC1000F7F784FDD6F80C5ECFE700BF186D002053
:10CC2000FAF7BEBEFAF7BCBEFAF7BABEFAF7B8BE5C
:10CC3000FAF7B6BEFAF7B4BE10B50409013C032CEE
:10CC400018D80E4A32F8141000F00F0341FA03F21C
:10CC500012F0010210D001209840013808406BF01A
:10CC600031FB074B074A1B5D184400EB400002EB09
:10CC7000800010BD002010BD104610BDA48607081E
:10CC8000A0860708542800202DE9F04F54220446BE
:10CC90000021BF4893B069F065FCBE4A611EE01CEC
:10CCA000144611F8013F5D1E052D88BF0023884200
:10CCB00044F8043BF5D102F11003114651F8040B7E
:10CCC000012800F07D819942F8D1114651F8040BFA
:10CCD000022800F053819942F8D1114651F8040B13
:10CCE000032800F077819942F8D152F8041B0429F7
:10CCF00000F03A819A42F8D10520FAF73FF8062071
:10CD0000FAF73CF8A24DDFF8A892DFF8A8821A26BD
:10CD100000272C7B002C40D02046FFF78DFF95F993
:10CD20000DA08346E0B103689B498BF8076003F1CF
:10CD30003F4303F57E039B0A0522C85C8BF806205F
:10CD400000238BF8083060F02DF9944ABBF80430CA
:10CD50000492DBF80000039303A9F6F709FE2C7B8D
:10CD60000023302201E019F8332094422ED0013301
:10CD7000102BF8D100200AEB4A0A08EBCA03012263
:10CD8000D3F8B41728618C180720C3F8B447297565
:10CD9000A8756A7583F8B02717440136F6B2202EBD
:10CDA00005F10C05B5D177B17D4CDFF80CA2DFF8A9
:10CDB0000C920025237C7BB90135032D04F1180466
:10CDC0000AF58C7AF6D113B0BDE8F08F754A02EB04
:10CDD000C303D3F8E005CEE7607960F0E3F820798B
:10CDE00060F0E0F8A068F6F72DFD2368A068CDF8A4
:10CDF00014A04C3304936369142202FB03F30793DA
:10CE00000023CDE90E33CDE9103306930893E36890
:10CE100003934FF480624FF40063CDE909234FF48C
:10CE200000514FF48073CDE90B134FF4003303A985
:10CE30000D9360F08BF8A2685B49136843F001031F
:10CE40001360D9F8043023F4733323F4477323F0C9
:10CE5000030343F44033C9F804302268636950681F
:10CE6000012B20F0407020F48070D4BF00260126F2
:10CE700040EA062050609068014041F00201916054
:10CE8000D16A013B21F47001DBB241EA0353D36262
:10CE90003F4B012103F148074FFA85F802E00C33BC
:10CEA000BB422ED0587D0028F9D093F90D004045A3
:10CEB000F5D1187C9E7D01F1010C09285FFA8CFCEC
:10CEC00030D800EB400E06FA0EF6D2F810B00196FC
:10CED000072606FA0EFE019E2BEA0E0E46EA0E0605
:10CEE0001661062930D8013901EB81011F268840DF
:10CEF0008E406146D2F834C02CEA060630435063B7
:10CF0000CDE7936843F400739360936843F48073B0
:10CF10009360936843F001039360936843F0804308
:10CF2000936049E7A0F10A0E0EEB4E0E4FF0070B8F
:10CF300006FA0EF60BFA0EFED2F80CB02BEA0E0E25
:10CF400046EA0E06D660CCE70C294DD8073901EB2E
:10CF500081011F2688408E406146D2F830C02CEAFD
:10CF60000606304310639AE7104B93F8942A302159
:10CF7000013283F8701A83F8942ABDE60B4991F8C0
:10CF8000940A3524013081F8584A81F8940AA4E6BD
:10CF900058770020245C00208486070803000100E5
:10CFA00000150020B0860708FDF7FFC0186D0020AF
:10CFB0008C8C0708600D0020B07700200023014012
:10CFC000104991F8940A3424013081F84C4A81F8D0
:10CFD000940A7AE60B4991F8940A2024013081F8EA
:10CFE000644A81F8940A80E60D3901EB81011F261D
:10CFF00088408E406146D2F82CC02CEA06063043A9
:10D00000D0624CE7186D002010B503681A79022A27
:10D01000044603D000232371236010BD987AFFF7E4
:10D020000BFE0028F6D040F61A610022C180027281
:10D030002021FCF739FE00232371236010BD00BFBF
:10D0400070B506461C48336803F13F4303F57E0381
:10D050009B0A82B0C05C0C4615465FF0A3FFB28805
:10D060000092B2FA82F304F003028DF80420C4F3B4
:10D07000810230688DF80520C3F11F03C4F300124C
:10D0800064098DF80740C3F3CC0400EB840403F07B
:10D0900007038DF806209B00226A0F269D4006FAA2
:10D0A00003F322EA03032362226A154369462562D9
:10D0B000F6F75EFC02B070BD848607082DE9F04FDC
:10D0C000A84CA94DAC4283B050D21E4602E00C34AD
:10D0D000AC424BD294F805C08C45F8D194F804C00A
:10D0E000844501D00028F2D194F807C09445EED1D0
:10D0F0002568002D3BD000236B60AB60EB602B619B
:10D100006B61AB61EB612C6022792A71A779AF600A
:10D11000217AE960012A33D0022A27D1E07AFFF789
:10D120008BFD94F90980A861A07A85F81080FFF73B
:10D1300083FD6861F8B18D4C08EB880A4FEA8809D5
:10D1400054F82A3004EB8A0AABB19AF8123003B3D0
:10D150000E2200238671C27103720921FCF7A4FD1F
:10D160006B6923B11A689B88138300E00025284669
:10D1700003B0BDE8F08F2846FFF746FF0025F6E72D
:10D18000E07AFFF759FD627AA37A6B74A8612A747A
:10D19000EDE79AF808005FF005FF9AF808104A09D1
:10D1A000012301F01F01023A8B40032A08D8DFE86F
:10D1B00002F0A7ADA1026E494A6922EA03034B615E
:10D1C00009EB080304EB830308F1010A5879FFF720
:10D1D00033FD5FFA8AFA014620B140F60A3380F83F
:10D1E00008A0C38009EB080304EB83030091D879FE
:10D1F000FFF722FD0099034620B140F60A5280F85D
:10D2000008A0C28009EB080204EB8202CDE90013FA
:10D210009079FFF711FDDDE90013834620B140F658
:10D220000A4280F808A0C28009EB080204EB8202DF
:10D2300017F0040A527A6FD039B108464A21019397
:10D240000092FFF7FDFEDDE900232BB118462A21ED
:10D250000092FFF7F5FE009ABBF1000F03D058468D
:10D260000A21FFF7EDFE09EB080B04EB8B0B9BF893
:10D270000470002F6BD109EB08033E4A54F82330A9
:10D28000934200F099803C4A934200F0AB803B4AC5
:10D29000934200F09C803A4A934200F08280394ADF
:10D2A000934273D0384A934200F0A7801A88BAF1AB
:10D2B000000F02F441510CBF032200220A4342F442
:10D2C00045721A809A8B22F400621204120C9A831F
:10D2D00007221A821A8892B242F040021A806FBB6B
:10D2E000C844686904EB88040123A37400283FF450
:10D2F00034AF2DE71E490A6922EA03030B615FE799
:10D300001B494A6A22EA03034B6259E718490A6A31
:10D3100022EA03030B6253E739B108460A2101935D
:10D320000092FFF78DFEDDE90023002B94D0184614
:10D330000A210092FFF784FE009A8DE73846FFF736
:10D340007BFC0028CCD0036882881A83C8E7384663
:10D35000FFF772FC00288ED09BF809200921FFF707
:10D360006FFE88E748A60808F8A70808600D0020A7
:10D37000003802400030014000380040003C0040CE
:10D3800000340140005001400054014002F5684261
:10D39000516A41F480115162516A21F48011516245
:10D3A00084E702F58232516A41F400515162516AB8
:10D3B00021F40051516279E702F58432516A41F457
:10D3C00080515162516A21F4805151626EE702F539
:10D3D000FE32116A41F400411162116A21F40041E8
:10D3E000116263E702F50032116A41F48041116273
:10D3F000116A21F48041116258E702F56442516AD2
:10D4000041F400115162516A21F4001151624DE75B
:10D410002DE9F043002383B01A4636210120FFF79F
:10D420004DFEDFF87C900746C9F8100E60B34FF050
:10D430000508962603F0A8FA04460D4603F0A4FA60
:10D44000031B61EB0501B3F57A7F71F10003F5D39E
:10D45000013EEFD10DF1070231463846FEF7ECF9F7
:10D46000044668B9B8F10108E3D199F8143ED9F837
:10D47000100E0C2B04BF0223C9F8183EFFF7C4FDA1
:10D48000204603B0BDE8F08399F8143E0C2B01D080
:10D490000446F5E70123C9F8183E0446F0E700BF4B
:10D4A000186D0020074B53F8203021B14BB11A689A
:10D4B0009B8853837047002BFCD01A689B8813838A
:10D4C00070477047948607081D4B70B5D3F81C4110
:10D4D00074B193F8CC3D05465BB162685379032B78
:10D4E0002BD8DFE803F021242702136840331D60A6
:10D4F00070BDE068666881680A6822F001020A600F
:10D500003168104A767932F816608A8992B222EA36
:10D5100006028A8123740A8892B242F001020A80CC
:10D520000377FAF741FBD8E713683433DFE7136872
:10D530003833DCE713683C33D9E700231B60FFDE98
:10D54000205C0020BC850708254BD3F81C219AB12C
:10D5500093F8CC1D81B110B5224C94F8381E0329E4
:10D560000BD0022911D0002283F8CC2DFAF738FA1B
:10D5700008B984F8390E10BD704752685379032BEF
:10D580002AD8DFE803F023201D1852685379032BB3
:10D590001FD8DFE803F00D0A0702136840330022AA
:10D5A0001A6010BD13683C33F9E713683833F6E7A7
:10D5B00013683433F3E71368403364221A6010BDF4
:10D5C00013683C33F9E713683833F6E713683433EC
:10D5D000F3E700231B60FFDE00231B60FFDE00BFBC
:10D5E000205C0020186D00202DE9F04FBA4BDFF8C9
:10D5F000F4E293F83C9E93F83D8E93F83E7EDFF87C
:10D60000E8A283B0002603F5646501960124AB7897
:10D61000E978C3F1FF039BB2002B40F092800B46E8
:10D620000F468C460A468846894601210191100220
:10D6300040EA0340172240EA0C0006EB020CACEB78
:10D6400002032A3304FA02F19BB201420EEB830378
:10D6500014BF02210121013AC3F82011531CEED15D
:10D660009E4B04351836AB42B6B2D0D19A4A4FF42D
:10D670004073A2F8C03E2023A2F8C23E019B2BB10A
:10D6800082F83C9E82F83D8E82F83E7E924B93F863
:10D69000393E002B52D0DEF81C31002B4ED0EFF378
:10D6A0001181102282F31288D8685D68846822682C
:10D6B00022F0010222602C68894A6D7932F81550F7
:10D6C000A28992B222EA0502A281026944681F2A55
:10D6D00040F2E080203A202000FA02F2E260CAB272
:10D6E00082F31188DA68DEF81C01926840F22B316F
:10D6F000516011680124214311601C7403681A7D74
:10D70000A24204BF02221A7593F82C100CBF4FF4EA
:10D7100000720022012904D1022183F82C1042F466
:10D72000806293F84410012900F0B98093F85C10EE
:10D73000012900F0BD80002A40F0BF8003B0BDE8A1
:10D74000F08FB5F800C0C3F1FF03AAFB0CB001FBDA
:10D7500003F340091B120A46052800F2B980DFE8EE
:10D7600000F0886C53361C03AAFB0C077F09C7EB3B
:10D770000717ACEB8707BFB2C81AC7F13C0700FB1D
:10D7800007F7AAFB07075FFA83F808EB57178946E4
:10D79000FFB20121BC46019149E7AAFB0C025209E4
:10D7A000C2EB0212ACEB820292B2A1EB030902FBC4
:10D7B00009F9AAFB09295FFA83F808EB59198C4685
:10D7C0005FFA89F90F4601214A4601912FE7AAFB2A
:10D7D0000C025209C2EB0212ACEB82081FFA88F865
:10D7E000CA1AC8F13C0802FB08F8AAFB08285FFA2D
:10D7F00083F909EB58188C465FFA88F80F46012127
:10D800001A460191434612E7AAFB0C025209C2EBE9
:10D810000212ACEB820292B2CF1A02FB07F7AAFB0C
:10D8200007275FFA83F909EB57171A46FFB20B4631
:10D8300088460121BC460191F9E6AAFB0C02520977
:10D84000C2EB0212ACEB82091FFA89F9CA1AC9F1BC
:10D850003C0902FB09F9AAFB0929DFB207EB5919B8
:10D860005FFA89F99C4688460B4601214A46019198
:10D87000DDE6A1EB03080CFB08F8DFB2AAFB080801
:10D8800007EB58185FFA88F89C46012301938946F4
:10D890004346CCE6202000FA02F2A2601FE70221F4
:10D8A00083F8441093F85C10012942F4006204D11B
:10D8B000022183F85C1042F4805243681B68002107
:10D8C0005962998989B20A439A8103B0BDE8F08F01
:10D8D00043464A46BC46AAE6186D0020D87B002085
:10D8E000BC850708205C002089888888F8B500215D
:10D8F0002120F5F779FA10B30446F5F71DFA254F04
:10D900000546C7F81C01D0B12120FFF795F9224E3A
:10D91000C6F8C40E40B140F21522C2800022027245
:10D92000227A4A21FFF78CFB96F8383E022B29D049
:10D93000032B1FD0FAF754F810B986F8390EF8BD4A
:10D9400040F6AC421548002168F00CFE96F8383ECF
:10D95000012B04BFFF23C7F8C83D97F8CC3D012237
:10D9600086F8392E002BEAD12B7C002BE7D1BDE8BD
:10D97000F84039E6FAF718F92846F5F7D1FB6423A1
:10D980000360F8BDFAF710F92846F5F7C9FB002344
:10D990000360F8BD205C0020186D0020405D002071
:10D9A0002DE9F04FDFF8A8A2A44E0021A7B04FF058
:10D9B0000A0B0C460AF6C8658FE096F8D43101963A
:10D9C0005F0618D404F1020C43F04003BCF18C0F45
:10D9D00086F8D43100F2E38004F198010DEB0109DF
:10D9E00004F199010DEB010764464FF0040C09F8AE
:10D9F0008CCC07F88C3CA71C8C2F42F0020C00F258
:10DA0000CE8004F198036B444FF0050103F88BCCF2
:10DA100004F1040CBCF18C0F03F88C1C00F2BF80E5
:10DA200004F19A010DEB01074FF0060907F88C9CF1
:10DA3000009F03F8897C4FEA880804EB09075FFA26
:10DA400088F88C2F414600F2AA8004F19C0CEC442B
:10DA50004FF007080CF88C8C04F1080CBCF18C0F0B
:10DA600003F8871C00F29B8007F198010DEB01077A
:10DA70004FF0050107F88C1C03F8852C04F10A020D
:10DA80008C2A00F28C8004F1A0010DEB010C0099AE
:10DA90000CF88C9C03F8831C04F10C018C297ED8B3
:10DAA00004F1A20204F1A3036A446B4402F88C8CD3
:10DAB0000C4603F88CEC410900F01F0755F82130A3
:10DAC0000122BA4023EA0203BBF1010B45F82130E1
:10DAD0006FD0411CB1F5F07F6BD23C222846FAF79B
:10DAE0008BF800285EDB0AEB4003C1B2B3F8043FB9
:10DAF00000915907C0F307225FFA83F84FEA132E0B
:10DB00003FF55BAF96F8D4710196790603D407F020
:10DB1000380CC44519D027F078073B4304F1020CB8
:10DB2000DBB2BCF18C0F86F8D43138D804F19801FF
:10DB30000DEB010804F199010DEB010764464FF06C
:10DB4000040C08F88CCC07F88C3CA31C8C2B26D832
:10DB500004F198010DEB010707F88B2C052207F85B
:10DB60008C2C221D8C2A1AD804F19A036B444FF096
:10DB7000060C04EB0C0103F88CCC8C29009B07F8F5
:10DB8000893C0CD804F19C0204F19D036A446B4467
:10DB90000C46072102F88C1C03F88CEC8BE76FF025
:10DBA000004488E7204614B927B0BDE8F08F234B26
:10DBB0000193019B2249D3F8CC5195F91030AA6802
:10DBC00003EB8303920751F8230023D5234603AACE
:10DBD000002161F08BFEAB689B0703D5012027B0C5
:10DBE000BDE8F08F174B18491A68184B4FF4FA70BC
:10DBF00000FB02F2A3FB0232486892094B681B1A31
:10DC00009A42FBD26B69002BE8D01A689B88138379
:10DC10000120C9E76B6913B11A689B885383094BCC
:10DC200009491A68094B4E68D200A3FB02329209D7
:10DC30004B689B1B9A42FBD2C8E700BF107E0020B6
:10DC4000600D0020CC330020001000E0D34D6210A6
:10DC5000186D0020F0B52A4CD4F8CC0183B010B177
:10DC600094F8D2310BB103B0F0BD0DF1070284215D
:10DC7000012384F8D231FDF7DFFD94F8D421D4F8E4
:10DC8000CC0142F004020421FBF786FED4F8CC015B
:10DC90000DF107028421FDF7CFFD9DF8073013F049
:10DCA0000406F3D1174D184884F8D43131463C228C
:10DCB00068F058FC05F570773146A5F13A0E01265B
:10DCC00035F8023F1A0A22F0200203F0040301F0A3
:10DCD0001F0013434FEA511C06FA00F001F1010145
:10DCE00004D05EF82C3018434EF82C00BD42E7D12A
:10DCF000FFF756FE0028FBD184F8D20103B0F0BD37
:10DD0000107E00201A7C0020E07B002070B5414D81
:10DD1000D5F8CC4182B094B395F8D031012B42D0E4
:10DD2000022B2ED1082294F910303B4885F8D321DC
:10DD300003EB8303042150F823008DF80520002312
:10DD40008DF80430A3688DF806109A078DF8071037
:10DD500042D504230DEB0302002161F0C7FDA36847
:10DD60009B0722D52D483C22FF2168F0FBFB95F84C
:10DD7000D13123B9FFF76EFF012385F8D13102B00D
:10DD800070BD0DF10302A0212046FDF755FD9DF861
:10DD9000033003F00503012B37D0002B2FD1D5F82A
:10DDA000CC410822BFE74822BDE71D4B1D491A6838
:10DDB0001D4B48684FF4FA7606FB02F2A3FB0232D1
:10DDC00092094B681B1A9A42FBD26369002BC9D097
:10DDD0001A689B881383C5E7636913B11A689B8827
:10DDE00053830F4B0F491A680F4B4E68D200A3FBA9
:10DDF000023292094B689B1B9A42FBD2A9E70B4A5D
:10DE0000126840F2DC539A42B9D9D5F8CC41482285
:10DE100089E700BF107E0020600D0020E07B00201D
:10DE2000CC330020001000E0D34D62104C270020BE
:10DE3000F0B54A4B8BB04FF4005103F5707223F8E4
:10DE4000021F9A42FBD1464E464C356804F2D31766
:10DE5000323502E033689D4250D9D4F8CC013A46BD
:10DE60008021FDF7E9FC0028F4D1102203463E4E44
:10DE700001250AE00EF8242C0132D2B2202A0346F2
:10DE800001F8245C0CF1040C12D0981C03F1280753
:10DE900003F1290122280DEB070E69449C46E9D9BC
:10DEA0000132D2B26FF00043202AB4461846ECD1BA
:10DEB000BCF1220F4FD800F128020DEB020003F154
:10DEC000280201216A4400F8241C4C21023302F884
:10DED000231CD4F8CC41254894F91020A16802EB0A
:10DEE000820250F822008A0722D501AA002161F09F
:10DEF000FDFCA3689B0704D50BB0F0BD10220023E6
:10DF0000B5E71B4B1B491A6848684FF4FA7303FBCB
:10DF100002F24FF47A73B2FBF3F24B681B1A9A4287
:10DF2000FBD26369002BE7D01A689B881383E3E771
:10DF3000626912B1116892884A830D4A0D4D1168C9
:10DF40006E68C9004FF47A72B1FBF2F16A68921BF5
:10DF50009142FBD2C9E76FF00043BAE71A7C002078
:10DF60004C270020107E002001000080600D002062
:10DF7000CC330020001000E02DE9F041334D95F83E
:10DF8000D23182B004460E46002BFDD195F8D32144
:10DF9000D5F8CC01194602F0F702012385F8D231F9
:10DFA00085F8D321FBF7F8FCE2B207460921D5F842
:10DFB000CC01FBF7F1FCB4F5807F3FD0D5F8CC0164
:10DFC000DFF88C8050220821FBF7E6FCD5F8CC0165
:10DFD0000DF10702A021FDF72FFC48B9D8F8D83081
:10DFE000B8F8DC2059690A4214BF5A831A83EDE756
:10DFF0009DF8074014F02004F0D1E2B20A21D5F8D0
:10E00000CC01FBF7C9FC3219D5F8CC01C021013491
:10E01000FDF712FC362CF0D157B995F8D321D5F87D
:10E02000CC0102F0F702394685F8D321FBF7B4FCA6
:10E03000002385F8D23102B0BDE8F081D5F8CC01DB
:10E0400040220A21FBF7A8FCB8E700BF107E0020A1
:10E05000542800202DE9F04F5F4E96F8D241C3B00E
:10E0600005460F46002CFDD196F8D321D6F8CC01F9
:10E0700002F0F7020123214686F8D32186F8D23137
:10E08000FBF78AFCFF2D4FF009038DF8055088BF80
:10E09000AD0801AA88BF05F0C008137098BFA0465C
:10E0A00002234FF0000C4FF00A0B0DF1050A4FF060
:10E0B0000B0914E0B4F5827F02F803B00AF80310EC
:10E0C00017F80C3017D80CF1010CBCF1360F02F820
:10E0D000059000F1060002F80E30234614D09D1C76
:10E0E00048EA0C01B5F5827F03F104041846C9B271
:10E0F00003F1030EDED90CF1010C6FF00044BCF10A
:10E10000360F36482346EAD1B0F5827F61D8082120
:10E1100011550DF10501A020C8540233D6F8CC41A9
:10E120002F4894F9101001EB810150F82100A168EB
:10E13000890722D5002161F0D9FBA3689B0731D55F
:10E14000284CD6F8CC010DF10302A021FDF774FB99
:10E1500048B9D4F8D830B4F8DC2059690A4214BF61
:10E160005A831A83EDE79DF8033013F02003F0D1B2
:10E1700086F8D23143B0BDE8F08F616911B10D6806
:10E18000898869831849194F0D681949D7F804C05F
:10E19000ED00A1FB0515AD097968A1EB0C018D42DD
:10E1A000FAD2C7E7104B11491A68114B48684FF46F
:10E1B000FA7505FB02F2A3FB023292094B681B1AA7
:10E1C0009A42FBD26369002BBAD01A689B881383EA
:10E1D000B6E76FF00043A1E7107E00200100008049
:10E1E000600D002054280020CC330020001000E0F7
:10E1F000D34D6210002ABCBF80185242002B30B5AC
:10E200003BDB5D180028B7BF121A841814460020A3
:10E21000A4F11D0C0029BCBF2B460021BCF1000F4E
:10E22000C8BFA2EB0C04A5F10F02C8BF2418002A36
:10E23000C4BF9B1A5D1884421EDBC1F1010C114A58
:10E24000AC44C1EB0113CCEB0C1C00EB43030134D9
:10E250004FEA4C0C02EB43024FF0200E8D42A8BF58
:10E26000002304DB22F813E01E339C45FAD1013071
:10E27000A04202F10202F1D130BD5C180D465B42B2
:10E280002146BFE71C7C00201B4B1C48196C1C4A14
:10E2900010B441F080510124196404625321FF2419
:10E2A000CA205462506251625B6FDB0085B013D4A8
:10E2B0000023144902930291029A134804320292F5
:10E2C000029A136003930391039B0393039B1860CB
:10E2D00005B05DF8044B70470A4B00220192019390
:10E2E000019B0193019A084B12689A42E0D105B054
:10E2F0005DF8044B704700BF0038024000000E423A
:10E30000002800405028004076614E690120704787
:10E310000120704731B10C4BD3ED007AF8EEE77A6B
:10E32000C1ED007A72B1084BDFED086A5B68A3F5B6
:10E33000D543333B07EE903AF8EEE77A87EEA67ABC
:10E3400082ED007A704700BF108000200000C842B4
:10E350000120704701207047704700BF034B03EB5B
:10E36000800083680BB19B681960704710800020A3
:10E37000044B03EB80039B680BB19B68196023F08F
:10E380005FB800BF10800020044B03EBC00040F2D8
:10E39000FF739942A8BF194681807047386A0020F0
:10E3A0000C4A13787BB10C4B93F8481059B193F891
:10E3B000491059B150680022FA2883F84920A8BFB3
:10E3C0004FF0FF3070476FF0010070476FF00200B0
:10E3D000704700BF48150020108000200B4B93F8B9
:10E3E0004A2082B193F84B2052B109498868002233
:10E3F000B0F5967F83F84B20A8BF4FF0FF307047F1
:10E400006FF0020070476FF001007047108000202D
:10E4100048150020014BDB6C5B681847108000201A
:10E42000014BDB6C9B68184710800020014BDB6CB4
:10E43000DB681847108000202DE9F041114C04F1F1
:10E44000500884F851101746002502234246FF2148
:10E45000064684F85050FCF7E9F980B14246304650
:10E460000223FF21FCF75AFA48B194F8502094F89F
:10E47000513003EB022328463B80BDE8F0816FF06A
:10E480000C00FAE710800020014BD868704700BFED
:10E4900048150020044B93F8503113B1034B186911
:10E4A00070476FF001007047108000204815002071
:10E4B000437A5A1C0344D2B242729972037A93424D
:10E4C00000D97047002AFCD010B5044604F10A01B7
:10E4D000D0E9003098470023637210BD2A4ED6F869
:10E4E0005451D6F8600108B52EF012F828462EF0E7
:10E4F0000FF8D6F8600141798B073ED50021084618
:10E50000FEF7D0FF00210120FEF7CCFF1F4CD6F80C
:10E51000600103685B689847D0B92B6828465B6840
:10E5200098470028F3D0D4F89C202B68B4F8A010AA
:10E53000DB685183284698470146D6F86001026897
:10E5400013689847D4F89C30B4F8A0201A83DEE70B
:10E55000D6F86001D4F8D8200368B4F8DC10DB6882
:10E56000518398472B6801461B6828469847D4F882
:10E57000D830B4F8DC201A83CFE7036841F00201F9
:10E580009B699847BAE700BF1080002054280020FC
:10E5900070B50668F06982B00D461446002848D070
:10E5A000D0F80530DFED266A9FED267A07EE903A27
:10E5B000F8EE677A77EEE67AF3EE096A67EE877A25
:10E5C000B2EE047A67EEA67AF4EEC77AF1EE10FAAC
:10E5D00022DCBAEE047AF4EEC77AF1EE10FA1BD41C
:10E5E000D0F801302DB19FED187A67EE877AC5ED2E
:10E5F000007A7CB107EE903A9FED146ADFED146A61
:10E60000B8EE677ADFED137AE7EE067A77EEA67A50
:10E61000C4ED007A02B070BD17EE900A61F01EFCE6
:10E620000D4ACDE9000104210320FAF72BF902B0CD
:10E6300070BD09211420FAF71BFAF061B0E700BFA2
:10E6400000000046000080380AD778430319C83D0F
:10E6500033938843000048C21427080830B52DEDD5
:10E66000028B574C94F8AC31022B85B019D0DFEDFA
:10E67000557A79B19FED547A9FED546ADFED546A73
:10E6800067EEA77A67EE877A87EE867A77EE267A44
:10E69000C1ED007A0AB14F4B136005B0BDEC028B9F
:10E6A00030BD94F850326BBB4B4B1B689B072DD58C
:10E6B000B4F9343200EE103AB4F93232B8EEC00A8E
:10E6C00007EE103A20EE000AB8EEC77AB4F93632F7
:10E6D000A7EE070A07EE903AF8EEE77AA7EEA70A48
:10E6E000B5EEC00AF1EE10FAC1DBB5EE400AF1EE6C
:10E6F00010FA5BD4F1EEC07AF4EE677AF1EE10FA1C
:10E70000B7D7B4E7344B1B68980704D4D4F84C321D
:10E71000D3ED347AADE7314D0DF10E00CDE90012A5
:10E7200028F0DAFDBDF80E30D5F8EC03DFED2C5AF9
:10E73000DFED2C6A9FED2C7A1B1A07EE903AF8EE6B
:10E74000E77AB0EE408A87EEA56ADDE90012A6EE10
:10E75000267AFDEEC77AB0EE470A17EE903A2033DC
:10E76000402B20D8F9F71AFEDDE900121F4BD4ED3B
:10E77000847A6C7CA3F144001D462C3B002C08BF1E
:10E78000034695ED007AD3ED056AA8EE407A37EEA0
:10E79000A60A20EE000AA7EE070AB5EEC00AF1EEBF
:10E7A00010FAA2DA63E79FED070ADFE7CDE900126E
:10E7B00063F03CF8DDE90012F0EE407A9CE700BF20
:10E7C0001080002000000000CDCC9C3F00409C4603
:10E7D00082E6C54733139043A0000010F8D1002013
:10E7E0000000C84235FA8E3CDB0FC93FF8D5002047
:10E7F00030B50C4D83B055F83030019183B107EE40
:10E80000901A93ED047A93ED030AF8EEE77A044642
:10E81000A7EE870A62F0FCFE55F834309B6818605A
:10E8200003B030BD386A0020F0B54D4E96F8483040
:10E8300083B03BB196F85152012D04465ED0022DB3
:10E840003ED00DB103B0F0BD012280210068454FDC
:10E85000FBF7A2F801223870FF212068FBF79CF833
:10E860002A46387029462068FBF796F896F8522217
:10E87000387091212068FBF78FF829463870012203
:10E880002068FBF789F82A463870FF212068FBF7DB
:10E8900083F82A46387080212068FBF77DF82946E6
:10E8A0000346012220683B70FBF776F82E4A387049
:10E8B0001268C6F85422012386F8513203B0F0BD25
:10E8C0000068284F01AA1321FCF7B6FF9DF8043019
:10E8D00038705B0725D1D6F85832002BB2D0224AC7
:10E8E000D6F85412126892B2521A9342AAD24FF03A
:10E8F000FF3200237A6086F85132A3E701AA00684C
:10E90000184F0021FCF798FF9DF804303870DA07A3
:10E91000E1D4154A02231268C6F8542286F851320F
:10E9200090E720682B4601AA1E21FBF7F7FFBDF8F0
:10E93000043002460B2120683A7001225CBAFBF7D2
:10E940002BF80A4B3870A4B2A3FB0434E40801226C
:10E9500000237C6086F8492086F8513272E700BFB8
:10E9600010800020481500204C270020CDCCCCCCB6
:10E97000F0B541F0010285B000212A4F2A4D2B4EFF
:10E980000446FBF709F83B68C6F85432287016E0D5
:10E99000A368DB070DF10F024FF0130120465EBFA5
:10E9A0000DF10F0293212046FCF7F2FE9DF80F3087
:10E9B000287013F007030ED1D6F858224ABB2379EA
:10E9C000012B18D0022BE3D09DF80F30002013F05C
:10E9D00007032870F0D001220B212046FAF7DCFF54
:10E9E00000220346114620462B70FAF7D5FF287007
:10E9F000012005B0F0BDA268617C94F9100002F01E
:10EA0000010201920DF10F0200921322F5F752FE5E
:10EA1000CCE73968D6F8540289B2091A8A42CED2B4
:10EA20001846E6E74C2700204815002010800020FB
:10EA300010B5174C84F85110017984F8522001293F
:10EA40004FF0000282B084F8502012D002290CD17D
:10EA5000032304F15002FF21FBF792FE002814BFAC
:10EA600000206FF00C0002B010BD6FF00C0002B07F
:10EA700010BD8268417C90F91000503402F0010210
:10EA8000CDE900420323FF22F5F748FEE6E700BF89
:10EA90001080002000680379012B0BD0022B08D1D5
:10EAA00083680F4A13F0010316D000235121FBF7AE
:10EAB00067BE704700B58368094A417C90F9100031
:10EAC00083B003F00103CDE9002300235122F5F7C1
:10EAD00025FE03B05DF804FBD121FBF751BE00BF5A
:10EAE0006C82002030B5184D95F84A3083B00BB9D0
:10EAF00003B030BD04460DF1050100685FF0D6FE9D
:10EB00009DF8053073B901212068104A85F852102C
:10EB10004FF406440323FF21A5F85040FBF786FE7F
:10EB200003B030BD0DF1060296212068FFF784FC8A
:10EB3000074ABDF806300749A2FB0323DB08012280
:10EB40008B6085F84B20DEE710800020608000207D
:10EB5000CDCCCCCC4815002030B5044600680379F4
:10EB6000012B85B029D0022B1ED1826812F0010F33
:10EB700018BF512103AA08BFD121FBF779FE98B134
:10EB8000BDF80C30194A5BBA9BB2D360D368B3F5B9
:10EB9000C87F0EDC1649174AD1F85C32156832334B
:10EBA000AB4218D305B030BD104B6FF00102DA60F4
:10EBB000F0E74FF0FF33D360ECE78368417C90F9D6
:10EBC000100003F00103019303AB009351220223D1
:10EBD000F5F770FDD3E701F51772C1F85C522068B4
:10EBE00000235121FBF722FE05B030BD481500205F
:10EBF000108000204C27002000B500680379012B0D
:10EC000085B008D0022B2FD0204B002283F8502152
:10EC100005B05DF804FB8368417C90F9100003F0B7
:10EC2000010303AACDE9002302230022F5F742FDE8
:10EC3000164B83F850010028EAD0BDF80C305BBABF
:10EC40009BB2B3F5FA6F1AD21149124AA1FB031312
:10EC5000DB0807EE903AF8EEE77AFDEEE77AC2EDD0
:10EC6000047A05B05DF804FB826812F0010F18BF4A
:10EC7000002103AA08BF8021FBF7FAFDD8E7054B66
:10EC80004FF0FF321A6105B05DF804FB10800020E0
:10EC9000CDCCCCCC4815002010B500680379012BF1
:10ECA00084B00C461DD0022B18D1826812F0010FDF
:10ECB00014BF0021802103AAFBF7DAFD60B15CB12B
:10ECC0009DF80D309DF90C20DB0903EB830302EB6B
:10ECD000820203EB4203238004B010BD002004B085
:10ECE00010BD8368417C90F9100003F0010301938B
:10ECF00003AB009300220223F5F7DCFC0028DED1F1
:10ED0000EAE700BF2DE9F843DFF8648004460F46C8
:10ED10001646002540F634092046202168F081FB84
:10ED20000446D0B103461C4613F8010B2028FAD044
:10ED30002046FAF78FFB4845A8BF4846B0F5617FEB
:10ED4000B8BF4FF46170A0F56170A8FB0030C00837
:10ED50004DB178703378013333700DB90125DBE79D
:10ED60002046BDE8F8833870337801333370F4E718
:10ED70001F85EB5130B583B005460846019160F020
:10ED800001FF0199044602462846FAF713F820B914
:10ED90002A5DA2F13001092902D8002003B030BD5C
:10EDA00022F02002413A192AF8D90134281903B077
:10EDB00030BD00BF10B4474C0023224692F9041026
:10EDC000012902F10C022AD00133052BF6D122468B
:10EDD000002392F90410032902F10C0235D001330B
:10EDE000052BF6D1002394F90420052A04F10C0424
:10EDF00041D00133052BF6D1374B5B68DB0351D48F
:10EE00000179A1F13403012B1BD901F0EF01A1F12C
:10EE10002000B0FA80F040095DF8044B70472F4A9B
:10EE200003EB430302EB8303D3F860320BB32C4BA9
:10EE300093F83D2093F83CC003799A4201D0634592
:10EE4000C5D101205DF8044B7047244A03EB43030E
:10EE500002EB8303D3F86032002BC4D0214B02793C
:10EE600093F83D1093F83C309142EAD09A42B9D1E0
:10EE7000E7E72246ADE7194A03EB430302EB8303BE
:10EE8000D3F86032002BB7D0174B027993F83D10BE
:10EE900093F83C309142D4D09A42D2D00E4B5B686A
:10EEA000DB03ADD5114C224600231179212902F153
:10EEB000140207D001330C2BA2D01179212902F1C1
:10EEC0001402F7D103EB8303026854F823309A420B
:10EED00096D1B6E770820020A000001010800020BC
:10EEE000200300206C050020B8070020040A002041
:10EEF0000D4B10B503F1F00C4FF0000E02E014338F
:10EF00009C450FD01A688242F9D1DA688A4218BF4C
:10EF1000D9600EF1010403F1140318BF5FFA84FEF7
:10EF20009C45EFD1704610BD040A00202DE9F04F3A
:10EF30003D4EDFF80091DFF800813C4D83B04FF08B
:10EF4000000B0190B2465F46DAF8004040460021CF
:10EF500001E055F83100844203D001310E29F8D187
:10EF6000FF21494491F8A012012944D0022909D176
:10EF7000DAF80C10480705D521F0040141F008012A
:10EF8000CAF80C105046FFF715FF48B9264B0BEB9B
:10EF90008B0103EB8101C96801F00C00042835D016
:10EFA0000BF1010BBBF10C0F0AF1140ACCD1204C70
:10EFB0003046FFF7FFFEC0B9F368590703F00C02B3
:10EFC00013D5042A11D07A1CD5B2019A23F0080077
:10EFD00040F00400BA42014623F004031ED9F06059
:10EFE0003068FFF785FF2844C7B21436B442DFD13A
:10EFF00003B0BDE8F08FDAF80C100B07C2D521F092
:10F00000080141F00401CAF80C10BBE72046FFF7E5
:10F010006FFF0137FFB20744FFB2C1E73068F3600A
:10F020001946FFF765FFE0E7040A00201486070889
:10F03000F40A0020108000200000014038B504468A
:10F04000BDF810502160084619B11946F3F7E8FEE3
:10F0500020682946F3F760FF236859680B68B3F806
:10F0600044206FEA42426FEA524292B2A3F844202F
:10F070001A8892B242F001021A804A79032A17D8FC
:10F08000DFE802F0110C070240330022A3601A608F
:10F0900038BD3C330022A3601A6038BD38330022EB
:10F0A000A3601A6038BD34330022A3601A6038BDF3
:10F0B0000023A3601B60FFDE2DE9F04F85B00646FC
:10F0C000BDF838A09DF83CB0894617469846F3F73E
:10F0D00033FE0546002842D0274A92F8AE42092C5A
:10F0E00038D804EB440302EB43130021C3F8B012F9
:10F0F00083F8B412631CDBB282F8AE3204EB440432
:10F1000002F52C723079039302EB4414FDF794FD61
:10F1100050B3039B80F8069002210372C1710390E3
:10F12000BBF1000F12D11121FAF7BEFD039A13684B
:10F1300092885A832046CDF800A043463A46294695
:10F14000FFF77CFF204605B0BDE8F08F327AFDF76F
:10F1500077FFEFE7094A00210420F9F793FB002429
:10F16000204605B0BDE8F08FBBF1000FE2D11121C0
:10F17000FAF79AFDDEE700BF108000203827080864
:10F180002DE9F0473E4D95F8703682B03BB93D4AC7
:10F190000221042002B0BDE8F047F9F773BB95F8EF
:10F1A000717695F872360137FF1A102F0DDD102396
:10F1B0000221009385F87316334A3B460021042050
:10F1C000F9F760FB02B0BDE8F08795F87C36012BBB
:10F1D000064611D0022B0BD15FF05AF82B4BC5F825
:10F1E000803695F87C1611F0FD040BD0284ACFE745
:10F1F000284BC5F88036F4E75FF04AF8264BC5F88F
:10F200008036EEE77368BB422FDB002FDADDDFF8D4
:10F210009880DFF898A0DFF884902C3604E0013461
:10F22000BC4248F8040BCDD0DAF80430B5F87416B7
:10F230000091C3F300720192B5F87636174AB9FB14
:10F24000F3F356F8040F9BB20321FFF735FF0028B4
:10F25000E5D1134A052601462346042085F8736646
:10F2600002B0BDE8F047F9F70DBB042000930D4A4A
:10F2700085F873063B462146F9F704FBA2E700BF79
:10F2800010800020742708089027080871E3000800
:10F290001C2808085DE300084114030840420F00E1
:10F2A000F4270808BC27080818800020A0000010D8
:10F2B00030B503682C4C2DED028BA34283B0F0EEE9
:10F2C000408AB0EE608A13D004F58064A3420FD068
:10F2D00004F57054A3420BD004F58064A34207D018
:10F2E00004F58064A34203D0204B1C68640801E04D
:10F2F0001E4B1C680192B4FBF1F202F57F42002321
:10F30000FF32120C0093B4FBF2F4B4FBF1F5224689
:10F31000ABB20221FFF7D0FEC0B1B5EE408AF1EEEC
:10F3200010FA17D007EE904AF8EE677A27EE888A2F
:10F330009FED0F7AC8EE076A0123037127EE667A04
:10F34000C0ED046AA8EEA77A80ED037A03B0BDECA5
:10F35000028B30BD07EE905AB8EE678A07EE904AEE
:10F36000F8EE677AE4E700BF00000140F40A0020ED
:10F3700000007A442DE9F04F2DED028BA74B93F856
:10F380000080B8F10C0F9BB000F30D81A44BA54D8C
:10F390009B792B70032B20D91A1F022A00F2FC80C4
:10F3A000052B00F02D81062B0CBF4FF47A544FF43F
:10F3B0007A649D4A9D49DFF8C8C2039216469C4A6A
:10F3C000C6F884260027002200264A60CCE90067A0
:10F3D000984AB2FBF4F20A6005E0934A03921146A0
:10F3E000954AC1F88426954A12F81330002B00F094
:10F3F0000A8103684345C0F26981B8F1000F00F04B
:10F400009F80DFF88092DFF880A29FED8D8A00F167
:10F41000040B0027D9F804202B785BF8046FC2F3A3
:10F420000072062B00F2DA80DFE803F0A99C8F76E9
:10F4300004040400052B00F0CF8082498248062B8B
:10F4400008BF01460024019200940A4614230221B9
:10F450003046FFF731FE0290002800F0BA807B4B67
:10F4600031681A787A4E22B9AAE00134944200F049
:10F47000A7802301F3589942F7D1E2B21301049314
:10F480000298744C016806914FF4907303FB02429A
:10F490000B68D1F804C05C6E049BC265F318DCF8FD
:10F4A0000000079205949A60002C00F0EF80B0F8FD
:10F4B0004430694A6FEA43436FEA53439BB2A0F872
:10F4C000443003889BB243F0800303809CF80630ED
:10F4D00013F0040F9CF80530D15C028C14BF042398
:10F4E00001238B409BB292B222EA03020284028C77
:10F4F00092B21343038403889BB243F00103038059
:10F50000059B002B00F0F980029A01231371029BE6
:10F510004AF83730FB000BE0414BDFED500A998889
:10F52000B0EE600A3046FFF7C3FE4AF83700FB0032
:10F530005AF80330002B54D00137B8457FF46AAF36
:10F540001BB0BDEC028BBDE8F08FDFED450A9FEDEF
:10F55000450A30464FF4FA61FFF7AAFEFB004AF86D
:10F560003700E5E7DFED400A3046B0EE600A4FF4C1
:10F570007A71FFF79DFEFB004AF83700D8E79FED50
:10F58000300AF0EE480A30464FF4C871FFF790FE9B
:10F59000FB004AF83700CBE7234A03921146334A6F
:10F5A000C1F884261FE72049314A0C23012000932B
:10F5B00081F87306434600210420F9F763F9BFE799
:10F5C00013010493F1502149531C072A0B707FF655
:10F5D00057AF002302939AE7264933E700234AF8FE
:10F5E0003730039C244A052084F873063B460021EB
:10F5F00004201BB0BDEC028BBDE8F04FF9F742B917
:10F600004FF4FA54D5E61D4A022104201BB0BDEC8C
:10F61000028BBDE8F04FF9F735B900BF9800001034
:10F62000006C0020ED69002010800020F8690020A7
:10F6300089E3000840420F00F1E70008D48607087C
:10F640006F12833AC0C62D00001BB700986A0020D5
:10F650009C6A002098860020B08607080000000001
:10F66000ACC5A737ACC5A7366F12033959E30008FC
:10F6700058280808808D5B00E028080884280808BE
:10F68000006A0020A0000010386A0020DCF810306A
:10F69000484C059A190B1B0ACDE908C008469C4640
:10F6A000530104EB421EE35880EA13318CEA132322
:10F6B00001F0030103F00F030B4302F1010211D02B
:10F6C000102AEDD1069A0023D36020E70398009317
:10F6D000032180F87316384A434600210420F9F7C5
:10F6E000D1F82DE7069BC3F80CE09EF81C30DDE94D
:10F6F00008C0002B3FF4DBAE09E7069B069CD868E8
:10F700002E4B42682E499A422E4A136B0CBF43F48B
:10F71000001343F4800313630723838303222346E8
:10F72000F3F768FEE3689868F4F78CF8E3686268BA
:10F7300098680799036823F0010303601368127C3B
:10F740000D914C330C93204B53F822300B93002334
:10F75000CDE91633CDE918331093149312230F9388
:10F760004FF4806311934FF4804C4FF48053CDE9F4
:10F77000123C40230E930BA94FF4003315935DF018
:10F78000E5FB2246E4680499A368106806923144B8
:10F7900056681A6842F010021A60446674790B4A7F
:10F7A00032F81420A0F868208A81069A4B60012361
:10F7B0001374A9E6F80A0020A42808080060024093
:10F7C000A102000800380240B4860708BC8507087B
:10F7D00010B5104CD4E90423A16882B002FB03F3F6
:10F7E0008B428DF8070012D06368E0680DF10701C5
:10F7F000184464F019FD63682269A16813446269C2
:10F80000B3FBF1F0013201FB10336360626102B0BF
:10F8100010BD00BF106A002010B51420FDF70CFACF
:10F8200090B1044601214FF40873C3800172FAF7C6
:10F830003BFA2168114BA0884883002283F88C2F63
:10F84000C3F8884F83F88D2F1520FDF7F5F904468E
:10F8500090B14FF408720223C28003720121FAF7BB
:10F8600023FA2168054BA0884883002283F8942F4F
:10F87000C3F8904F83F8952F10BD00BF1080002073
:10F8800010B50379012B84B00C4621D0022B1DD179
:10F890008368DB070DF10F024CBF01218121FBF7CB
:10F8A00077FF9DF80F30114A1070C3F3C002C3F305
:10F8B000001CC3F38001A270C3F38012DB0984F83B
:10F8C00000C06170E270237104B010BD0020E8E751
:10F8D00082680DF10F0102F00102CDE900121A4613
:10F8E000417C90F91000F4F7E5FEDAE748150020B6
:10F8F0002DE9F04383B014460F4601AA5021054676
:10F90000FBF79AFF9DF804303C4EDFF8F49030701E
:10F9100001335B00DBB201AA238046212846FBF7B6
:10F920008BFF2378DFF8DC80307009FB03F303F5ED
:10F93000FA73A8FB03239DF8042099090132DB091F
:10F9400002FB0133A280A8FB03239B0901AAE36009
:10F95000512102232846FAF7E1FF2378BDF804106D
:10F96000307009FB03F349BA03F5FA73A8FB0323CC
:10F97000CAB2C1F307218A40013292B29909DB0968
:10F9800002FB0133E280A8FB03239B09238201AA27
:10F9900070212846FBF750FF9DF80430307001338A
:10F9A0005B00DBB201AA6380712102232846FAF7CB
:10F9B000B5FFBDF80420F978307052BAD3B2C2F363
:10F9C0000722934001339AB2228119B1E388D31AF6
:10F9D0009AB22281A1780A4B0A4803FB01F101F592
:10F9E000FA71A0FB01139909DB0902FB0133A0FBAB
:10F9F00003239B09638203B0BDE8F0834815002010
:10FA0000002F3A00D34D62102DE9F043A84FA94CC6
:10FA1000DFF8A4828FB006464FF000094FF4FA7366
:10FA200009AA89210068C7F8583287F84890FBF77F
:10FA300003FF9DF82420207042F0010289213068E4
:10FA4000F9F7AAFF4A46207088213068F9F7A4FF29
:10FA50000122207080213068F9F79EFF012220707A
:10FA6000FF213068F9F798FF4A4620704946306810
:10FA7000F9F792FF09AA207091213068FBF7DCFEAC
:10FA80009DF82430207001224946306887F85232B0
:10FA9000F9F782FF4A462070FF213068F9F77CFFB2
:10FAA0004A46207080213068F9F776FF09AA207055
:10FAB00060213068FBF7C0FE9DF82420207042F0E2
:10FAC000120260213068F9F767FF202502232070B9
:10FAD00009AA442130688DF825508DF82490FAF752
:10FAE000A5FEFF22207001213068F9F755FF356827
:10FAF0002070012280212846F9F74EFF0122207054
:10FB0000FF212846F9F748FF4A4620704946284613
:10FB1000F9F742FF06222070FF212846F9F73CFF43
:10FB200009AA207083212846FBF786FE9DF8242031
:10FB3000207042F0040283212846F9F72DFF0722A6
:10FB40002070FF212846F9F727FF0122207081212C
:10FB50002846F9F721FF0122207080212846F9F775
:10FB60001BFF6B22207094212846F9F715FF4A46A7
:10FB7000207083212846F9F70FFFD8F80030207055
:10FB8000C7F8543214E0AB68DB0709AA4FF08301D1
:10FB900028465EBF09AA83212846FBF7F9FD9DF898
:10FBA0002430207083B9D7F85832002B40F00F83EF
:10FBB0002B79012B00F0FE82022BE4D09DF824303B
:10FBC00000202070002BEED0012283212846F9F777
:10FBD000E3FE09AA207092212846FBF72DFE0022A1
:10FBE0002070812128469DF82490F9F7D5FE062241
:10FBF0002070FF212846F9F7CFFE09AA2070832143
:10FC00002846FBF719FE9DF82420207002F0FB0225
:10FC100083212846F9F7C0FE01222070FF212846E3
:10FC2000F9F7BAFE0122207000212846F9F7B4FE48
:10FC300000222070FF212846F9F7AEFE0022207036
:10FC400080212846F9F7A8FE0623207007AAB021D4
:10FC50003068FAF763FE01222070FF213068F9F75F
:10FC60009BFE002220704F213068F9F795FE2C2270
:10FC700020704E213068F9F78FFE00222070FF219E
:10FC80003068F9F789FEB4222070B6213068F9F7A0
:10FC900083FE4FEAD918B8F1000F4FF0000520702D
:10FCA00018BF4FF00C0809F07F0EAC46012017E09A
:10FCB00010800020481500204C270020F44503F058
:10FCC000070317D011F81C2C42FA03F3DB070CF1E1
:10FCD000010105F1010548BF5FFA81FC302D12D00A
:10FCE000EBB20EAA02EBD301984503F0070200FA2B
:10FCF00002F2E3D911F81C3C013523EA0202302D4F
:10FD000001F81C2CECD1062307AAB0213068FAF7C1
:10FD10008DFD01222070FF213068F9F73DFE0022A1
:10FD2000114620703068F9F737FE00222070FF215D
:10FD30003068F9F731FE0022207009213068F9F7A8
:10FD40002BFE0022207010213068F9F725FE0022DA
:10FD5000207011213068F9F71FFE01222070242144
:10FD60003068F9F719FEFF22207025213068F9F775
:10FD700013FE0022207075213068F9F70DFE012274
:10FD80002070FF213068F9F707FE2C2220704E21E9
:10FD90003068F9F701FE0022207048213068F9F739
:10FDA000FBFD2946207020223068F9F7F5FD00227E
:10FDB0002070FF213068F9F7EFFD294620700922F5
:10FDC0003068F9F7E9FD0022207054213068F9F716
:10FDD000E3FD0422207031213068F9F7DDFD0322B4
:10FDE000207032213068F9F7D7FD8322207040213E
:10FDF0003068F9F7D1FD2522207046213068F9F7E7
:10FE0000CBFD0022207060213068F9F7C5FD00228B
:10FE1000207027213068F9F7BFFD0622207050219D
:10FE20003068F9F7B9FD0022207051213068F9F7E8
:10FE3000B3FD9622207052213068F9F7ADFD0822FB
:10FE4000207056213068F9F7A7FD2A462070572107
:10FE50003068F9F7A1FD0022207061213068F9F7C0
:10FE60009BFD0022207062213068F9F795FD002289
:10FE7000207064213068F9F78FFD00222070652121
:10FE80003068F9F789FDA022207066213068F9F703
:10FE900083FD01222070FF213068F9F77DFD3222B9
:10FEA000207022213068F9F777FD14222070472155
:10FEB0003068F9F771FDFF22207049213068F9F7A9
:10FEC0006BFD002220704A213068F9F765FD0022A1
:10FED0002070FF213068F9F75FFD0A2220707A2137
:10FEE0003068F9F759FD002220707B213068F9F75E
:10FEF00053FD2122207078213068F9F74DFD012251
:10FF00002070FF213068F9F747FD3422207023214B
:10FF10003068F9F741FD0022207042213068F9F77E
:10FF20003BFDFF22207044213068F9F735FD262281
:10FF3000207045213068F9F72FFD052220704621F9
:10FF40003068F9F729FD4022114620703068F9F732
:10FF500023FD062220700E213068F9F71DFD1A22BC
:10FF6000207020213068F9F717FD402220704321CE
:10FF70003068F9F711FD00222070FF213068F9F791
:10FF80000BFD0322207034213068F9F705FD44226F
:10FF9000207035213068F9F7FFFC01222070FF2125
:10FFA0003068F9F7F9FC0422207031213068F9F744
:10FFB000F3FC092220704B213068F9F7EDFC052293
:10FFC00020704C213068F9F7E7FC042220704D21A5
:10FFD0003068F9F7E1FC00222070FF213068F9F762
:10FFE000DBFC0022207044213068F9F7D5FC202288
:10FFF000207045213068F9F7CFFC08222070472196
:020000040801F1
:100000003068F9F7C9FC2822207048213068F9F7D8
:10001000C3FC0022207067213068F9F7BDFC042280
:10002000207070213068F9F7B7FC0122207071212F
:100030003068F9F7B1FCFE22207072213068F9F7C0
:10004000ABFC0022207076213068F9F7A5FC002275
:10005000207077213068F9F79FFC01222070FF2182
:100060003068F9F799FC012220700D213068F9F70A
:1000700093FC00222070FF213068F9F78DFC0122EB
:10008000207080213068F9F787FCF8222070012168
:100090003068F9F781FC01222070FF213068F9F700
:1000A0007BFC012220708E213068F9F775FC01225B
:1000B000207000213068F9F76FFC00222070FF21CA
:1000C0003068F9F769FC0022207080213068F9F768
:1000D00063FC042220700A213068F9F75DFC356862
:1000E000207009AA84212846FBF7A6FB9DF824204E
:1000F000207002F0EF0284212846F9F74DFC01221E
:1001000020700B213068F9F747FC05A92070306892
:100110000390FFF7B5FB039809AA05A9FFF7E8FBD1
:100120009DF81430002B65D00C9B03F684539DF88A
:100130001620002A55D00C9A02F2B22203EB420399
:100140009DF8172022B1BDF8342002F52572134422
:100150009DF8182022B1BDF8362002F22622134461
:1001600001213068C7F8A83FE822F9F715FCD7F855
:10017000A81F207044F61F639942306802D95EF0D0
:10018000CFFB306801221146F9F706FC40212070B0
:100190003068FEF7EDFB50B1012130680222F9F71B
:1001A000FBFB002120703068FEF7E2FB28BB0FB09C
:1001B000BDE8F083AA68697C95F9100002F001029D
:1001C000019209AA00928322F4F774FAE7E4D8F8BE
:1001D0000020D7F8541292B2521A9342BFF4E8ACFE
:1001E000E5E79DF81520002AAAD00C9A02F52572A1
:1001F0001344A5E740F6363399E7E8220121306839
:10020000F9F7CAFB002502234FF0200C09AA207041
:10021000442130688DF825C08DF82450FAF706FB8C
:10022000D6F80080207005A94046FFF729FB09AAEF
:1002300005A94046FFF75CFB502257214046F9F7DD
:10024000ABFB0822207056214046F9F7A5FB082297
:10025000207050214046F9F79FFBBDF834202070F4
:100260004FF47A7148F20E6301FB02337C4A9342E9
:1002700040F2F2807B4AA2FB03231B0C5A1E32F091
:10028000FF0309D02B465208013322F0FF019BB235
:100290000029F8D11B029BB21343C3F30722DBB240
:1002A0008DF810208DF8113004AA02235121404608
:1002B000FAF7BCFA0C9A20704FF47A7148F20E6388
:1002C00001FB0233684A934200F2C480654AA2FBF4
:1002D0000332120C013AD2B246214046F9F75CFBD8
:1002E000D7F8A81F207044F61F63994202D94046F0
:1002F0005EF016FB04AA01214046FBF79DFA02229C
:100300002070012140469DF81050F9F745FB00216F
:1003100020704046FEF72CFB2A4601214046F9F7A3
:100320003BFB3568207005A92846FFF7A9FA09AA02
:1003300005A92846FFF7DCFA482211462846F9F7B6
:100340002BFB0822207047212846F9F725FB0322C2
:10035000207032212846F9F71FFB07222070302138
:100360002846F9F719FB01222070FF212846F9F7EA
:1003700013FB2022207030212846F9F70DFB0022C4
:100380002070FF212846F9F707FB06222070702114
:100390002846F9F701FBBDF83610344A207046F6BE
:1003A00044034FF47A7000FB0133A2FB03239DF852
:1003B00017201B0B1AB1BDF82A2013449BB2002B47
:1003C00046D05A1E32F0FF0309D0002352080133F1
:1003D00022F0FF019BB20029F8D11B029BB213430C
:1003E000C3F30722DBB28DF810208DF81130712194
:1003F000022304AA2846FAF719FAD7F8A81F207092
:1004000044F61F63994202D928465EF089FA04AA8D
:1004100001212846FBF710FA02222070012128460C
:100420009DF81060F9F7B8FA002120702846FEF711
:100430009FFA324601212846F9F7AEFA64220123D9
:100440002070C7F8582287F848300FB0BDE8F08315
:100450001A46C8E7FF223FE72B462A4620E700BF9F
:100460001B0C0100950370F41B280D014963A413B4
:1004700010B5174C84F85110017952BAA4F85220E3
:1004800001294FF0000282B084F8502012D00229D6
:100490000CD1042304F15002FF21FAF771F900286E
:1004A00014BF00206FF00C0002B010BD6FF00C0004
:1004B00002B010BD8268417C90F91000503402F007
:1004C0000102CDE900420423FF22F4F727F9E6E711
:1004D000108000202DE9F04FA24FA34D06680021A7
:1004E0003C4685B0834685F84A105A37C4F12D0939
:1004F00005F1500A884615E0022A0FD1B26812F0C1
:10050000010F4FF0030352464FF0FF01304601BF89
:1005100003235246FF213046FAF732F9BC421AD083
:1005200014F8011F327985F8521009EB0403012AEF
:1005300085F8508085F85130DED1B368717C96F92A
:10054000100003F00103CDE900A3FF220323F4F719
:10055000E5F8BC42E4D14FF40743A5F850304023FE
:1005600085F8523052460323FF213046FAF75EF9F0
:1005700000238DF80E300DF10E0130465EF096F935
:100580009DF80E30002BF6D04FF40640A5F8500031
:100590000120764A85F852000323FF213046FAF7FE
:1005A00045F94FF40740714AA5F850000024032391
:1005B000FF21304685F85240FAF738F94FF40060D1
:1005C000A5F850000920694A85F852000323FF214D
:1005D0003046FAF72BF94FF43063A5F85030634AF0
:1005E00085F8524030460323FF21FAF71FF900280F
:1005F0007FD0DBF800600DF10E025E213046FDF782
:100600001BFFBDF80E30B3F5D77F00F0A38079D87B
:10061000512B75D040F29480AD2B00F09B80D62BEF
:1006200040F08A80212408BB0A224B213046FEF785
:10063000FFF90F2260213046FEF7FAF90D226321FF
:100640003046FEF7F5F9B82269213046FEF7F0F999
:1006500040F60D7278213046FFF70AFF40F60E6231
:100660007A213046FFF704FF002875D0DBF8000040
:1006700021215EF06BF8DBF800400DF10E02DE2167
:100680002046FDF7D9FEBDF80E309FED397AC3F351
:100690000903ADF80E3003EB8303DB0007EE903A5D
:1006A000F8EEE77A204667EE877A0623FCEEE77AD3
:1006B0004FF4D84417EE902A110E85F85210110C01
:1006C00052BA85F85310A5F85420FF215246A5F8D8
:1006D0005040FAF7ABF84FF407414023DBF8000035
:1006E000A5F8501085F8523052460323FF21FAF73F
:1006F0009DF885F84A0005B0BDE8F08F1E2BB5D1F6
:10070000142490E740F2E132934221D00AD940F21A
:100710008F42934203D040F291529342A6D14FF4BC
:10072000FA7480E740F2D922934211D040F2E122DC
:10073000934209D1642476E7602B3FF473AF95E7C9
:100740001D2BDBD10F246EE7B3F5E67FF2D08DE7EA
:10075000C82468E7322466E7214630465DF0F6FF9C
:1007600084E700BF788D070810800020608000209B
:100770009A99893F03682DE9F041DF691FB13B4633
:10078000BDE8F0411847002A164611DD04460D4623
:100790000E4400E023689B68204698470028F9D063
:1007A000236815F8011B1B6820469847AE42F1D11B
:1007B000BDE8F081DEE700BF224B1B6813F0100F8D
:1007C000214B03D0B3F8AC2F520717D493F8C62FA0
:1007D00002BB93F8D42FD3F8D03F52B143B120B12C
:1007E0001A689B88138370474BB31A689B8853839E
:1007F000704780F00100002BF1D1F9E793F8C62F84
:10080000B2B993F8D42FD3F8D03F002AECD1002B03
:10081000E6D17047D3F8C82F002AE9D058B19268C2
:10082000B3F8CC1F094BB3FBF1F35B1013607047B7
:10083000D3F8C82F22B1936800221A60704770471E
:10084000704700BF9C0000101080002040420F0045
:10085000BFF34F8F0549064BCA6802F4E0621343A9
:10086000CB60BFF34F8F00BFFDE700BF00ED00E09E
:100870000400FA0508B572B600224FF0FF3193006C
:1008800003F1604303F561430132082AC3F8801085
:10089000C3F88011F3D1FFF7DBFF00BF012108B5DA
:1008A0000846F4F79BF8FFF7E5FF00BF00B583B0FB
:1008B0000D49002200920091009B04330093009B9D
:1008C0001B68012B02D003B05DF804FB019201917B
:1008D000019B064904330193019B1A600B6883F363
:1008E00008884B689847FEE7502800400000FF1F2B
:1008F00010B4EFF31183102282F31288094C0A48D6
:1009000022684FF0E021013222608A69C0F8D82FB6
:100910000022C0F8DC2F0A69DBB283F311885DF88E
:10092000044B70474C2700201080002030B4EFF3B8
:100930001182102383F312884FF0E023D2B2996919
:10094000186910F4803F0D481EBF0121C0F8DC1F5C
:1009500099690B4B1D68D0F8DC3F82F31188094878
:1009600004684FF47A7202FB04F02B44401A002111
:10097000B0FBF4F030BCE3FB0201704710800020B4
:100980004C270020CC330020124B5B68C3F30803D4
:10099000FBB9EFF31183E3B930B40F4A0F4C4FF0BA
:1009A000E02C1168DCF8180013688B42F9D1D4F8F8
:1009B000D81F8142F5D30A4A15684FF47A7404FBB4
:1009C00005F20021101AB0FBF5F0E3FB040130BC86
:1009D0007047ABE700ED00E04C27002010800020BE
:1009E000CC33002090B170B5461EFFF7CDFF044612
:1009F0000D46FFF7C9FF031B61EB0502B3F57A7FD4
:100A000072F10003F5D3013EEFD270BD704700BF15
:100A100070B5006801220921F8F7BEFF6426FFF7D0
:100A2000B3FF04460D46FFF7AFFF031B61EB050262
:100A3000B3F57A7F72F10003F5D3013EEFD170BDBB
:100A40002DE9804883B0431C0193DFF83C810A23E1
:100A50000093D8F89C10D8F8D830B8F8A000B8F8AF
:100A6000DC20DDF804B048834FF0320A1A834FF0DF
:100A700005094C69204214BF4883088359690A421A
:100A800014BF5A831A830120FFF796FE5646574635
:100A9000FFF77AFF04460D46FFF776FF001B61EB78
:100AA0000501B0F57A7F71F10003F5D3013FEFD175
:100AB000D8F89C30B8F8A02059690A4214BF5A836C
:100AC0001A83D8F8D830B8F8DC2059690A4214BF24
:100AD0005A831A830020FFF76FFEFFF755FF044685
:100AE0000D46FFF751FF001B61EB0501B0F57A7F62
:100AF00071F10003F5D3013EEFD1B9F1000F0BD036
:100B0000B9F1010910D0B8F8A000D8F89C10B8F8D5
:100B1000DC20D8F8D830ACE70BF1FF3BBBF1000F7D
:100B200019D04FF00009EEE74FF4FA76FFF72CFFEB
:100B300004460D46FFF728FF001B61EB0501B0F5E9
:100B40007A7F71F10003F5D3013EEFD14FF0FA0A3D
:100B5000BBF1000FE5D14FF47A76FFF715FF04469D
:100B60000D46FFF711FF031B61EB0501B3F57A7F1B
:100B700071F10003F5D3013EEFD1009B013B0093DF
:100B80007FF467AFFFF78AFE5428002018B103688E
:100B90001B6A03B118470020704700BF10B50C4610
:100BA00020B10368DB6A0BB1984768B9074B002096
:100BB000C4E90000C4E90200C4E906332D21302253
:100BC0002061217584F8202010BD00BF747D0808C5
:100BD0000178F9B1F8B5104F0546002602E015F886
:100BE000011FB1B1D7F8E04F637A5A1C2344D2B247
:100BF00062729972237A9342F1D8002AEFD004F1FD
:100C00000A01D4E900309847667215F8011F0029DF
:100C1000E8D1F8BD704700BF1080002070B50446D1
:100C20000F48FFF7D5FF2046FFF7D2FF0D48FFF72B
:100C3000CFFF0D4BB3F8E46F16B970BD013EFCD089
:100C4000FFF7A2FE04460D46FFF79EFE031B61EB75
:100C50000502B3F57A7F72F10003F5D3EEE700BF2A
:100C6000082908089C8808081080002030B583B047
:100C70000F4C01900F480091FFF7AAFFDDE9003209
:100C80000D49D4F8E00F5CF03BFBD4F8E05F6A7AE2
:100C900032B12B68686805F10A01984700236B722E
:100CA00094F8E63F13B1012384F8E73F03B030BD69
:100CB0001080002010290808B1E400080FB470B5B6
:100CC00082B006A951F8040B0191FFF7CFFF0E483F
:100CD000FFF77EFF0D4BB3F8E46F36B902B0BDE805
:100CE000704004B07047013EF8D0FFF74DFE044657
:100CF0000D46FFF749FE031B61EB0502B3F57A7F52
:100D000072F10003F5D3EEE79C88080810800020FC
:100D100000283DD00378002B3AD02DE9F04F87B062
:100D20005A4905AA64F08EFA0446002800F0A28011
:100D30004FF0000BDFF88091DFF88081DFF880A1B1
:100D40005D465F464FF0FF360BE0BBF1000F26D04B
:100D50004E4905AA002064F075FA0BF1010B044618
:100D600010B3BBF1010F15D0BBF1020FEDD1494615
:100D7000204666F0B0FB00286ED045F001054146E4
:100D8000204666F0A8FB00285FD045F00205DFE7AB
:100D90003F4893E72046F8F75DFB0746D8E7204633
:100DA000F8F758FB0646D3E770B23A4A002392F9A7
:100DB0000010814225D00133052B02F10C02F6D13F
:100DC000002F50D0002D08BF03250023EDB2CDE940
:100DD000015300971A4619462BF002FB04460028DF
:100DE0004ED02D48DFF8DC803A463146F7F714FD47
:100DF00031462A48F7F710FDD8F8540121465AF039
:100E000015F8DFF8C08003EB430308EB8303D3F846
:100E1000EC4F002CD4D022483146F7F7FDFC5DB1F1
:100E20006179A94208D01F482A46F7F7F5FC2368E4
:100E3000E9B29B6920469847E36A002BD8D01A484C
:100E4000F7F7EAFC0023E362D2E72046514666F05A
:100E500042FB002899D17BE71449204666F03BFB12
:100E600000288AD18BE712483146F7F7D5FC07B046
:100E7000BDE8F08F4FF0FF3025462746064694E741
:100E800031460C48F7F7C8FCF1E700BFFC7E0808C4
:100E9000102A0808F88F002070290808E02908089F
:100EA00090290808A8290808C8290808A84108089E
:100EB00028290808502908081C290808202908089A
:100EC0002429080810800020002868D02DE9F04F60
:100ED00090F800C085B00446BCF1000F2AD000F1A4
:100EE00000475A4E8646023F01466346722207E09B
:100EF000984526D1B94212D011F8013F16F8012FBA
:100F0000A3F14105192DA2F1410098BF2033192802
:100F100002F12008ECD99A4213D1002AEAD14C4CB4
:100F20000023C4F81C3E84F8233EA4F8243E05B0F8
:100F3000BDE8F08F0021012005B0BDE8F04F59F069
:100F4000CFBF444E214663466C2207E098452AD124
:100F5000B94212D011F8013F16F8012FA3F1410553
:100F6000192DA2F1410098BF2033192802F1200861
:100F7000ECD99A4217D1002AEAD1374B1B685B079C
:100F8000D5D4334C94F9223E002BD0D194F91D3E98
:100F9000002BC5DC05B0BDE8F04F51F0B9BF002112
:100FA000012059F09DBF2D48732307E065455BD1B3
:100FB000774513D01EF801CF10F8013FACF1410185
:100FC0001929A3F1410298BF0CF1200C192A03F151
:100FD0002005EBD9634547D1002BE9D11C4B0022FA
:100FE00093F9230E83F81C2E1C46164693F8CE1454
:100FF0000129A1F1030509D0052D07D90EB184F807
:10100000230E174805B0BDE8F04F57E693F8CF140C
:10101000A52903F1140303D00132782AE6D1EDE7C4
:10102000012803D0013840B20126F5E70D4984F8C4
:101030001C0E0023013284F81D2E01F8D43C84F8E4
:10104000233E05B0BDE8F04F4FF04CBD1C2A080808
:10105000F8D10020242A08089C000010183908083C
:10106000102A080808910020DFF880A22046F8F72F
:10107000F1F91AF9D47C07FA80F5772D064600F2CB
:10108000D1802046202166F0CCF98046002800F06F
:101090001C810346984613F8012B202AFAD04046BB
:1010A000F8F7D8F901245FFA80F94046202166F06C
:1010B000B8F98046002800F00D810346984613F8E1
:1010C000012B202AFAD04046F8F7C4F901340090E9
:1010D000E4B24046202166F0A4F98046002800F0E2
:1010E000F7800346984613F8012B202AFAD0404691
:1010F000F8F7B0F901340190E4B24046202166F0DF
:1011000090F98046002800F0BF800346984613F807
:10111000012B202AFAD04046F8F79CF901340290BE
:10112000E4B24046202166F07CF98046002800F0B9
:10113000A9800346984613F8012B202AFAD040468E
:10114000F8F788F901340FFA80FBE4B24046202119
:1011500066F067F90246002800F0B58003461A469B
:1011600013F8011B2029FAD010460392F8F772F900
:101170000134039A0FFA80F8E4B21046202166F099
:1011800050F9002856D003461A4601331178202919
:10119000FAD010460392F8F75DF9039A03461BB2A2
:1011A00010462021039366F03CF9039B002800F0D1
:1011B000938002461046013201782029FAD0039329
:1011C000F8F748F904F0FD04042C039B08BFC2B2F1
:1011D0007FF417AFB9F1010F04D9A9F10301052973
:1011E0003FF60FAF22B1A52A2FD0482A7FF409AFCE
:1011F0003DB33B4905EB850501EB850181F8CE94B4
:101200000098C1F8BC040198C1F8C0040298C1F864
:10121000C404A1F8C8B4A1F8CA84A1F8CC3481F8F8
:10122000CF2484E62F4930487723002205B0BDE85B
:10123000F04F43E55FFA88F203468046062CC9D09A
:10124000DFE6274981F8235ED8E7FDB9244C0099F1
:10125000C4F8BC140199C4F8C0140299A4F8CC34A1
:1012600084F8CE94C4F8C414A4F8C8B4A4F8CA840A
:1012700084F8CF24012301373E440AF8D46C84F863
:10128000233E54E6834661E702904AE7144C0098F7
:1012900005EB850504EB8501A1F8CC3494F8233ED9
:1012A000C1F8BC040198C1F8C0040133029881F868
:1012B000CE94C1F8C404A1F8C8B4A1F8CA8481F8D6
:1012C000CF245BB2D7E7804657E704468146ECE679
:1012D000019012E70090FCE60134E4B20246ADE76B
:1012E000F8D100202C2A0808382A08080891002084
:1012F0002DE9F04782B03E4901AA63F0A3FF002820
:1013000072D04FF0000A4FF0FF34394DD1465646A7
:10131000D0462746BAF1040F09D8DFE80AF0443E68
:10132000380E03000378482B46D0562B41D0314865
:10133000FFF7C4FC02B0BDE8F087F8F78BF83F2850
:101340000646F4D8002001AA294663F07BFF0AF183
:10135000010A0028DED1BAF1040F3AD02FDDBAF12C
:10136000050FE4D1244AB30103F47C6308F03F087D
:1013700043EA0803B9F1000F01D043F4005393216D
:1013800001FB074402EB440424F8D03CD2E7F8F711
:1013900061F83F288046D5D9C9E7F8F75BF892286D
:1013A0000446CFD9C3E7F8F755F803280746C9D94B
:1013B000BDE74FF00109C5E74FF00009C2E7BAF1F8
:1013C000020FB4DC0D4923463A46012059F00EFEC7
:1013D000B0E7094A932303FB074302EB430333F8C7
:1013E000D09CC9F34039BEE74FF0FF373C46E9E7F0
:1013F000FC7E0808102A0808089100203890002078
:1014000080B51948194DFFF7E3FB1948FFF7E0FBDA
:10141000D5F8E04F627A32B12146606851F80A3B54
:10142000984700236372D5F854713B6838465B696E
:101430009847B0B90A26FFF7A7FA04460D46FFF70A
:10144000A3FA031B61EB0502B3F57A7F72F1000387
:10145000F5D3013EEFD13B6838465B6998470028D9
:10146000E8D0012007F0C2FA582A080810800020AE
:10147000742A080830B42F4C94F8C833012B86B076
:1014800002D006B030BC704794F8CD330A2B04D09C
:10149000294806B030BCFFF79BBB41218DF80110F5
:1014A000264900231520097D8DF80200CDE903337C
:1014B000EB20CDE90133A6228DF803008DF804104E
:1014C000B22003218DF805008DF814308DF800202E
:1014D0008DF80610EC460DF1120541F2210083EA69
:1014E0000223082213F4004F80EA43010ABF5B0085
:1014F0008BB29BB2013AF5D1654502D01CF8012FA1
:10150000EDE7C3F307228DF814308DF81320EC4675
:101510001523C4F83834BCE80F00094D0FC59CE80A
:10152000030045F8040B0748297006B030BCFFF7EC
:101530004FBB00BF08910020802A080848150020F2
:10154000F0940020902A0808F8B52F482F4FFFF795
:101550003FFB2F48FFF73CFBB7F8E46F002E44D168
:10156000D7F8E04F627A32B12146606851F80A3B01
:10157000984700236372274B002583F83C54C3F837
:101580007C5483F8805422F0ADF82348FFF720FB09
:10159000D7F8E04F627A2AB12146606851F80A3BD9
:1015A00098476572D7F854713B6838465B6998472D
:1015B000B0B90A26FFF7E8F904460D46FFF7E4F94B
:1015C000031B61EB0502B3F57A7F72F10003F5D3DB
:1015D000013EEFD13B6838465B6998470028E8D068
:1015E000002007F003FA013EBAD0FFF7CDF9044618
:1015F0000D46FFF7C9F9031B61EB0502B3F57A7FCE
:1016000072F10003F5D3EEE7AC2A08081080002041
:101610009C88080808910020742A0808F8B5304909
:101620000522044665F012FF18BB2E4E96F8E63FE1
:1016300023B9012286F8E62F86F8E73F2A48FFF70C
:10164000C7FA2A48FFF7C4FAB6F8E46F16B9F8BD2E
:10165000013EFCD0FFF798F904460D46FFF794F9D8
:10166000031B61EB0502B3F57A7F72F10003F5D33A
:10167000EEE71F490322204665F0E8FE50BB194EF5
:1016800096F8E63F13B196F8E73FFBB91948FFF724
:101690009FFA1648FFF79CFAB6F8E47F3FB900239B
:1016A00086F8E63F86F8E73FF8BD013FF7D0FFF741
:1016B0006BF904460D46FFF767F9031B61EB050262
:1016C000B3F57A7F72F10003F5D3EEE70A48FFF72E
:1016D000F5FAE4E7BDE8F8400848FFF7EFBA00BFC5
:1016E000D82A080810800020E02A08089C880808EA
:1016F000184A0808302B0808F82A0808442B08085C
:10170000F8B52C4C94F8E63F1BB194F8E73F002B5A
:1017100044D1294D29480126FFF75AFA85F88764F4
:1017200085F8BC64F7F736FF254B85F8B2641B6873
:101730002448C5F89434002685F8BC6485F887648D
:10174000FFF746FAD4F8E05F6A7A02BBD4F8547126
:101750003B6838465B699847B0B90A24FFF714F92B
:1017600005460E46FFF710F9401B61EB0601B0F588
:101770007A7F71F10003F5D3013CEFD13B68384625
:101780005B6998470028E8D0002007F02FF9D5E9D9
:10179000003005F10A0198476E72D7E70A48FFF753
:1017A0008DFA0A48FFF78AFA002384F8E63F84F8A6
:1017B000E73FF8BD1080002008910020742B080836
:1017C0004C270020742A0808F82A0808542B080817
:1017D000F8B5284C284F012605462848FFF7F8F9A8
:1017E00005F010FF84F8876484F8BC64F7F7D2FE34
:1017F000234A2449126884F8B26400232846C4F8B6
:10180000942484F8BC3484F8873487F8E73FFDF7E4
:10181000B1FA00B1F8BD04461B48FFF7D9F9D7F873
:10182000E05F6A7A2AB1D5E9003005F10A019847EC
:101830006C72D7F854713B6838465B699847B0B909
:101840000A26FFF7A1F804460D46FFF79DF8031B93
:1018500061EB0502B3F57A7F72F10003F5D3013E27
:10186000EFD13B6838465B6998470028E8D00020F4
:1018700007F0BCF808910020108000207C2B08089D
:101880004C270020942B0808742A0808F8B5374B19
:101890001B68002B52D05B69984700284ED0344813
:1018A000344DFFF795F93448FFF792F93348FFF7C5
:1018B0008FF9B5F8E47F97BB3148FFF789F9D5F880
:1018C000E04F627A002A49D14FF47A77FFF75CF84B
:1018D00004460E46FFF758F8031B61EB0602B3F50A
:1018E0007A7F72F10003F5D3013FEFD1D5F85401AF
:1018F0002AF00EFE234B1A784AB12349384651F894
:1019000037300BB19B68186001379742F7D102213D
:101910000120F3F763F8FEF7ADFF013FCCD0FFF7EE
:1019200033F804460E46FFF72FF8031B61EB06025F
:10193000B3F57A7F72F10003F5D3EEE71348FFF7B2
:1019400047F90C4BD3F8E04F627A32B1D4E900305A
:1019500004F10A01984700236372F8BD23686068A8
:1019600004F10A01984700236372ADE7A02A002022
:101970000829080810800020A02B08089C88080867
:10198000742A080898000010386A0020C02B080844
:1019900070B50C48FFF71CF90B4BB3F8E46F16B9A0
:1019A00070BD013EFCD0FEF7EFFF04460D46FEF78A
:1019B000EBFF031B61EB0502B3F57A7F72F10003C5
:1019C000F5D3EEE79C88080810800020800601D53A
:1019D000002933D10CB470B5194C1A49D4F8E00F72
:1019E00082B007AB069A01935BF08AFCD4F8E05F03
:1019F0006A7A32B12B68686805F10A0198470023BA
:101A00006B721148FFF7E4F8B4F8E46F3EB90120B7
:101A100002B0BDE8704002B07047013EF7D0FEF75B
:101A2000B3FF04460D46FEF7AFFF031B61EB050253
:101A3000B3F57A7F72F10003F5D3EEE7002070472B
:101A400010800020B1E400089C880808F0B5044626
:101A500083B070B302785AB300F10040434D214681
:101A60000238722307E0974237D1884214D011F828
:101A7000012F15F8013FA2F1410EBEF1190FA3F19C
:101A8000410C98BF2032BCF1190F03F12007EAD9AD
:101A9000934222D1002BE8D1354B364AC3F8C024FB
:101AA000C3F8C424C3F8C824C3F8CC2403B0F0BDE1
:101AB0001446314D314E35F8241005EB840332467F
:101AC0005888CDE900100120234600210444FFF787
:101AD0007DFF042CEFD103B0F0BD2046F7F7BAFC30
:101AE000032805462FD82046202165F09AFC04469D
:101AF000002839D003461C4613F8012B202AFAD0BF
:101B00002046F7F7A7FC012706462021204665F06E
:101B100088FC034688B1184601330278202AFAD09F
:101B2000F7F798FC4FB1A6F2EE2240F2DC539A424E
:101B300003D8A0F2EE229A420ED9114803B0BDE8B4
:101B4000F040FFF7BBB80F490F480323002203B052
:101B5000BDE8F040FFF7B2B8054B03EB8505A5F8EB
:101B6000C064A5F8C204A1E70746CEE71C2A08080E
:101B700008910020E803D007C8950020F02B080842
:101B8000102A0808042C0808382A08082DE9F04310
:101B900087B040B3037807462BB300F10040564EA0
:101BA00039460238722207E09C4532D1814212D078
:101BB00011F8013F16F8012FA3F14105192DA2F1EB
:101BC000410498BF2033192C02F1200CECD99A4221
:101BD0001FD1002AEAD149486022002107B0BDE8A0
:101BE000F04364F0BFBC454D454F0024D5E90106E4
:101BF00015F80C1B0091CDE90106012023463A4659
:101C000004440021FFF7E2FE082CEFD107B0BDE845
